:1080000040520020DDF00100F5F00100F7F0010022
:10801000F9F00100F9F00100F9F0010000000000A2
:10802000000000000000000000000000F9F0010066
:10803000F9F0010000000000F9F00100BBA0000011
:10804000F9F00100F9F00100F9F00100F9F0010088
:10805000F9F00100F9F00100FF9C0000F9F00100C7
:10806000F9F00100F9F00100F9F00100F9F0010068
:10807000F9F00100F9F00100F9F00100F9F0010058
:10808000F9F00100F9F00100F9F00100F9F0010048
:10809000F9F00100F9F00100F9F00100F9F0010038
:1080A000F9F00100F9F00100F9F00100F9F0010028
:1080B000F9F00100F9F00100F9F00100F9F0010018
:1080C000F9F00100F9F00100F9F00100F9F0010008
:1080D000F9F00100F9F00100F9F00100F9F00100F8
:1080E000F9F00100F9F0010000000000F9F00100D2
:1080F000F9F00100F9F00100F9F00100F9F00100D8
:10810000F9F00100F9F00100F9F00100F9F00100C7
:108110000000000000000000F9F00100F9F001008B
:10812000F9F00100F9F00100F9F00100F9F00100A7
:10813000F9F00100F9F00100F9F00100F9F0010097
:10814000000000000000000000000000000000002F
:10815000F9F00100F9F00100F9F00100F9F0010077
:10816000000000000000000000000000000000000F
:1081700000000000000000000000000000000000FF
:1081800000000000000000000000000000000000EF
:1081900000000000000000000000000000000000DF
:1081A00000000000000000000000000000000000CF
:1081B000F9F00100F9F00100F9F00100F9F0010017
:1081C000F9F00100F9F00100F9F00100F9F0010007
:1081D000F9F00100F9F00100F9F00100F9F00100F7
:1081E000F9F00100F9F00100F9F0010000000000D1
:1081F00000000000F9F00100F9F00100F9F00100C1
:10820000F9F00100F9F0010000000000000000009A
:10821000F9F00100F9F00100F9F00100F9F00100B6
:10822000F9F00100F9F00100F9F00100F9F00100A6
:10823000F9F00100F9F00100F9F00100F9F0010096
:10824000F9F00100F9F00100F9F00100F9F0010086
:10825000F9F00100F9F00100F9F00100F9F0010076
:10826000F9F00100F9F00100F9F00100012000210E
:10827000DFF8542BC2E900010020DFF8501B086032
:10828000704738B501F07FFC002840F0FB81DFF833
:108290003C0B0068012805D101F0A5FBDFF8282B75
:1082A000C2E90001DFF8200BD0E9002301240025FA
:1082B000AB4204D1A24202D100F001FAECE1D0E9D4
:1082C0000023002B04D1022A02D100F091FAE3E14D
:1082D000D0E90023B3F5807F05D1002A03D1012026
:1082E00000F024FBD8E1D0E90023B3F5007F05D1ED
:1082F000002A03D1022000F019FBCDE1D0E90023D0
:1083000000240125AB4204D1A24202D100F0C6FAFA
:10831000C2E1D0E90023002B04D1042A02D100F0ED
:1083200072FBB9E1D0E90023002B04D1082A02D165
:1083300000F0B5FBB0E1D0E90023802B04D1002A86
:1083400002D100F021FCA7E1D0E90023002B05D1E8
:10835000102A03D1012000F06AFC9DE1D0E900233E
:10836000022B05D1002A03D1012000F0B7FD93E1D3
:10837000D0E90023002B05D1202A03D1022000F0F0
:1083800056FC89E1D0E90023042B05D1002A03D152
:10839000022000F0A3FD7FE1D0E90023002B05D1EE
:1083A000402A03D1032000F042FC75E1D0E900230C
:1083B000082B05D1002A03D1032000F08FFD6BE1CB
:1083C000D0E90023002B05D1802A03D1042000F03E
:1083D0002EFC61E1D0E90023B3F5005F05D1002A4E
:1083E00003D1042000F07AFD56E1D0E90023002BF0
:1083F00005D1B2F5000F02D100F0EAFC4CE1D0E962
:108400000023002B05D1B2F5800F02D100F0DDFD75
:1084100042E1D0E90023002B06D1B2F5801F03D141
:10842000012000F080FE37E1D0E90023002B06D1C7
:10843000B2F5001F03D1022000F075FE2CE1D0E957
:108440000023B3F5806F04D1002A02D100F0C1FEF1
:1084500022E1D0E90023202B04D1002A02D100F030
:1084600001FF19E1D0E90023B3F5006F04D1002A20
:1084700002D100F0F8FC0FE1D0E90023002B06D177
:10848000B2F5807F03D1002000F03EFF04E1D0E987
:1084900000235FF080740025AB4205D1A24203D1D6
:1084A000012000F031FFF7E0D0E9002300245FF065
:1084B0008075AB4205D1A24203D1002001F027F81C
:1084C000EAE0D0E9002300245FF00075AB4205D15B
:1084D000A24203D1012001F01AF8DDE0D0E9002327
:1084E00000245FF08065AB4205D1A24203D1022097
:1084F00001F00DF8D0E0D0E9002300245FF0006522
:10850000AB4205D1A24203D1032001F000F8C3E041
:10851000D0E9002300245FF08055AB4205D1A24290
:1085200003D1042000F0F3FFB6E0D0E900230024DB
:108530005FF00055AB4205D1A24203D1052000F007
:10854000E6FFA9E0D0E9002300245FF08045AB42BC
:1085500005D1A24203D1062000F0D9FF9CE0D0E96A
:10856000002300245FF00045AB4205D1A24203D1B5
:10857000072000F0CCFF8FE0D0E90023002B06D1CC
:10858000B2F5805F03D1002001F02AF884E0D0E941
:108590000023002B06D1B2F5005F03D1012001F0CA
:1085A0001FF879E0D0E90023002B06D1B2F5804F07
:1085B00003D1022001F014F86EE0D0E90023002B73
:1085C00006D1B2F5004F03D1032001F009F863E0B2
:1085D000D0E90023002B06D1B2F5803F03D104205F
:1085E00000F0FEFF58E0D0E90023002B06D1B2F5E1
:1085F000003F03D1052000F0F3FF4DE0D0E9002358
:10860000002B06D1B2F5802F03D1062000F0E8FF41
:1086100042E0D0E90023002B06D1B2F5002F03D1B0
:10862000072000F0DDFF37E0D0E90023402B05D123
:10863000002A03D1002000F0F5FE2DE0D0E9002350
:10864000B3F5805F05D1002A03D1012000F0EAFED6
:1086500022E0D0E90023002B05D1B2F5007F02D142
:1086600001F074F818E0D0E90023002B05D1B2F531
:10867000006F02D101F02AF80EE001220023C0E9C8
:10868000002309E001F06CFCDFF8CC1B0968401AFC
:10869000652801D301F06DFC082001F064FC31BDB8
:1086A00030B4DFF8B82BD2E9004520432943C2E9B2
:1086B000000130BC7047DFF8A81B0860704770B538
:1086C000DFF8380C0068002852D1DFF8344C29203C
:1086D000207001F0E7F960708820A0705320E070EE
:1086E000442020714B2060714520A0715620E0711C
:1086F0004F202072002060720020A0720020E072E3
:1087000000202073002060730020A0730020E0731D
:10871000002020740E2001F003FC60740F2001F093
:10872000FFFBA074FF20E074207560758420A075A5
:108730007B20E075002004E0002104EB00021176AC
:10874000401C1328F8D3042001F0F1FC002806D1C6
:10875000342084F82200312084F8230005E0302002
:1087600084F82200302084F8230001F066F83EE00F
:10877000DFF8904B200001F046FA012835D16078EF
:10878000BB2802D101F0F5FB31E0A078882829D17F
:10879000A07DE17D71F0FF01C94388421FD101F046
:1087A00012FD0A2694F8220001F040FE05007543F0
:1087B00094F8230001F03AFE55FA80F001F029FD0B
:1087C000607C01F033FE05007543A07C01F02EFEB5
:1087D00055FA80F001F020FD01F01EF807E001F0ED
:1087E0001BF804E000F0F3FF01E000F0FFFF70BDB4
:1087F00038B5DFF8080B006800280DD1DFF8004B12
:108800000520207001F04EF960702F20A07001F05B
:108810002AF801F012F840E0DFF8E84A200001F001
:10882000F2F9012837D16078BB2802D101F01FF995
:1088300033E0A078A12824D1DFF8205AD5E900013F
:1088400010F0000011F48071002907D1002805D133
:10885000A37962792179E07802F098F9D5E90001ED
:1088600010F0000011F40071002907D1002805D193
:10887000A37A627A217AE07902F09BF900F0CCFFCA
:108880000BE0F92804D100F0C7FF01F0F0F804E094
:1088900000F09DFF01E000F0A9FF31BD10B5DFF849
:1088A0005C0A0068002814D1DFF8544A07202070C1
:1088B00001F0F8F860705220A07000F0D4FF7F2023
:1088C00002F0ECF9E071E079C043207200F0B5FFEE
:1088D0002BE0DFF8304A200001F095F9012822D181
:1088E0006078BB2802D101F0C2F81EE0A07886288B
:1088F00004D100F0E8FF00F08FFF16E0F02808D167
:10890000E078522802D100F087FF0EE000F05FFF10
:108910000BE0F92804D100F07FFF01F0A8F804E093
:1089200000F055FF01E000F061FF10BD38B5040014
:10893000DFF8C8090068002836D1DFF8C4590A20DA
:10894000287001F0AFF868708720A870012C14D14E
:1089500000F0A6FF0120E871002002F04CF9287217
:10896000012002F048F96872022002F044F9A8726E
:10897000032002F040F9E87213E000F07EFF0220CD
:10898000E871002002F045F92872012002F041F957
:108990006872022002F03DF9A872032002F039F952
:1089A000E87200F04AFF2DE0DFF85859280001F086
:1089B0002AF9012824D16878BB2802D101F057F8A0
:1089C00020E0A878F02811D1E87887280BD1012C75
:1089D00002D102F0E3F803E0022C01D102F0F9F831
:1089E00000F01AFF0EE000F0F2FE0BE0F92804D1CF
:1089F00000F012FF01F03BF804E000F0E8FE01E0B7
:108A000000F0F4FE31BD10B5DFF8F0080068002872
:108A100023D1DFF8EC480E20207001F043F860709D
:108A20000620A0700020E0715FF0FF3001F07FFBB6
:108A30000100090E21720100090C61720100090A8E
:108A4000A172E07200202073002060730020A073E8
:108A50000020E07300F0F1FE20E0DFF8A8482000DD
:108A600001F0D1F8012817D16078BB2802D100F0BD
:108A7000FEFF13E0A078862804D100F024FF00F068
:108A8000CBFE0BE0F92804D100F0C6FE00F0EFFFAA
:108A900004E000F09CFE01E000F0A8FE10BD10B55F
:108AA000DFF858080068002812D1DFF854480E207B
:108AB000207000F0F7FF60700720A0700020E070C9
:108AC00002F04CFA2071000A607100F0B6FE5AE024
:108AD000DFF83048200001F096F8012851D1607885
:108AE000BB2802D100F0C3FF4DE0A07877283ED12B
:108AF000E078217910EB012002F084F96079A17906
:108B000010EB012002F093F9607AA17A10EB0120BA
:108B100002F093F9E07A217B10EB012002F078F962
:108B2000607BA17B10EB012002F07BF9E07B217CD4
:108B300010EB012002F087F9E07D00F0FF00217EBC
:108B400010EB012002F067F901F087FB01280BD13F
:108B5000E07E0006217F50EA0140617F50EA01205B
:108B6000A17F084302F03DFA00F056FE0BE0F92821
:108B700004D100F051FE00F07AFF04E000F027FE7F
:108B800001E000F033FE10BD10B5DFF8700700689B
:108B9000002824D1DFF868470D20207000F082FF04
:108BA00060708520A07000F05EFE02F060F90100A8
:108BB000090EE1710100090C21720100090A6172BC
:108BC000A072C0430100090EE1720100090C21737B
:108BD0000100090A6173A07300F02FFE26E0DFF8A0
:108BE0002447200001F00FF801281DD16078BB2830
:108BF00002D100F03CFF19E0A078F0280AD1E0781B
:108C0000852804D102F036F900F006FE0EE000F0EF
:108C1000DEFD0BE0F92804D100F0FEFD00F027FF97
:108C200004E000F0D4FD01E000F0E0FD10BD38B537
:108C30000400DFF8C806006800282ED1DFF8C0560F
:108C40000520287000F02EFF6870012C06D101204D
:108C5000A87000F008FE00F0F0FDB4E0022C02D194
:108C60000220A870F5E7032C02D10320A870F0E7DA
:108C700001F0F3FA012802D10420A870E9E7DFF837
:108C8000DC05D0E900235049D1E90045A243AB43BC
:108C9000C0E9002300F0C0FD95E0DFF86856280029
:108CA00000F0B1FF012840F08C806878BB2802D129
:108CB00000F0DDFE87E0A87884281CD1042C1AD1AE
:108CC000DFF89805D0E9000110F0000011F4005120
:108CD00000290DD100280BD1002407E005EB04008A
:108CE000C17814F1600002F0B8F9641C1F2CF5D3B0
:108CF00000F092FD67E083281CD1032C1AD1DFF825
:108D00005C05D0E9000110F0000011F00801002915
:108D10000DD100280BD1002407E005EB0400C17839
:108D200014F1400002F099F9641C1F2CF5D300F0F7
:108D300073FD48E082281CD1022C1AD1DFF81C05F3
:108D4000D0E9000110F0000011F0040100290DD15C
:108D500000280BD1002407E005EB0400C17814F1D2
:108D6000200002F07AF9641C1F2CF5D300F054FDAA
:108D700029E081281BD1012C19D1DFF8E004D0E9CA
:108D8000000110F0000011F0020100290CD10028B0
:108D90000AD1002406E005EB0400C178200002F0AF
:108DA0005CF9641C1F2CF6D300F036FD0BE0F928AB
:108DB00004D100F031FD00F05AFE04E000F007FDA0
:108DC00001E000F013FD31BDE01000204011002053
:108DD00010B586B0DFF82405006800280DD1DFF853
:108DE00020450720207000F05DFE60701320A07009
:108DF00000F039FD00F021FD33E0DFF808452000E8
:108E000000F001FF01282AD16078BB2802D100F0D0
:108E10002EFE26E0A0781F281ED1DFF84004D0E9FE
:108E2000000110F0000011F40061002911D10028A8
:108E30000FD1E07801F0DEF9002005E004EB00013D
:108E400009796A461154401C1828F7D3684601F086
:108E5000D7F900F0E1FC04E000F0B9FC01E000F01B
:108E6000C5FC06B010BD10B5DFF8900400680028FE
:108E700014D1DFF88C440720207000F013FE6070DE
:108E80007320A07000F00CFD01F0DBF9E07101F03F
:108E9000D8F9C043207200F0D0FC1EE0DFF8644433
:108EA000200000F0B0FE012815D16078BB2802D167
:108EB00000F0DDFD11E0A078F02802D100F0ACFC5C
:108EC0000BE0F92804D100F0A7FC00F0D0FD04E08D
:108ED00000F07DFC01E000F089FC10BD70B50400DD
:108EE000DFF818040068002834D1DFF81454242077
:108EF000287000F0D7FD6870012C02D18120A87085
:108F00000BE0022C02D18220A87006E0032C02D1D3
:108F10008320A87001E08420A87000F0C1FC012C1F
:108F200001D1002408E0022C01D1202404E0032C0C
:108F300001D1402400E06024002606E0301902F050
:108F400089F805EB0601C871761C1F2EF6D300F0D8
:108F500074FC39E0DFF8AC53280000F054FE01281F
:108F600030D16878BB2802D100F081FD2CE0A878D0
:108F7000E978F0281CD1012C03D10800C0B2812867
:108F800010D0022C03D10800C0B282280AD0032CD2
:108F900003D10800C0B2832804D0042C05D1C9B283
:108FA000842902D100F038FC0EE000F010FC0BE048
:108FB000F92804D100F030FC00F059FD04E000F085
:108FC00006FC01E000F012FC70BD38B5DFF82C03A0
:108FD000006800280DD1CA4C0220207000F062FD0C
:108FE00060700B20A0709E480068E07000F025FCC7
:108FF00098E0C44C200000F006FE012840F090806C
:109000006078BB2802D100F032FD8BE0A0788B287D
:109010007CD1934DE0782968884274D12179286801
:1090200002F00BF96179A07951EA0021E07951EA67
:109030000041207A51EA0061286802F08AF8627AD9
:109040000023A07A0021090241EA106100020243D4
:109050000B43E07A0021090441EA10410004024375
:109060000B43207B0021090641EA10210006024340
:109070000B43607C00210100002002430B43A07CD5
:1090800000210102002002430B43E07C0021010487
:10909000002002430B43207D0021010600200243F3
:1090A0000B43286802F06EF8617BA07B51EA002137
:1090B000E07B51EA0041207C51EA0061286802F01F
:1090C00076F86648D0E9000110F0000011F48061E4
:1090D000002909D1002807D1617D286802F0CBF86A
:1090E000A17D286802F071F8E27D0021286802F075
:1090F0008EF8227E0121286802F089F8002028607D
:1091000000F08AFB0EE000F062FB0BE0F92804D1CE
:1091100000F082FB00F0ABFC04E000F058FB01E043
:1091200000F064FB31BD70B504007448006800288D
:109130000BD1734D0220287000F0B4FC68700C2035
:10914000A870EC7000F079FB42E06E4D280000F052
:109150005AFD01283AD16878BB2802D100F087FC7B
:1091600036E0A978E8788C2926D1A04224D1287944
:10917000697910EB012001F0BCFFA879E97910EBC7
:10918000012001F0B3FF287A697A10EB012001F089
:10919000B3FF00260BE002F06EF807E0B01C05EB11
:1091A0000601897A012CF6D102F047F8761C0E2EC2
:1091B000F4D300F031FB0BE0F92904D100F02CFBD3
:1091C00000F055FC04E000F002FB01E000F00EFBB3
:1091D00070BD38B549480068002817D1484C0720B1
:1091E000207000F05FFC60708A20A0701C4D286821
:1091F000E070286802F029F820710020607128686A
:1092000001F0DAFFA07100F018FB23E03D4C2000D4
:1092100000F0F9FC01281BD16078BB2802D100F0D6
:1092200026FC17E0A078E178F02807D18A2902D13E
:1092300000F0F2FA0EE000F0CAFA0BE0F92804D1CF
:1092400000F0EAFA00F013FC04E000F0C0FA01E0DC
:1092500000F0CCFA31BD000048110020E8100020D9
:109260005411002010B525480068002820D1244C56
:109270000B20207000F016FC60708F20A07000F0B2
:10928000F2FA002002F01CF8E071012002F018F858
:109290002072022002F014F86072042002F010F82C
:1092A000E072052002F00CF8207300F0C6FA24E00A
:1092B000144C200000F0A7FC01281CD16078BB28CA
:1092C00002D100F0D4FB18E0A078E178F02808D1B2
:1092D000C9B28F2902D100F09FFA0EE000F077FAB0
:1092E0000BE0F92804D100F097FA00F0C0FB04E08D
:1092F00000F06DFA01E000F079FA10BD4411002091
:10930000100E0020900D0020FEB50400DFF870075D
:10931000006800280ED1DFF86C570620287000F096
:10932000C1FB68700D20A87000F09DFAEC7100F090
:1093300084FA76E0DFF85057280000F064FC01283A
:109340006DD16878BB2802D100F091FB69E0AA7862
:10935000E97F9D2A59D154EA0100002803D0002951
:1093600053D0002C51D0002C00D00624DFF81C076D
:10937000D0E9002312F0000213F04003002B41D18A
:10938000002A3FD1D0E9000110F0000011F4805113
:10939000002937D1002835D1EE78F00705D5002C0B
:1093A00003D1012001F0F4FF04E0002C02D10020E1
:1093B00001F0EEFF002723E000208DF8000006E01A
:1093C0000220B8400642F7D001208DF8000005EBDE
:1093D0008700C0798DF8010005EB8700007A8DF8D1
:1093E000020005EB8700407A8DF8030005EB87004B
:1093F000807A8DF804006946E01901F0F8FF7F1CBF
:10940000062FDDD300F008FA0BE0F92A04D100F0B2
:1094100003FA00F02CFB04E000F0D9F901E000F0C1
:10942000E5F9F7BDFEB50400DFF854060068002832
:1094300046D1DFF850562520287000F033FB6870C5
:109440009D20A87000F00FFA01F0A5FF012803D1BC
:10945000002C01D1012700E00027002C00D00624B9
:1094600000261FE06946A01901F0E3FF9DF8000007
:10947000002802D00220B04007439DF8010005EB10
:109480008601C8729DF8020005EB860108739DF8FD
:10949000030005EB860148739DF8040005EB860187
:1094A0008873761C0C2EDDD3EF710020287200200B
:1094B00068720020A87285F8234000F0BEF925E00C
:1094C000DFF8C445200000F09EFB01281CD1607825
:1094D000BB2802D100F0CBFA18E0A078E178F028A0
:1094E00008D1C9B29D2902D100F096F90EE000F032
:1094F0006EF90BE0F92804D100F08EF900F0B7FA0C
:1095000004E000F064F901E000F070F9F7BD7CB50B
:109510000400DFF86C05006800283BD1DFF86455D3
:109520002620287000F0BEFA68709020A87000F025
:109530009AF9EC71002628E06A463100200001F01B
:10954000D8FF9DF80000052101FB06F129440872AF
:109550009DF80100052101FB06F1294448729DF8A0
:109560000200052101FB06F1294488729DF80300E1
:10957000052101FB06F12944C8729DF8040005216C
:1095800001FB06F129440873761C062ED4D300F0A3
:1095900054F924E0DFF8F054280000F034FB0128EF
:1095A0001BD16878BB2802D100F061FA17E0AA78D5
:1095B000E8782979F02A06D1902804D1A14202D175
:1095C00000F02AF90BE0F92804D100F025F900F0A9
:1095D0004EFA04E000F0FBF801E000F007F973BD7B
:1095E0007CB50400DFF89804006800280ED1DFF88D
:1095F00094540620287000F055FA68701020A87066
:1096000000F031F9EC7100F018F95EE0DFF8785401
:10961000280000F0F8FA012855D16878BB2802D15B
:1096200000F025FA51E0A878902842D100205FF0A0
:109630008071220001F0A0FFDFF85024D2E900235E
:1096400010401940002931D100282FD1E8788442F8
:109650002CD1002628E0052000FB06F028440079E4
:109660008DF80000052000FB06F0284440798DF8B5
:109670000100052000FB06F0284480798DF80200E7
:10968000052000FB06F02844C0798DF80300052072
:1096900000FB06F02844007A8DF804006A46310089
:1096A000200001F0F1FE761C062ED4D300F0B4F8B1
:1096B0000BE0F92804D100F0AFF800F0D8F904E08D
:1096C00000F085F801E000F091F873BD10B5DFF807
:1096D000B003006800280DD1DFF8A84305202070F2
:1096E00000F0E0F960700E20A07000F0BCF800F00F
:1096F000A4F82AE0DFF89043200000F084FA012863
:1097000021D16078BB2802D100F0B1F91DE0A0782A
:1097100091280ED12079617950EA0120A17950EA8F
:109720000140E17950EA016001F03BFF00F074F87C
:109730000BE0F92804D100F06FF800F098F904E08C
:1097400000F045F801E000F051F810BD38B5CC4804
:10975000006800280CD1CB4C0520207000F0A2F945
:1097600060700F20A07000F07EF800F066F82DE029
:10977000C54D280000F047FA012825D16878BB289C
:1097800002D100F074F921E0A878782812D1E878A5
:1097900000F045FD287900F049FE04000A2044430A
:1097A000687900F043FE54FA80F000F03BFD00F0D1
:1097B00033F80BE0F92804D100F02EF800F057F947
:1097C00004E000F004F801E000F010F831BD80B5CD
:1097D000AF480168491C01600021A94A1160006876
:1097E0000B2802D3102000F09DFC01BD80B500F0D5
:1097F000B7FBA8490968401A65280CD30020A04986
:109800000860A5480168491C016000680A2802D365
:10981000102000F087FC01BD80B500209C49086045
:1098200000209D490860002095490860102000F044
:1098300073FC01209949086001BD38B5914800F0DA
:10984000A5F901208E49086000F08AFB9149086063
:109850008E48D0E900239249D1E90045A243AB43A9
:10986000C0E9002331BD87483321C1703121017126
:109870003021417131218171704710B5814C002038
:1098800001F0C0F9E070012001F0BCF92071022064
:1098900001F0B8F96071032001F0B4F9A07110BDB6
:1098A00010B5784C002001F09FF9E070012001F024
:1098B0009BF92071022001F097F96071032001F0FB
:1098C00093F9A07110BD38B56F4CE078000621798E
:1098D00010EB0140617910EB0120A179401801F0F3
:1098E0005DFEE07901F0F8FE627A00231B0643EA90
:1098F00012231206A07A0021090441EA1041000453
:1099000002430B43E07A0021090241EA10610002A0
:1099100002430B43207B002102430B43607B002169
:109920000102002002430B43A07B00210100002024
:109930001043194301F052FEE07C0006217D10EB3C
:109940000140617D10EB0120A17D401801F0C0FEB7
:10995000E07D0006217E10EB0140617E10EB0120CE
:10996000A17E401801F03AFB484DD5E9000110F006
:10997000000011F00101002905D1002803D1217F49
:10998000E07E01F068F9607F01F036FA94F820007B
:1099900001F02EFED5E9000110F0000011F02001C9
:1099A00000291FD100281DD194F82310002001F0B8
:1099B00083FC94F82410012001F07EFC94F825101B
:1099C000022001F079FC94F82610032001F074FCC9
:1099D00094F82710042001F06FFC94F8281005205B
:1099E00001F06AFC31BD38B52D48D0E9004500F0E2
:1099F00034FC002803D000F049FC012808D123489A
:109A0000D0E9002332F4000233F40063C0E90023FC
:109A10001E49D1E9002352F0040253F00003C1E9CA
:109A20000023002000E0401C40281AD200225FF0F2
:109A300000439D4206D801D3944203D2002D04D1A5
:109A4000002C02D10124002503E06D0045EAD47505
:109A50006400D1E9002322402B40002B01D1002AD1
:109A6000E1D000200D4908602000290034BD01200C
:109A700000210B4AC2E90001002008490860704734
:109A800044110020100E0020900D0020E81000204E
:109A900050110020481100204C11002040110020DE
:109AA000E010002080B50D2000F041FB002801D01F
:109AB000BB2000E0002002BD10B5BB4802F057F803
:109AC000BA4802F054F802F09DF9B94802F0ACF936
:109AD0000121B84802F0E5FA0120B7490860B7480B
:109AE000B7490860FF20B74908608021B64802F0F6
:109AF000D8FA8020B5490860B54802F0FCFAB548AC
:109B000002F0F9FA3021B44802F0E7FA02F0CDF899
:109B1000B24C60234FF461420100200002F010FBC0
:109B200010220221200002F007FBAD48016831F04D
:109B3000100101601021200002F055FB200002F00E
:109B40002DFB0321200002F05CFB162002F0E1F95E
:109B5000172002F0DEF9C021162002F060FB16206B
:109B600002F06EFB0F21162002F061F99D491620CC
:109B700002F074F90F21172002F059F99A491720C1
:109B800002F06CF910BD994800687047F8B50500FF
:109B90000127974E02203070002415E0285DC0B2E6
:109BA0000009C0B200F055FC06EB44014870285D86
:109BB00010F00F0000F04DFC06EB44018870002C03
:109BC00001D0285D3F18641C2878801C8442E5D3AE
:109BD000FF4307F0FF073800000900F03AFC06EBEE
:109BE0004401487017F00F07380000F032FC06EB14
:109BF00044018870032006EB4401C8706000001D1A
:109C000000F0BDF8F1BD2DE9F8430500002000E0AB
:109C1000401CB0F5807F06DA76490A5C032AF7D14A
:109C2000040000220A54B0F5807F01DA002C01D133
:109C3000002062E0671E00E07F1E002F5CD46D4EA6
:109C4000F05D0228F8D10020F055E41B641C083CAC
:109C5000E00701D5022050E06408201F792801D3D5
:109C600002204AE0781C00F0FF00411C01F0FF01D7
:109C7000715C305C00F0C2F828702878844201D012
:109C800002203AE05FF00108F81C00F0FF00411CE0
:109C900001F0FF01715C305C00F0B0F8687068782A
:109CA00018EB00085FF0000917E0781D10EB490081
:109CB00000F0FF00411C01F0FF01715C305C00F01E
:109CC0009DF805EB09018870A14504D205EB090058
:109CD000807858FA80F819F101094C45E5D27FEAFD
:109CE000080808F0FF0805EB04008078804501D0E3
:109CF000022002E0012000E00020BDE8F28310B560
:109D0000364C0121200002F073FA0100200002F01D
:109D100075FA36480068002807D1162002F0E5F8E9
:109D2000002808D100F008F805E0334800688006F4
:109D300001D500F001F810BD80B500202B49086066
:109D400000201D490860002020490860162002F00C
:109D500063F8002003E00021264A1154401CB0F5AE
:109D6000807FF8D34FF480700090224B1B4A012172
:109D7000162002F07FF8162002F049F801BD80B5E8
:109D800001211A4A11608021104A116001210A4AFA
:109D900011600090114B164A0121172002F06AF859
:109DA000172002F034F801BD011800F0000C00F09B
:109DB0000008002000400240044002404B434F4C4A
:109DC0002075004024750040007000400072004083
:109DD00002100200021402000060004000D00040A7
:109DE0002CD000400080000C008000C03C110020FE
:109DF000A00B0020A00A00203CD0004038B50C0089
:109E0000C0B200F013FB05002D012000C0B200F02D
:109E10000DFB45192800C0B232BD30B4002513E057
:109E200050F8042BD30744BFA9F101039A18091F66
:109E3000042942F8045BFAD213468C0744BF15800C
:109E40009B1CC90748BF1D7050F8041B0029E7D1AF
:109E500030BC70471CB59B4C10221021200002F032
:109E6000A7FA2078532826D16078442823D1A078F7
:109E70004B2820D1E07845281DD1207956281AD1C9
:109E800060794F2817D1A079002814D1E0790028F3
:109E900011D1207A00280ED1607A00280BD1A07A47
:109EA000002808D1E07A002805D1207B002802D1C3
:109EB000607B002803D0082000F034F902E008207D
:109EC00000F02AF904220A21684602F071FA0420FF
:109ED00000F02DF900280DD000208DF800000020A2
:109EE0008DF8010004220A21684602F076FA002863
:109EF000F8D114E09DF80000342803D19DF801004A
:109F000031280CD034208DF8000031208DF801006C
:109F100004220A21684602F060FA0028F8D113BD35
:109F20006849085C704710B504005FF0804002F09B
:109F3000DDFA012803D15FF0804002F0CFFA6248D9
:109F4000444321005FF0804002F0D7FA5FF0804088
:109F500002F0BFFA10BD5D4800685D4908607047B7
:109F60005A48006870475B490A68C0B210430860ED
:109F7000704780B502F04CF90F2002F085F91620E9
:109F800002F082F9544801F001FE544801F0FEFD50
:109F9000534801F0FBFD534853490860FBE7534821
:109FA0000068704780B502F033F94FF40040504923
:109FB000086002F0B1FA4F4801F006FE012001F0FE
:109FC000FFFD4D4801F0D3FD4C4801F0D0FD4C4859
:109FD00001F0CDFD4B4801F0CAFD4B4801F0C7FD33
:109FE0004A4801F0C4FD4A4801F0C1FD02F0C4F93D
:109FF000002803D001203D49086002E000203B49D1
:10A000000860314802F09CFA02F08EFA00210F201D
:10A0100002F005F90F2002F013F902F08BFA02F0BA
:10A02000F3F85FF0704001F0A2FD5FF0804002F0B5
:10A030005DFA012803D15FF0804002F04FFA354904
:10A040005FF0804002F059FA5FF0804002F03BFA86
:10A050005FF0804002F059FA5FF0804002F032FA7F
:10A060005FF0804002F035FA01BD80B51748006806
:10A07000174908601420FFF756FF002015490860B3
:10A0800001BD80B5134800681F2802D0012000F0F0
:10A0900049F80E4801680E480068091A0B2902D3D6
:10A0A000012000F03FF8002001F07FFD000703D5FC
:10A0B0000C480D490860FBE701BD04480168491CD4
:10A0C00001607047D010002080380100201200206D
:10A0D0002412002028120020050400F0011800F0CE
:10A0E000000C00F00400FA050CED00E02C1200203A
:10A0F00008ED00E0800300C1000800F0010800F056
:10A10000020800F0030800F0040800F0050800F061
:10A11000005800F000B4C4041A490A6832EA00008A
:10A120000860704717490A6810430860704715496E
:10A1300009680840704713480178C90702D540F202
:10A1400059201EE00178890702D540F25A2018E014
:10A150000178090702D54FF4177012E0017849071A
:10A1600002D540F25B200CE00178C90602D540F22E
:10A170005D2006E00078800602D540F25E2000E017
:10A1800000207047381100209848002101600068C5
:10A19000C0439749086000209649087000209649FE
:10A1A0000870002095490870002095490870704794
:10A1B0008E4800688E490968C943884201D1012050
:10A1C00000E00020704780B5042801D0062805D1A2
:10A1D000864908602020FFF79FFF05E000208349A3
:10A1E00008602020FFF79EFF80480068C043804938
:10A1F000086001BD052800D300208249086070472F
:10A20000002103E0425C804B5A54491C1829F9D3C1
:10A2100070477849087070477749087070477749E8
:10A22000087070477649087070477048006870473A
:10A23000002103E0744A525C4254491C1829F9D3A6
:10A2400070477048006870476A48007870476A48ED
:10A25000007870476A4800787047644801680429AC
:10A2600007D164480078282801DA00200DE0012099
:10A270000BE00068062807D15E480078202801DA44
:10A28000002002E0012000E00020704757480068ED
:10A29000062801D1012000E00020704780B5534816
:10A2A0000068042806D11E2000F0BBFE072801D15B
:10A2B000012000E0002002BD80B54C480068042861
:10A2C00006D11E2000F0ADFE082801D1012000E0DB
:10A2D000002002BD80B545480068042806D11E2034
:10A2E00000F09FFE092801D1012000E0002002BDFE
:10A2F00080B53E480068042806D11E2000F091FE7B
:10A30000042801D1012000E0002002BD80B53748BB
:10A310000068042806D11E2000F083FE0A2801D11F
:10A32000012000E0002002BD80B530480168062908
:10A3300001D1002014E00068042810D11E2000F094
:10A3400070FE042809D0092807D0082805D007285E
:10A3500003D00A2801D0012002E0002000E0012003
:10A3600002BD10B50C001100042805D1274A2000B9
:10A3700002F049FA012035E0062805D1244A2000E0
:10A3800002F041FA01202DE0072805D1214A2000E2
:10A3900002F039FA012025E0092805D11E4A2000E3
:10A3A00002F031FA01201DE0082805D11B4A2000E7
:10A3B00002F029FA012015E0102806D1184B0AA254
:10A3C000200002F020FA01200CE00A2805D1154AED
:10A3D000200002F018FA012004E0134A200002F0E5
:10A3E00012FA002010BD000025730000F0110020BB
:10A3F000F41100203A1200203B1200203C120020F1
:10A400003D120020F81100208810002050FD0100AE
:10A4100058FD010060FD010068FD010070FD0100B4
:10A42000ACF4010078FD010080FD01000021010075
:10A43000C9B230390A2902D23038C0B208E001006E
:10A44000C9B24139062902D23738C0B200E0002033
:10A45000704710F00F00DFF84015085C70470028C7
:10A4600001D120207CE0C10701D5002078E08107E0
:10A4700001D5012074E0410701D5022070E00107F9
:10A4800001D503206CE0C10601D5042068E08106F7
:10A4900001D5052064E0410601D5062060E00106F3
:10A4A00001D507205CE0C10501D5082058E08105F1
:10A4B00001D5092054E0410501D50A2050E00105ED
:10A4C00001D50B204CE0C10401D50C2048E08104EB
:10A4D00001D50D2044E0410401D50E2040E00104E7
:10A4E00001D50F203CE0C10301D5102038E08103E5
:10A4F00001D5112034E0410301D5122030E00103E1
:10A5000001D513202CE0C10201D5142028E08102DE
:10A5100001D5152024E0410201D5162020E00102DA
:10A5200001D517201CE0C10101D5182018E08101D8
:10A5300001D5192014E0410101D51A2010E00101D4
:10A5400001D51B200CE0C10001D51C2008E08100D2
:10A5500001D51D2004E0400001D51E2000E01F2091
:10A560007047002903D1002801D14020BEE102003C
:10A57000D20701D50020B9E10200920701D50120E0
:10A58000B4E10200520701D50220AFE10200120738
:10A5900001D50320AAE10200D20601D50420A5E1DD
:10A5A0000200920601D50520A0E10200520601D565
:10A5B00006209BE10200120601D5072096E1C205A4
:10A5C00001D5082092E1820501D509208EE14205DE
:10A5D00001D50A208AE1020501D50B2086E1C204DB
:10A5E00001D50C2082E1820401D50D207EE14204D8
:10A5F00001D50E207AE1020401D50F2076E1C203D5
:10A6000001D5102072E1820301D511206EE14203D1
:10A6100001D512206AE1020301D5132066E1C202CE
:10A6200001D5142062E1820201D515205EE14202CB
:10A6300001D516205AE1020201D5172056E1C201C8
:10A6400001D5182052E1820101D519204EE14201C5
:10A6500001D51A204AE1020101D51B2046E1C200C2
:10A6600001D51C2042E1820001D51D203EE14200BF
:10A6700001D51E203AE1002801D51F2036E110F057
:10A68000000211F00103002B01D1002A01D020208B
:10A690002CE110F0000211F00203002B01D1002A7E
:10A6A00001D0212022E110F0000211F00403002B60
:10A6B00001D1002A01D0222018E110F0000211F08F
:10A6C0000803002B01D1002A01D023200EE110F055
:10A6D000000211F01003002B01D1002A01D0242028
:10A6E00004E110F0000211F02003002B01D1002A38
:10A6F00001D02520FAE010F0000211F04003002BF9
:10A7000001D1002A01D02620F0E010F0000211F063
:10A710008003002B01D1002A01D02720E6E010F0B1
:10A72000000211F48073002B01D1002A01D02820EF
:10A73000DCE010F0000211F40073002B01D1002ABC
:10A7400001D02920D2E010F0000211F48063002B28
:10A7500001D1002A01D02A20C8E010F0000211F433
:10A760000063002B01D1002A01D02B20BEE010F0A5
:10A77000000211F48053002B01D1002A01D02C20BB
:10A78000B4E010F0000211F40053002B01D1002AB4
:10A7900001D02D20AAE010F0000211F48043002B1C
:10A7A00001D1002A01D02E20A0E010F0000211F407
:10A7B0000043002B01D1002A01D02F2096E010F099
:10A7C000000211F48033002B01D1002A01D0302087
:10A7D0008CE010F0000211F40033002B01D1002AAC
:10A7E00001D0312082E010F0000211F48023002B10
:10A7F00001D1002A01D0322078E010F0000211F4DB
:10A800000023002B01D1002A01D033206EE010F08C
:10A81000000211F48013002B01D1002A01D0342052
:10A8200064E010F0000211F40013002B01D1002AA3
:10A8300001D035205AE010F0000211F48003002B03
:10A8400001D1002A01D0362050E010F0000211F4AE
:10A850000003002B01D1002A01D0372046E010F080
:10A86000000211F08073002B01D1002A01D03820A2
:10A870003CE010F0000211F00073002B01D1002A1F
:10A8800001D0392032E010F0000211F08063002B7B
:10A8900001D1002A01D03A2028E010F0000211F086
:10A8A0000063002B01D1002A01D03B201EE010F0F4
:10A8B000000211F08053002B01D1002A01D03C206E
:10A8C00014E010F0000211F00053002B01D1002A17
:10A8D00001D03D200AE010F0000011F08041002975
:10A8E00001D1002801D03E2000E03F207047012127
:10A8F00011FA00F0704730B43C22B0FBF2F23C2475
:10A9000004FB120008603C20B2FBF0F304FB1322AE
:10A910004A601820B3FBF0F2182000FB12338B6062
:10A92000101D0723B0FBF3F403FB1400886102F24F
:10A93000DB2240F2B550B2FBF0F340F2B55000FB21
:10A9400013203C2802D35B1C0C2400E00224D01A04
:10A9500040F26D15B0FBF5F0443048614D69443D5F
:10A9600040F26D1000FB1522D21A002000E0401CBE
:10A97000A04204D2094B53F820309A42F7D2431E2A
:10A980000B61064B03EB800050F8040C121A521CAA
:10A99000CA6030BC704700009CF4010040F0010028
:10A9A00078B58BB005005FF000465FF080446946E3
:10A9B0003000FFF7A0FF6946280000F01BF80DE00B
:10A9C000361B02E00128FBDBA6196408694630004B
:10A9D000FFF791FF6946280000F00CF8002801D02D
:10A9E000002CEFD1002801D1300001E05FF0FF30F2
:10A9F0000CB070BD4A6943699A4201DA012048E00F
:10AA000042694B699A4202DA5FF0FF3041E00A691D
:10AA100003699A4201DA01203BE002690B699A421C
:10AA200002DA5FF0FF3034E0CA68C3689A4201DAA4
:10AA300001202EE0C268CB689A4202DA5FF0FF3054
:10AA400027E08A6883689A4201DA012021E082685F
:10AA50008B689A4202DA5FF0FF301AE04A68436876
:10AA60009A4201DA012014E042684B689A4202DA05
:10AA70005FF0FF300DE00A6803689A4201DA0120B6
:10AA800007E000680968884202DA5FF0FF3000E002
:10AA90000020704780B5624830210170302141703C
:10AAA000302181703021C1705E4830210170302129
:10AAB0004170302181703021C17000F06FF800F0DA
:10AAC00088F801BDF0B40400049D0120E4B2002C1C
:10AAD00029D1554C0E002778F6B2BE4201D0002095
:10AAE00013E016006778F6B2BE4201D000200CE0F9
:10AAF0001E00A778F6B2BE4201D0002005E02E006D
:10AB0000E478F6B2A64200D00020C9B2332933D18E
:10AB1000D2B2312A30D1DBB2302B2DD1EDB2312D72
:10AB20002AD1012028E0414C0E002778F6B2BE421F
:10AB300001D0002013E016006778F6B2BE4201D0C3
:10AB400000200CE01E00A778F6B2BE4201D0002023
:10AB500005E02E00E478F6B2A64200D00020C9B28B
:10AB6000332909D1D2B2312A06D1DBB2302B03D13D
:10AB7000EDB2312D00D10120F0BC704710B4294C4A
:10AB800020706170A270E37010BC704710B4264C46
:10AB900020706170A270E37010BC70472248214998
:10ABA0000A7802704A7842708A788270C978C170D7
:10ABB000704710B41D4C20706170A270E37010BC1F
:10ABC000704710B4164C20706170A270E37010BC16
:10ABD0007047164812490A7802704A7842708A789B
:10ABE0008270C978C1707047042801D3302001E019
:10ABF0000D49085C7047042801D3302001E0094961
:10AC0000085C7047042801D3302001E00749085C44
:10AC10007047042801D3302001E00149085C7047E7
:10AC20001412002018120020101200200C12002014
:10AC30005948002101600068C043584908607047C6
:10AC40005548006855490968C943884201D1012027
:10AC500000E0002070470200C943D2B2C9B28A4264
:10AC600006D14D49C0B208600868C0434B4908602E
:10AC7000704749490A68C0B2104308600868C04379
:10AC800046490860704744490A68C0B232EA000089
:10AC900008600868C0434149086070473E49096838
:10ACA000C0B2084070473C480178890701D50A20A6
:10ACB0004EE00178C90706D50078400701D5092084
:10ACC00046E0082044E00178890606D50078400770
:10ACD00001D507203CE006203AE0017849060BD573
:10ACE0000178090701D50C2032E00078C00601D5B3
:10ACF0000D202DE00B202BE0017811F0180F06D16C
:10AD00000078400701D5032022E0002020E00178F0
:10AD100011F01801182906D10078400701D50F203D
:10AD200016E00E2014E00178090706D500784007E8
:10AD300001D504200CE001200AE00178C90606D5FF
:10AD40000078400701D5052002E0022000E0002045
:10AD5000704738B504000D00FFF7A5FF0C2806D199
:10AD60000F4B104A2900200001F04DFD10E00D2886
:10AD700006D10B4B0C4A2900200001F044FD07E0EE
:10AD80000A4951F8203003A22900200001F03BFDC0
:10AD900031BD00002573200004120020081200209D
:10ADA00080F40300A8FD0100B0FD0100480200206E
:10ADB00080B5FFF73DFFFFF7E7F900F08BF9FFF7EC
:10ADC00069FE00F01BF94FF6FF7000F0D0F801BDEE
:10ADD00080B5FFF7EDF9002803D0FFF731FF002819
:10ADE00003D10220FFF79EF902E00220FFF794F959
:10ADF0001020FFF7B8F801BD5F49087070475E4842
:10AE0000007870475D49086070475D48006870478A
:10AE10005B49086070475B490860704759480068A3
:10AE2000704759490860704757480068704757494C
:10AE3000086070475548006870475549086070477A
:10AE4000534800687047010402D45249086005E085
:10AE500040F07F4050F47F004E49086070474D48F5
:10AE6000006870474C490A681043086070474A48B8
:10AE700000687047002048490860704780B50A00A4
:10AE80003D4B1978002903D1444901F061FB64E08E
:10AE90001978012903D1424901F05AFB5DE0197884
:10AEA000022903D13F4901F053FB56E019780329E9
:10AEB00003D13D4901F04CFB4FE01978042903D13F
:10AEC0003A4901F045FB48E01978052903D1384992
:10AED00001F03EFB41E01978062903D1354901F024
:10AEE00037FB3AE01978072903D1334901F030FBE9
:10AEF00033E01978082903D1304901F029FB2CE00F
:10AF00001978092903D12E4901F022FB25E019788F
:10AF10000A2903D12B4901F01BFB1EE019780B29EC
:10AF200003D1294901F014FB17E019780C2903D14A
:10AF3000264901F00DFB10E019780D2903D12449B1
:10AF400001F006FB09E01978802903DB214901F0B3
:10AF5000FFFA02E01E4901F0FBFA01BD1E49086834
:10AF60004FF6FF720B68934200D00A6070471A498F
:10AF7000086070470000000039120020981100207E
:10AF8000AC1100209C110020A0110020A411002071
:10AF9000A8110020B4110020B8110020A0E3030084
:10AFA000C0E3030080DD0300E0E3030000E40300EE
:10AFB00020E4030040E4030060E4030080E40300B5
:10AFC000A0E40300C0E40300E0E4030020DF03008A
:10AFD00020E5030040E50300B011002005490860AA
:10AFE000704705490860704702480068704702488A
:10AFF00000687047DC110020E01100200020334978
:10B00000086070473249496C0840704730494A6CC3
:10B010001043486470472E494A6C32EA0000486485
:10B0200070470100C9B2442902D12948406C10E0A0
:10B030000100C9B2402902D12548006C09E0010095
:10B04000C9B2602902D12248006E02E02049C0B294
:10B05000085C70471E49085C7047802801D21C4A72
:10B060001154402802D3012018490860704702009B
:10B07000D2B20300DBB2802B23DA0300DBB2402B19
:10B0800002D1134801641CE00300DBB2602B02D143
:10B090000F48016615E00300DBB2442B02D10C48D7
:10B0A00041640EE00300DBB2382B02DBC0B254284F
:10B0B00005D107488154521CC943815401E004481A
:10B0C000815470470148006870470000D811002083
:10B0D000900E0020002006E0FF216B4A1154002151
:10B0E0006A4A1154401C0E28F6D37047684908601C
:10B0F000704768490860704767490860704780B5C5
:10B100005720FFF78EFF012802D16148006800E058
:10B11000002002BD80B55720FFF783FF012802D130
:10B120005D48006800E0002002BD80B55720FFF7B1
:10B1300078FF012802D15748006800E0002002BDD6
:10B1400056490968884202D15548006800E000204D
:10B150007047524A106052480160704780B501281C
:10B1600005D15FF0FF304F4900F03CFA09E04B4950
:10B170000968884203D14C48D0E9000101E0002071
:10B18000002104BD454908604748C0E900237047D5
:10B1900080B5012802D1FFF727FF07E03F49096882
:10B1A000884202D14148006800E0002002BD3B4ACD
:10B1B00010603E480160704738490968884202D1F2
:10B1C0003B48006800E000207047344A106038486F
:10B1D0000160704710B50C0001280FD1FFF734F85B
:10B1E000002C03D10A21B0FBF1F004E00A21B0FBEE
:10B1F000F1F201FB1200FFF72CF907E0274909687B
:10B20000884202D12B48005D00E0002010BD234B96
:10B21000186028484254704780B5811E0E2904D218
:10B220001A49084410F8020C06E0012803D11E2038
:10B23000FFF7F7FE00E0002002BD821E0E2A03D2B7
:10B24000124A104400F8021C704780B5811E0E2976
:10B2500004D20D49084410F8020C0BE0012808D173
:10B260005920FFF7DEFE002801D0012002E0002077
:10B2700000E0002002BD821E0E2A03D2024A1044C2
:10B2800000F8021C70470000C0100020B010002021
:10B29000BC110020C4110020C0110020C8110020E2
:10B2A000CC110020FFFF0F00F8100020D01100206B
:10B2B000D4110020361200202C4AC0B2115470471D
:10B2C0002A49C0B2085C7047F8B584B004000D008C
:10B2D0000320FFF7F5FF012805D10422244903A824
:10B2E00001F036F92CE0022805D10422214903A8F7
:10B2F00001F02EF924E0032805D104221E4903A8F9
:10B3000001F026F91CE0042805D104221B4903A8FA
:10B3100001F01EF914E0052805D10422184903A8FC
:10B3200001F016F90CE0062805D10422154903A8FE
:10B3300001F00EF904E00422134903A801F008F912
:10B340000520FFF7BDFF06000420FFF7B9FF070047
:10B350000220FFF7B5FF02960197009003AB0B4A5E
:10B360002900200001F04FFA05B0F0BD08110020BF
:10B3700000EB030020EB030040EB030060EB030055
:10B3800080EB0300A0EB0300C0EB030054F30100CB
:10B3900073490860704772480068704710B50C0028
:10B3A0000F281CD20C2807D16E48036B6E4A162159
:10B3B000200001F028FA19E00D2807D16948436BF5
:10B3C0006A4A1621200001F01EFA0FE0654951F883
:10B3D000203062A21621200001F015FA06E0614833
:10B3E00003685EA21621200001F00DFA10BD10B412
:10B3F0000C281CD25E4A0B78052404FB00F413557C
:10B400004B78052404FB00F4144463708B78052406
:10B4100004FB00F41444A370CB78052404FB00F46F
:10B420001444E3700B79052148431044037110BCA8
:10B4300070470C281DD24E4B052202FB00F29A5C8D
:10B440000A70052202FB00F21A4452784A70052263
:10B4500002FB00F21A4492788A70052202FB00F285
:10B460001A44D278CA7005225043184400790871F2
:10B4700009E000200870002048700020887000203B
:10B48000C870002008717047F0B406292FD2082830
:10B490002DD21E23374C03FB00F52544052606FB61
:10B4A00001F61778AF5503FB00F52544052606FB8A
:10B4B00001F6354456786E7003FB00F525440526E9
:10B4C00006FB01F635449678AE7003FB00F5254483
:10B4D000052606FB01F63544D678EE70584304EB9A
:10B4E00000030520414303EB010011790171F0BC19
:10B4F000704770B406292FD208282DD21E231D4C68
:10B5000003FB00F52544052606FB01F6AD5D15702D
:10B5100003FB00F52544052606FB01F635446D784E
:10B52000557003FB00F52544052606FB01F635445E
:10B53000AD78957003FB00F52544052606FB01F662
:10B540003544ED78D570584304EB000305204143A2
:10B5500003EB01000079107170BC70472573200067
:10B560001C12002088020020B8FD0100C0FD01006F
:10B57000780F0020A00C0020D2B2203A22BF00FA9F
:10B5800002F1002070475242D041D2F12002914096
:10B590004140D04090404140704700003E49086023
:10B5A00070473E49086070473B490968084070474A
:10B5B0003A4909680840704780B53749086800284B
:10B5C0000AD00868FEF74BFF202803D2344951F80F
:10B5D000200002E0002000E0002002BD314AC2E964
:10B5E000000170472F4AD2E90023104019407047EC
:10B5F0002D49086070472C48006870471CB504004E
:10B600000800FEF72CFF0A2808D1284800900B23D9
:10B61000274A1621200001F0F6F816E00B2808D181
:10B62000244800900C23224A1621200001F0EBF858
:10B630000BE0214951F820100091194951F82030B0
:10B640001E4A1621200001F0DEF813BD1CB50400CF
:10B650000800FEF704FF1A4951F82010009119491B
:10B6600051F82030154A1621200001F0CCF813BD06
:10B670001CB5040010001900FEF773FF124951F8C1
:10B6800020100091114951F820300C4A1621200059
:10B6900001F0B9F813BD0000E4110020E81100200A
:10B6A000F0E9010000110020EC110020A0D50300FA
:10B6B00040F3010080D503000000002048FD010098
:10B6C0004001002070EA0100800000207CE70100BA
:10B6D000DFF8E81308607047DFF8E413086070478C
:10B6E000DFF8D80300687047DFF8D40300687047BC
:10B6F00080B51300B3F11802082A07D30A00DFF857
:10B70000C41351F8231000F023FF07E0DFF8B4233F
:10B7100052F82330DFF8B02301F075F801BD22287C
:10B7200001D3002003E0DFF8A41351F82000704794
:10B73000012801D1022080E0022801D11E207CE0F6
:10B74000032801D1212078E0042801D1092074E0E8
:10B75000052801D11E2070E0062801D11F206CE0D1
:10B76000072801D1042068E0082801D1052064E001
:10B77000092801D1062060E00A2801D107205CE0F9
:10B780000B2801D1182058E00C2801D1082054E0E2
:10B79000102801D11D2050E00F2801D11C204CE0C1
:10B7A0000D2801D10E2048E00E2801D11A2044E0D6
:10B7B000112801D10B2040E0122801D10A203CE0E1
:10B7C000132801D1152038E0142801D1142034E0C9
:10B7D000152801D1132030E0162801D112202CE0C9
:10B7E000172801D1192028E0182801D1012024E0D0
:10B7F000192801D1032020E01A2801D10F201CE0D4
:10B800001B2801D1102018E01C2801D1112014E0C0
:10B810001D2801D10D2010E01E2801D116200CE0BA
:10B820001F2801D11B2008E0202801D10C2004E0B2
:10B83000212801D1172000E000207047022801D103
:10B84000012080E0202801D102207CE0212801D1C4
:10B85000032078E0092801D1042074E01E2801D1DA
:10B86000052070E01F2801D106206CE0042801D1DA
:10B87000072068E0052801D1082064E0062801D1EE
:10B88000092060E0072801D10A205CE0182801D1D6
:10B890000B2058E0082801D10C2054E01D2801D1CC
:10B8A000102050E01C2801D10F204CE00E2801D1BF
:10B8B0000D2048E01A2801D10E2044E00B2801D1C8
:10B8C000112040E00A2801D112203CE0152801D1C6
:10B8D000132038E0142801D1142034E0132801D1BA
:10B8E000152030E0122801D116202CE0192801D1B2
:10B8F000172028E0012801D1182024E0032801D1D5
:10B90000192020E00F2801D11A201CE0102801D1B5
:10B910001B2018E0112801D11C2014E00D2801D1B2
:10B920001D2010E0162801D11E200CE01B2801D19B
:10B930001F2008E00C2801D1202004E0172801D1A5
:10B94000212000E00020C0B2704780B51300DBB2B8
:10B95000012B04D10A005E4900F0FAFDADE01300AE
:10B96000DBB2022B04D10A005A4900F0F1FDA4E039
:10B970001300DBB2032B04D10A00574900F0E8FDA5
:10B980009BE01300DBB2042B04D10A00534900F002
:10B99000DFFD92E01300DBB2052B04D10A00504911
:10B9A00000F0D6FD89E01300DBB2062B04D10A00BB
:10B9B0004C4900F0CDFD80E01300DBB2072B04D131
:10B9C0000A00494900F0C4FD77E01300DBB2082B00
:10B9D00004D10A00454900F0BBFD6EE01300DBB264
:10B9E000092B04D10A00424900F0B2FD65E01300C2
:10B9F000DBB20A2B04D10A003E4900F0A9FD5CE04D
:10BA00001300DBB20B2B04D10A003B4900F0A0FD70
:10BA100053E01300DBB20C2B04D10A00374900F0CD
:10BA200097FD4AE01300DBB20D2B04D1344B354AAD
:10BA300000F0E9FE41E01300DBB20E2B04D1304BE5
:10BA4000314A00F0E0FE38E01300DBB20F2B04D1E6
:10BA50000A002E4900F07CFD2FE01300DBB2102B12
:10BA600004D10A002A4900F073FD26E01300DBB27E
:10BA7000112B04D10A00274900F06AFD1DE01300D4
:10BA8000DBB2122B04D10A00234900F061FD14E05F
:10BA90001300DBB2132B04D1204B214A00F0B3FE7C
:10BAA0000BE0D2B2142A04D11C4B1E4A00F0ABFEAC
:10BAB00003E00A001C4900F04BFD01BDFC11002011
:10BAC00000120020C00100200CF8010068E901000C
:10BAD000A0E8030020E50300C0E80300E0E803005D
:10BAE00020DF030020E9030040E9030060E90300D0
:10BAF00080E90300A0E9030040E70300C0D403008D
:10BB0000ACF4010088FD010090FD010038F801004F
:10BB1000ACF30100E0D2030060F7030080F70300FC
:10BB200098FD0100A0FD010080E6030038B581000A
:10BB3000DFF87C22C0F3072301F47F71D31841EAB8
:10BB4000431343F0844301241C600025009502E068
:10BB5000009B5B1C0093009B102BF9D3C0F30720C4
:10BB6000121841EA421141F084410D6031BDC0F329
:10BB70000722DFF8401280008A1800F47F7040EA44
:10BB8000421040F08440012101607047C0F3072259
:10BB9000DFF8201280008A1800F47F7040EA42101B
:10BBA00040F08440002101607047DFF80C1208B1BA
:10BBB00088687047086870470138FDD17047704742
:10BBC000DFF8F8110860704770B5DFF8EC211469F0
:10BBD000136A014624F4800401F0010544F4006472
:10BBE00004F0010085F0010543F40063146128426C
:10BBF000136210D061F001004FF48075044095602D
:10BC000014614FF400201568EE0502D4401EFAD1ED
:10BC100070BD002848D00D0965F30A14DFF8B001A3
:10BC2000DFF8B06103400E40CD00334305F040051E
:10BC30002B4314611362480B60F34D3460F34D33B2
:10BC400040209060002B47BF13621461146113629F
:10BC5000DFF88401DFF8845104400D402C43C80D07
:10BC60004D0060F3DC5308D5DFF8740123F4800342
:10BC7000084044F48004034301E023F080430805B6
:10BC80000CD44FF40040DFF85C110D68EE0701D4CE
:10BC9000401EFAD124F4006423F40063146113629B
:10BCA0001020BDE8704087E770BDF0B54E490A6DC1
:10BCB0000B6E002B4CBF03F0700002F0300040B15F
:10BCC000102846D0202846D0302846D0702847D0AB
:10BCD00049E03C48C2F3841450F82450434C04EA31
:10BCE0000306B6F1004F4FF0FF3003D0002B41D4D4
:10BCF00017053FD4344E376876680968C6F3042CBC
:10BD000006F01F060CF1010C761C16FB0CF67600F3
:10BD1000B5FBF6F5C7F30906C7F389276F4301F4AE
:10BD20007041BF0AB1F5005F06FB057542F4800261
:10BD30000DD0B1F5405F18D0B1F5804F17D0B1F5F7
:10BD4000E04F16D0B1F5104F08BF294812E029483E
:10BD500010E01B4DC2E7284DC0E747F23055BDE764
:10BD60004FF40045BAE70020F0BD244802E0244823
:10BD700000E01648510217D5002B10D559000BD5FD
:10BD80001C40B4F1004F03D0002B05D4120503D49E
:10BD90006D00C3F3865104E0C3F3C55101E0C2F363
:10BDA000C351491CB5FBF1F5A84288BF2846F0BD38
:10BDB00000E50F4000E60F4050E00F407CE00F40F0
:10BDC0000024F40068EB010060E10F4040787D0141
:10BDD0008FFFFF7F30000080FEFF3FF80100C007AB
:10BDE0000000404068E10F4010E00F400008008074
:10BDF000002D310100B4C40400093D0080F0FA02B6
:10BE0000005A62024C49FFE7012008607047012197
:10BE100000F01F00494A03E0012100F01F00484ADA
:10BE200001FA00F01060704746490860704710B58D
:10BE300000F00EF8444ACB0748BF10608C0748BF9B
:10BE400090614B0748BF1062090748BF906010BD62
:10BE500000F01F00012202FA00F07047394A126810
:10BE600000F03F0002EB001238489368034019438A
:10BE700091607047F0B5334C2568354C00F03F00B9
:10BE800005EB0016B7682740840604D5042914BFC3
:10BE9000062941F00101DDF814C0ACF1010E41EAC0
:10BEA0000E14274307F04064B4F1406F04D0A40E91
:10BEB0000CFA04F4A218521E326007F04042B2F1AC
:10BEC000404F0FD0042918BF062906D140F02000AA
:10BED00005EB001000F10C0304E0920F0CFA02F0E5
:10BEE00003445B1E7360B760F0BD1649096800F03B
:10BEF0003F0001EB0010806800F007004108490096
:10BF000004291EBF42085200062A04BF4008400010
:10BF1000704700F0FF0110B5CB080E4A02EB830218
:10BF2000890001F01C0113680F248C40000CA3430E
:10BF300088401843106010BD04F00F4028F00F40F7
:10BF40002CF00F4008F00F401CF00F40F73FFC00B2
:10BF500008C0FFFF10F50F4030B5CB4300F58064FB
:10BF6000D50725684CBF0D431D40256000F5846052
:10BF7000920747BF0368194301681940016030BD4B
:10BF8000F0B5002400F6C4750126A640314210D059
:10BF90006600D5F800C00327B7402CEA07072F60DA
:10BFA000C2F34117D5F800E007FA06F646EA0E0696
:10BFB0002E60641C082CE7DBCC4300F5A065D60797
:10BFC0002E684CBF0E4326402E6000F204559607A3
:10BFD0002E684CBF0E4326402E6000F5A165560723
:10BFE0002E684CBF0E4326402E6000F5A365160751
:10BFF0002E684CBF0E4326402E6000F23C55D20600
:10C000002A684CBF0A4322402A60DD0700F20C5226
:10C0100015684CBF0D432540156000F5A2629D07D1
:10C0200015684CBF0D432540156000F214525D07A2
:10C0300015684CBF0D432540156000F21C521D07CA
:10C0400015684CBF0D432540156000F244529D0514
:10C0500015684CBF0D432540156000F5A86213F428
:10C06000407F156814BF0D432540156000F5A5609D
:10C07000002B07BF026841EA020401680C4004601B
:10C08000F0BD00EB810002607047012278E738B50F
:10C0900000F02DF82946204601B0BDE830400823C5
:10C0A000F3E738B504460D460823FFE70122FFF702
:10C0B00067FF29462046BDE8384001224CE7044688
:10C0C0000D46022248E738B5FFF7F9FF294620461A
:10C0D00001B0BDE830400823D7E738B5FFF7EFFFE0
:10C0E0002946204601B0BDE830400823CDE704468C
:10C0F0000D46002230E730B50D4B0E4A1C68C0F3E8
:10C100000741CC40E50746BF02EBC101496852F840
:10C11000311001F22C51020A0B680F24944000F0F8
:10C120000F00A34390401843086030BD000000009A
:10C130006CE00F40D8E80100114340F8341F70470D
:10C14000F8B504460E4617461D4600F034F804F1D3
:10C150003000B6EB071F016804D241F020010160F6
:10C160007F0802E021F020010160F600B6FBF7F045
:10C17000401C400804F12402810904F128031160E5
:10C1800000F03F00186004F1180204F12C000021B7
:10C19000056011602046BDE8F240FFE700F12C0188
:10C1A0000A6842F010020A6040F2013150F8303F54
:10C1B0000B430360704700F118010A681307FCD4B1
:10C1C00000F12C010A6822F010020A6050F8303F9A
:10C1D00002490B400360704700000000FEFCFFFFB7
:10C1E00011430160704750F8302F22F01002F7E73A
:10C1F000002914BF40303C300068704740F8441FAD
:10C20000704750F8482FEBE780B500F03DFB02E0A7
:10C2100080B500F035FB00B10120C0B202BD10B501
:10C22000304A830852F823201368C00000F0180039
:10C23000FF248440A34381401943116010BD0000D6
:10C2400010B50428284903D1086840F480300AE07A
:10C25000052803D1086840F4003004E0062804D122
:10C26000086840F48020086010BD0F2804D11F48E2
:10C27000016841F0020104E004D900BF1CA400F0F1
:10C2800026F8016010BD000010B50428164903D13E
:10C29000086820F480300AE0052803D1086820F4FB
:10C2A000003004E0062804D1086820F480200860EB
:10C2B00010BD0F2804D10D48016821F0020104E0EF
:10C2C00004D900BF0FA400F002F8016010BDA0F176
:10C2D000100310384009012103F01F0354F8200017
:10C2E000994070473CE8010024ED00E010E000E0D8
:10C2F00000E100E004E100E008E100E00CE100E022
:10C3000010E100E080E100E084E100E088E100E08D
:10C310008CE100E090E100E038B5044600F029F837
:10C32000604D03202860E40900F023F8012000FAA2
:10C3300004F45D49E4430C6000F01BF80020286021
:10C340000A20BDE83240FFF737BC10B500F011F805
:10C35000544C0320206000F00CF853490020086082
:10C3600000F007F8002020600A20BDE81040FFF729
:10C3700023BC0A20FFF720BC10B50220FFF71CFCED
:10C380004A4C00F00EF808D14948FFF7CFFB0220D5
:10C39000FFF712FC00F005F801D0022010BD0020CC
:10C3A00010BD2068C107FCD4606810F00C0F704706
:10C3B00010B5404B8C091C60C1F383019208596091
:10C3C0000AD004E0596811B91C68641C1C60521E34
:10C3D000196940F8041BF5D110BD2DE9F84F8146CD
:10C3E0008A46344D6869C007FCD4DFF8CC80334FEF
:10C3F000334E89092960CAF383009408686005D127
:10C400002AE0686810B92968491C296030683840FA
:10C41000404505D13168080404BF5046FFF77CFF52
:10C42000D9F800002861FFF7A4FFD5F814B05FEA3F
:10C43000CB70FAD45FEACB610AD530680740474534
:10C4400004D13168080408BFFFF77FFF58460DE0AC
:10C45000641E09F10409D4D130680740474504D16E
:10C460003168080408BFFFF770FF6869BDE8F28F04
:10C4700038B50D461249104B0A6804460F48024071
:10C480009A4205D10968080404BF2846FFF744FF13
:10C490000848A9090160C5F383014160046140694E
:10C4A00032BD0000FCD00F40C0E20A4018F00A4044
:10C4B000005800F004F00A40000005100000FF7072
:10C4C00000E00F401BE050F8081F41F0020101603E
:10C4D000704700F5406001210160704700F5406041
:10C4E000014901607047000051E5CC1A00F5406039
:10C4F0000068012818BF002070470160704750F89D
:10C50000081F41F001010160704700F58360016878
:10C5100041F48071016070470248016841F0404178
:10C520000160704734EF00E00748016841F0050101
:10C53000016070470448016841F0020101607047E2
:10C540000249401E0860704710E000E014E000E07F
:10C5500010B4002403E00B5D0355641C521E002A36
:10C5600002D00B5D002BF6D1002A04D0002101552A
:10C57000641C521EF8E710BC70472DE9F0470C0010
:10C580000021002C00D0641E5FF0000980461600D8
:10C590001F000AE038683F1D002C04D088F8000016
:10C5A00018F10108641E19F101093078002800F023
:10C5B0001981002500E06D1C705D252802D0705D9A
:10C5C0000028F8D1AC4207D2220031004046FFF7E4
:10C5D000BFFFA044002406E02A0031004046FFF7D8
:10C5E000B7FFA844641B15EB09092E4430782528B1
:10C5F000DBD1761C002520220CE016F8010C302837
:10C6000002D1002D00D130220A20454316F8010C3A
:10C61000303845193000461C0078253800F0BF80BE
:10C620000B380928E9D9283856D00B38B2D0401E2B
:10C630000AD0401F08D0C01F4ED0C01E0FD0801E91
:10C6400044D0C01E48D0B6E03B683F1D002B02D549
:10C650005B42012000E000205FF00A0C41E03968F5
:10C660003F1D5FF0000A01E01AF1010A11F80A000B
:10C670000028F9D1AA4503D215EB0909B9EB0A093B
:10C68000544506D222004046FFF762FFA044002432
:10C6900018E052464046FFF75BFFD044B4EB0A0473
:10C6A000AA450FD2B5EB0A05AC4200D225006C4278
:10C6B00004E0202088F8000018F101082800451E39
:10C6C0000028F6D11AEB090AD1466EE73B683F1DF8
:10C6D0005FF00A0C002004E03B683F1D5FF0100C87
:10C6E0000020012102E00CFB01F16D1E0CFB01FE9C
:10C6F000734505D30CFB01FEBEFBFCFE8E45F2D05C
:10C70000002800D06D1E002810D0002C0ED09646B8
:10C710005FFA8EFEBEF1300F08D12D2088F80000A0
:10C7200018F10108641E19F101090020B5F1020E8B
:10C730004FF6FE7AD6450DD26D1E09E0002C04D0CE
:10C7400088F8002018F10108641E19F101096D1E16
:10C75000002DF3D100281FD0002C1DD02D2088F8EB
:10C76000000018F10108641E19F1010914E0002C01
:10C770000ED0B3FBF1F0B0FBFCF20CFB1200DFF8C3
:10C78000F8201268105C88F8000018F10108641E97
:10C7900019F10109B1FBFCF10029E8D105E7002CF2
:10C7A00006D016F8010C88F8000018F10108641E84
:10C7B00019F10109F9E6052C09D30522DFF8BC10AF
:10C7C0004046FFF7C5FE18F10508641F07E0220088
:10C7D000DFF8A8104046FFF7BBFEA044002419F183
:10C7E0000509E2E6002088F800004846BDE8F08729
:10C7F0000CB480B50A0002AB4FF6FF71FFF7BDFE27
:10C8000002BC5DF80CFB08B400B501ABFFF7B5FE48
:10C810005DF808FB70B406E0DBB2E4B2A34224D3B7
:10C82000401C491C521E002A22D00378002B02D142
:10C830000B78002B0CD00378413B1A2B0AD20378DB
:10C8400020330C78413C1A2C06D20C78203404E0BA
:10C8500000200EE00378F4E70C7825001E00EDB20E
:10C86000F6B2B542D8D2012003E05FF0FF3000E01D
:10C87000002070BC70470000DCFD0100C8FD010015
:10C88000EFF3108072B67047EFF3108062B6704716
:10C89000F0B5C3B0050070200021FBF701FF1622A0
:10C8A000DFF8A41A3DA8FFF753FE3DA9002001F0D0
:10C8B000E5FB032001F0ADFB042001F002FCFDF7D5
:10C8C000EDFC012803D0FDF721FD012856D1DFF84A
:10C8D000EC3BDFF8EC2B16216846FFF794FFDFF8FE
:10C8E000E43BDFF8E42B16210DF11600FFF78BFF78
:10C8F000DFF8D83BDFF8D82B16210BA8FFF783FF12
:10C90000DFF8D03BDFF8D02B16210DF14200FFF706
:10C910007AFFDFF8C83BDFF8C82B162116A8FFF70F
:10C9200072FFDFF8C03BDFF8C02B16210DF16E005F
:10C93000FFF769FFDFF8B43BDFF8B42B162121A81D
:10C94000FFF761FFDFF8AC3BDFF8AC2B16210DF1F0
:10C950009A00FFF758FF45A4220016212CA8FFF7E4
:10C9600052FF220016210DF1C600FFF74CFF2200F6
:10C97000162137A8FFF747FF08248BE0DFF83C3B80
:10C98000DFF83C2B16216846FFF73DFFDFF86C3BD4
:10C99000DFF8342B16210DF11600FFF734FFDFF816
:10C9A000243BDFF82C2B16210BA8FFF72CFFDFF818
:10C9B0001C3BDFF8242B16210DF14200FFF723FF6B
:10C9C000DFF8103BDFF8182B162116A8FFF71BFF26
:10C9D000DFF8143CDFF8102B16210DF16E00FFF785
:10C9E00012FFDFF8F83ADFF8082B162121A8FFF72D
:10C9F0000AFFDFF8F03ADFF8002B16210DF19A005C
:10CA0000FFF701FFDFF8E43ADFF8E02B16212CA84E
:10CA1000FFF7F9FEFDF73AFC012812D1DFF8D03B11
:10CA2000DFF8D02B16210DF1C600FFF7ECFEDFF882
:10CA3000C43ADFF89C2C162137A8FFF7E4FE0B243C
:10CA400028E0FDF739FC012812D1DFF8A83ADFF819
:10CA5000A42B16210DF1C600FFF7D5FE03A2162167
:10CA600037A8FFF7D0FE0A2414E000BF0000000042
:10CA7000DFF8803ADFF87C2B16210DF1C600FFF7B6
:10CA8000C2FEDFF8503CDFF8482C162137A8FFF72C
:10CA9000BAFE0B24200002F0DFF9002002F00BFAAE
:10CAA000401C01F0BAFA022002F005FA060016272F
:10CAB000684607FB06F10144012001F0DFFA6846F1
:10CAC00007FB06F1084410F11601022001F0D6FA26
:10CAD000684607FB06F1084410F12C01032001F021
:10CAE000CDFA68467E43304410F14201042001F043
:10CAF000C5FA082002F001FC002800F05E81012048
:10CB000002F0D9F90400FDF7C9FB012804D0FDF7B4
:10CB1000FDFB012840F08380002C04D101216F200F
:10CB200002F003FA78E0012C0ED10121722002F00C
:10CB3000FCF94020FEF766FA002802D100202863A5
:10CB40006AE00120286367E0022C0FD101217320E5
:10CB500002F0EBF94FF48060FEF754FA002802D19E
:10CB60000020286358E00120286355E0032C1CD1E5
:10CB70000121742002F0D9F94FF48070FEF742FAD7
:10CB8000002807D15D20FEF74CFA002802D10020D2
:10CB9000286341E05D20FEF744FA002802D001201E
:10CBA000286339E00220286336E0042C07D10121F4
:10CBB000762002F0BAF903F0BAF828632CE0052CCD
:10CBC0000AD10121772002F0B0F94F20FEF729FAAF
:10CBD00010F00F0028631FE0062C0ED101217920F0
:10CBE00002F0A3F98020FEF70DFA002802D0012000
:10CBF000286311E0002028630EE0072C0CD10121EE
:10CC00007D2002F092F901F0EAF9002802D100201B
:10CC1000286301E001202863286BE863CAE0002C48
:10CC200004D101216F2002F080F9C3E0012C08D16A
:10CC30000121702002F079F91420FEF7F2F928633F
:10CC4000B8E0022C0ED10121722002F06EF94020D2
:10CC5000FEF7D8F9002802D100202863AAE00120BD
:10CC60002863A7E0032C0FD10121732002F05DF9A6
:10CC70004FF48060FEF7C6F9002802D10020286337
:10CC800098E00120286395E0042C1CD10121742038
:10CC900002F04BF94FF48070FEF7B4F9002807D189
:10CCA0005D20FEF7BEF9002802D10020286381E054
:10CCB0005D20FEF7B6F9002802D00120286379E054
:10CCC0000220286376E0052C08D10121752002F0AE
:10CCD0002CF93D20FEF7A5F928636BE0062C07D15F
:10CCE0000121762002F021F903F021F8286361E0A8
:10CCF000072C0AD10121772002F017F94F20FEF707
:10CD000090F910F00F00286354E0082C0ED1012197
:10CD1000792002F00AF98020FEF774F9002802D089
:10CD20000120286346E00020286343E0092C0CD151
:10CD3000FDF7ACFA012808D10121712002F0F5F8C5
:10CD40003C20FEF76EF9286334E0092C0DD1012157
:10CD50007D2002F0EAF801F042F9002802D100201B
:10CD6000286327E00120286324E00A2C11D1FDF775
:10CD70008DFA01280DD101217D2002F0D6F801F0B5
:10CD80002EF9002802D10020286313E00120286337
:10CD900010E00A2C0ED101217B2002F0C6F84FF4DE
:10CDA0008050FEF72FF9002802D00120286301E00F
:10CDB00000202863286BE8630AE0012002F09DFA56
:10CDC000002802D002F009F902E0200002F01FF969
:10CDD00043B0F0BD10B586B070200021FBF760FCB9
:10CDE0001E20FEF71EF916226946FDF7BAFA6946BB
:10CDF000002001F043F91622DFF8E01B6846FFF738
:10CE0000A7FB6946012001F039F9DFF8B0369BA293
:10CE100016216846FFF7F7FC6946052001F02EF958
:10CE2000CDA42100022001F029F92100032001F006
:10CE300025F92100042001F021F92100062001F04C
:10CE40001DF92100072001F019F92100082001F047
:10CE500015F9042001F0DDF8032001F032F9082073
:10CE600002F04BFA002809D00420FDF7FBFF002058
:10CE70008021FBF715FC02F0B0F806E0012002F07B
:10CE80003CFA002801D002F0A8F806B010BD38B571
:10CE90008EB0040070200021FBF702FCDFF85C3646
:10CEA000AEA2162108A8FFF7AEFC236BDFF84C2CCE
:10CEB000162102A8FFF7A7FC042001F0AAF804201D
:10CEC00001F0FFF8002001F0A8F808A9002001F007
:10CED000D5F802A9012001F0D1F89FA52900022070
:10CEE00001F0CCF82900032001F0C8F82900042043
:10CEF00001F0C4F82900052001F0C0F8290006203F
:10CF000001F0BCF82900072001F0B8F8290008203A
:10CF100001F0B4F8012002F0F0F9002802D002F08C
:10CF20005CF82BE0082002F0E8F900281BD0206B09
:10CF3000E16B884207D0216B1420FEF798F800209F
:10CF40000221FBF7ADFB02217E2001F0EEFF4FF442
:10CF50008040FEF757F8002802D0012020630DE042
:10CF6000002020630AE001200190002000900123AE
:10CF700014226421206B02F0BDF820630FB030BD95
:10CF800038B58EB0040070200021FBF789FBDFF874
:10CF90006C3572A2162108A8FFF735FC08A90020FD
:10CFA00001F06CF8206B002806D11622DFF84C1C2B
:10CFB00002A8FFF7CDFA05E0DFF8442C162102A8FD
:10CFC000FFF721FC042001F024F8042001F079F897
:10CFD000002001F022F802A9012001F04FF85EA51F
:10CFE0002900022001F04AF82900032001F046F848
:10CFF0002900042001F042F82900052001F03EF844
:10D000002900062001F03AF82900072001F036F83F
:10D010002900082001F032F8082002F06EF90028FB
:10D0200016D0E06B216B88420FD0206B002804D112
:10D030004FF48040FDF7EFFF03E04FF48040FDF731
:10D04000E5FF00200821FBF72BFB01F0C6FF12E0F3
:10D05000012002F052F9002802D001F0BEFF0AE0E0
:10D060000020019001200090012300220121206B6B
:10D0700002F040F820630FB030BD000025733F0080
:10D0800038B58EB0040070200021FBF709FB162292
:10D09000DFF85C1508A8FFF75BFA236BDFF8582C64
:10D0A000162102A8FFF7AFFB042000F0B2FF042016
:10D0B00001F007F8002000F0B0FF08A9002000F000
:10D0C000DDFF02A9012000F0D9FF23A529000220DD
:10D0D00000F0D4FF2900032000F0D0FF2900042035
:10D0E00000F0CCFF2900052000F0C8FF2900062031
:10D0F00000F0C4FF2900072000F0C0FF290008202D
:10D1000000F0BCFF082002F0F8F800280ED0206BD9
:10D11000E16B884207D0216B3C20FDF7A8FF00207F
:10D120000421FBF7BDFA01F058FF12E0012002F0E4
:10D13000E4F8002802D001F050FF0AE0012001903D
:10D1400000200090012302221821206B01F0D2FF61
:10D1500020630FB030BD0000000000002573000008
:10D1600038B58EB0040070200021FBF799FA162222
:10D17000D44908A8FFF7ECF9206B002806D1162245
:10D18000DFF8781C02A8FFF7E3F905E01622DFF8C4
:10D19000701C02A8FFF7DCF9042000F03AFF04201D
:10D1A00000F08FFF002000F038FF08A9002000F0F9
:10D1B00065FF02A9012000F061FFBFA52900022040
:10D1C00000F05CFF2900032000F058FF2900042034
:10D1D00000F054FF2900052000F050FF2900062030
:10D1E00000F04CFF2900072000F048FF290008202C
:10D1F00000F044FF082002F080F8002814D0206BD3
:10D20000E16B88420DD0206B002803D14020FDF750
:10D2100002FF02E04020FDF7F9FE00200821FBF7A5
:10D220003FFA01F0DAFE12E0012002F066F8002871
:10D2300002D001F0D2FE0AE000200190012000900F
:10D24000012300220121206B01F054FF20630FB065
:10D2500030BD38B58EB0040070200021FBF720FAF5
:10D2600016229A4908A8FFF773F9206B002806D107
:10D270001622DFF8941B02A8FFF76AF905E01622D0
:10D28000DFF8881B02A8FFF763F9042000F0C1FE55
:10D29000042000F016FF002000F0BFFE08A90020C7
:10D2A00000F0ECFE02A9012000F0E8FE82A52900B2
:10D2B000022000F0E3FE2900032000F0DFFE290039
:10D2C000042000F0DBFE2900052000F0D7FE290035
:10D2D000062000F0D3FE2900072000F0CFFE290031
:10D2E000082000F0CBFE082002F007F8002816D036
:10D2F000E06B216B88420FD0206B002804D14FF4E3
:10D300008060FDF788FE03E04FF48060FDF77EFE4D
:10D3100000200821FBF7C4F901F05FFE12E00120B4
:10D3200001F0EBFF002802D001F057FE0AE00020D8
:10D33000019001200090012300220121206B01F0C7
:10D34000D9FE20630FB030BD20D4030038B58EB0B5
:10D35000040070200021FBF7A3F91622DFF8B01AB1
:10D3600008A8FFF7F5F8206B002806D11622DFF891
:10D37000A41A02A8FFF7ECF80FE0206B012806D1F1
:10D380001622DFF8941A02A8FFF7E2F805E0162249
:10D39000DFF8881A02A8FFF7DBF8042000F039FE56
:10D3A000042000F08EFE002000F037FE08A90020C7
:10D3B00000F064FE02A9012000F060FE3EA52900F5
:10D3C000022000F05BFE2900032000F057FE290038
:10D3D000042000F053FE2900052000F04FFE290034
:10D3E000062000F04BFE2900072000F047FE290030
:10D3F000082000F043FE082001F07FFF002846D0FF
:10D40000206B00280AD100215D20FDF730FE4FF48B
:10D410008070FDF700FE01F0E0FD33E0206B012895
:10D4200026D15D20FDF7FDFD002803D0E06B216BC8
:10D43000884207D001215D20FDF719FE0020082158
:10D44000FBF72EF94FF48070FDF7E5FDFCF71EFFAA
:10D45000012802D101F0C1FD14E05D20FDF7E1FDDE
:10D460002063206BE06302217C2001F05EFD09E077
:10D470004FF48070FDF7CAFD00215D20FDF7F7FD38
:10D4800001F0ABFD00200821FBF70AF912E00120B2
:10D4900001F033FF002802D001F09FFD0AE00020D8
:10D4A000019001200090012300220221206B01F055
:10D4B00021FE20630FB030BD0000000020DB030020
:10D4C000D0FC010080DB0300D8FC0100E0F3030086
:10D4D000E0FC0100C0DB0300E8FC010000DC03000D
:10D4E000F0FC010020DC0300F8FC010040DC03003C
:10D4F00000FD010000E1030008FD010040D503002C
:10D5000038B58EB0040070200021FBF7C9F8DFF8B1
:10D5100008090090DFF80839DFF80829162108A863
:10D52000FFF771F9236BA4A2162102A8FFF76BF98C
:10D53000042000F06EFD08A9002000F09FFD02A964
:10D54000012000F09BFDD8A52900022000F096FDE7
:10D550002900032000F092FD2900042000F08EFD38
:10D560002900052000F08AFD2900062000F086FD34
:10D570002900072000F082FD2900082000F07EFD30
:10D58000002000F04AFD082001F0B7FE00280ED070
:10D59000206BE16B884207D0216B5D20FDF767FDB2
:10D5A00000200821FBF77CF801F017FD19E00120AD
:10D5B00001F0A3FE002802D001F00FFD11E0FCF7FE
:10D5C00065FE012802D1012020630AE000200190BD
:10D5D00001200090012301220A21206B01F08AFD25
:10D5E00020630FB030BD0000E0DB030010FD010040
:10D5F00060DB030018FD010038B58EB00400702018
:10D600000021FBF74DF81622DFF81C1808A8FEF7DA
:10D610009FFF236BDFF81428162102A8FFF7F3F809
:10D62000042000F0F6FC042000F04BFD002000F088
:10D63000F4FC08A9002000F021FD02A9012000F05F
:10D640001DFD99A52900022000F018FD29000320E6
:10D6500000F014FD2900042000F010FD2900052031
:10D6600000F00CFD2900062000F008FD290007202D
:10D6700000F004FD2900082000F000FD082001F062
:10D680003CFE00280ED0206BE16B884207D0216B56
:10D690003D20FDF7ECFC00200421FBF701F801F030
:10D6A0009CFC12E0012001F028FE002802D001F0CD
:10D6B00094FC0AE001200190002000900123012247
:10D6C0005F21206B01F016FD20630FB030BD00001C
:10D6D00020FD010000F5030038B58EB00400702075
:10D6E0000021FAF7DDFF1622DFF8441708A8FEF73D
:10D6F0002FFF206B002806D11622DFF8381702A86A
:10D70000FEF726FF05E01622DFF82C1702A8FEF729
:10D710001FFF042000F07DFC042000F0D2FC00205C
:10D7200000F07BFC08A9002000F0A8FC02A9012061
:10D7300000F0A4FC5CA52900022000F09FFC290059
:10D74000032000F09BFC2900042000F097FC290036
:10D75000052000F093FC2900062000F08FFC290032
:10D76000072000F08BFC2900082000F087FC08202F
:10D7700001F0C3FD002809D0206BE16B884202D084
:10D78000206B02F0D7FA01F028FC12E0012001F032
:10D79000B4FD002802D001F020FC0AE00020019036
:10D7A00001200090012300220121206B01F0A2FC46
:10D7B00020630FB030BD00002532640038B58EB054
:10D7C000040070200021FAF76BFF1622DFF86C16B8
:10D7D00008A8FEF7BDFE206B002806D11622DFF850
:10D7E000601602A8FEF7B4FE05E01622DFF8241644
:10D7F00002A8FEF7ADFE042000F00BFC042000F0B0
:10D8000060FC002000F009FC08A9002000F036FCB4
:10D8100002A9012000F032FC23A52900022000F01B
:10D820002DFC2900032000F029FC2900042000F031
:10D8300025FC2900052000F021FC2900062000F02D
:10D840001DFC2900072000F019FC2900082000F029
:10D8500015FC082001F051FD002810D0206BE16B71
:10D86000884209D0206B002803D1002000F0BBFBC8
:10D8700002E0012000F0B7FB01F0AFFB12E0012055
:10D8800001F03BFD002802D001F0A7FB0AE00020D8
:10D89000019001200090012300220121206B01F062
:10D8A00029FC20630FB030BD0000000038B58EB0F9
:10D8B000040070200021FAF7F3FE1622DFF8841529
:10D8C00008A8FEF745FEDFF880358BA2162102A8D6
:10D8D000FEF799FF02A9012000F0D0FB206B002881
:10D8E00007D1DFF83035C2A2162102A8FEF78BFF60
:10D8F00005E0236BBFA2032102A8FEF784FF02A963
:10D90000052000F0BBFB042000F083FB042000F0A6
:10D91000D8FB002000F081FB08A9002000F0AEFB3E
:10D92000B5A52900022000F0A9FB2900032000F082
:10D93000A5FB2900042000F0A1FB2900062000F02F
:10D940009DFB2900072000F099FB2900082000F02A
:10D9500095FB082001F0D1FC002822D0206BE16B60
:10D96000884212D04F20FDF75CFB10F0F00094F8D5
:10D97000301011F00F0108432063216B4F20FDF799
:10D9800076FB00200821FAF78BFE0221782001F0B7
:10D99000CCFA4F20FDF745FB00092063206BE063C4
:10D9A00019E0012001F0A9FC002802D001F015FBCC
:10D9B00011E0FCF76BFC012802D10022032101E0F9
:10D9C00000220A2101200190012000900123206BF8
:10D9D00001F090FB20630FB030BD000040DB03007E
:10D9E00038B58EB0040070200021FAF759FE1622D7
:10D9F000DFF8501408A8FEF7ABFDDFF850343EA264
:10DA0000162102A8FEF7FFFE02A9012000F036FB56
:10DA1000206B002807D1DFF8FC3375A2162102A87D
:10DA2000FEF7F1FE05E0236B72A2032102A8FEF7C8
:10DA3000EAFE02A9052000F021FB042000F0E9FA2B
:10DA4000042000F03EFB002000F0E7FA08A90020C7
:10DA500000F014FB68A52900022000F00FFB29004C
:10DA6000032000F00BFB2900042000F007FB290035
:10DA7000062000F003FB2900072000F0FFFA290030
:10DA8000082000F0FBFA082001F037FC002817D02E
:10DA9000206BE16B884210D04F20FDF7C2FA10F0E6
:10DAA0000F00216B50EA01102063216B4F20FDF71E
:10DAB000DEFA00200821FAF7F3FD01F08EFA19E0F2
:10DAC000012001F01AFC002802D001F086FA11E0D2
:10DAD000FCF7DCFB012802D10122032101E0002236
:10DAE0000A2101200190002000900123206B01F009
:10DAF00001FB20630FB030BD25733A0028FD010003
:10DB000038B58EB0040070200021FAF7C9FD162246
:10DB1000CF4908A8FEF71CFD206B002805D116226E
:10DB2000CC4902A8FEF714FD04E01622B94902A868
:10DB3000FEF70EFD042000F06CFA042000F0C1FA9C
:10DB4000002000F06AFA08A9002000F097FA02A964
:10DB5000012000F093FA28A52900022000F08EFA97
:10DB60002900032000F08AFA2900042000F086FA38
:10DB70002900052000F082FA2900062000F07EFA34
:10DB80002900072000F07AFA2900082000F076FA30
:10DB9000082001F0B2FB002814D0206BE16B884212
:10DBA0000DD0206B002803D18020FDF734FA02E06D
:10DBB0008020FDF72BFA00200821FAF771FD01F013
:10DBC0000CFA12E0012001F098FB002802D001F0CD
:10DBD00004FA0AE0002001900020009001230022B6
:10DBE0000121206B01F086FA20630FB030BD0000E8
:10DBF00025730000256400000000000020F40300ED
:10DC00008CF4010038B58EB0040070200021FAF7C2
:10DC100047FD1622904908A8FEF79AFC206B0028C1
:10DC200005D016228B4902A8FEF792FC04E01622CA
:10DC3000784902A8FEF78CFC042000F0EAF90420E1
:10DC400000F03FFA002000F0E8F908A9002000F0F9
:10DC500015FA02A9012000F011FA6AA52900022094
:10DC600000F00CFA2900032000F008FA2900042033
:10DC700000F004FA2900052000F000FA290006202F
:10DC800000F0FCF92900072000F0F8F9290008202D
:10DC900000F0F4F9082001F030FB002816D0206BCA
:10DCA000E16B88420FD0206B002804D14FF4006054
:10DCB000FDF7B1F903E04FF40060FDF7A7F900208C
:10DCC0000821FAF7EDFC01F088F912E0012001F0DB
:10DCD00014FB002802D001F080F90AE00020019036
:10DCE00001200090012300220121206B01F002FAA3
:10DCF00020630FB030BD000030FD010038B58EB09C
:10DD0000040070200021FAF7CBFC1622534908A822
:10DD1000FEF71EFC206B002805D016224D4902A8F4
:10DD2000FEF716FC04E016223A4902A8FEF710FCA2
:10DD3000042000F06EF9042000F0C3F9002000F088
:10DD40006CF908A9002000F099F902A9012000F05F
:10DD500095F92CA52900022000F090F92900032054
:10DD600000F08CF92900042000F088F92900052032
:10DD700000F084F92900062000F080F9290007202E
:10DD800000F07CF92900082000F078F9082001F063
:10DD9000B4FA002816D0206BE16B88420FD0206BBC
:10DDA000002804D14FF48050FDF735F903E04FF41B
:10DDB0008050FDF72BF900200821FAF771FC01F0E3
:10DDC0000CF919E0012001F098FA002802D001F0C6
:10DDD00004F911E0FCF79AFA012802D1002020632F
:10DDE0000AE000200190012000900123002201217F
:10DDF000206B01F07FF920630FB030BDC0DC030061
:10DE0000A0DC03000000000060F2030040F4030007
:10DE1000E0DC030080E6030020DD030000DD0300FA
:10DE200000D6030038FD0100E0DB030040FD0100E7
:10DE300000DC030040DD030060DD030000E10300BF
:10DE4000E0EA030020DC0300A0D5030080D5030036
:10DE500040DC0300E0D9030028F8010000F50300CE
:10DE600010B5DFF8344A10212000FEF71AF910220D
:10DE700010212000FEF705F9DFF84C4C0422282180
:10DE80002000FEF795FA2068002804D020680128B9
:10DE900001D00020206001F05FFF0020DFF82C1C83
:10DEA0000870FCF75DF80A38DFF8241C08600120D0
:10DEB000DFF8201C086010BD10B5DFF8180C0068F2
:10DEC000002800F08B80FCF74BF8DFF8044C216849
:10DED000401A0A28C0F07F80FCF742F820604FF417
:10DEE00080400021FDF77EFB002906D1002804D1E7
:10DEF000DFF8D40B0068012830D1012002F0B5FA18
:10DF000000280ED1022002F0B0FA002809D1042026
:10DF100002F0ABFA002804D1082002F0A6FA00288B
:10DF200004D0FCF71DF8DFF8641C0860FCF718F853
:10DF3000DFF8581C0968401ADFF8541C884206D3E1
:10DF400000221021DFF85009FEF79BF811E01022A3
:10DF50001021DFF84409FEF794F80AE0102210219E
:10DF6000DFF83409FEF78DF8FBF7FAFFDFF81C1C29
:10DF70000860DFF8201C0868401C086064200A68FC
:10DF80000968B1FBF0F100FB1120002801D102F07B
:10DF9000ADFADFF8380B0178012902D100F03BF926
:10DFA00019E00178022902D100F071FA13E001783A
:10DFB000032902D100F08EFB0DE00178042902D183
:10DFC00000F019FC07E00078052802D100F066FC9B
:10DFD00001E000F0B1F80420FBF7C5FF10BDDFF849
:10DFE000E80A0068704780B5002801D0012806D1F2
:10DFF000DFF8D42A106028211068FEF739FA01BD35
:10E00000DFF8940B0068002801D0012000E0002018
:10E010007047DFF8B81A08707047DFF8B01A0A784E
:10E02000032A0AD1052803D2DFF8081D086024E07E
:10E030000020DFF8001D08601FE00A78042A0AD1DA
:10E04000092803D2DFF8EC1C086016E00020DFF896
:10E05000E41C086011E00A78052A03D1DFF8D41C1B
:10E0600008600AE00978012903D1DFF8C81C0860BC
:10E0700003E00020DFF8BC1C0860704730B40023C8
:10E080000AE0DFF8B44C0500EDB21622554304EB6C
:10E090000502CC5CD4545B1CCA5C002A01D0152B51
:10E0A000EFD31621DFF8902C0400E4B24C43144463
:10E0B0000025E554C0B2484310440021417530BCEE
:10E0C000704780B5DFF8741CC0B20860086800288B
:10E0D00005D1DFF86C0CDFF86C1C08602BE00868D9
:10E0E000012805D1DFF8600CDFF8581C086022E039
:10E0F0000868022805D1DFF8540CDFF8481C0860D6
:10E1000019E00868032805D1DFF8440CDFF8341C57
:10E11000086010E00868042805D1DFF8380CDFF843
:10E12000241C086007E0DFF8180CDFF8181C0860F2
:10E130000120FBF7F7FF01BDF0B585B0DFF8184C03
:10E1400001F02CFE2060002005E0DFF8101C095CC7
:10E1500022681154401CB0F5806FF6D3DFF8004CF4
:10E1600025000021686840686A68126A9047686103
:10E1700025007FF07F41686840686A68126A9047AE
:10E1800028612500DFF8DC6BA86902F081FC07003C
:10E190005FF0FF323100280002F098FA002101916F
:10E1A0007F08D7F105070097022190FBF1F3D3F127
:10E1B00040035FF0FF323100280002F0BBFA31204B
:10E1C00000903423DFF8A02B0C2102A8FEF71BFBE4
:10E1D000250002AEA86902F05BFC07005FF0FF3289
:10E1E0003100280002F072FA002101917F08D7F176
:10E1F00037070097022190FBF1F3D3F140035FF062
:10E20000FF323100280002F095FA61684868496AD7
:10E21000884705B0F0BD2DE9FE43DFF83C5B01F017
:10E22000BDFD2860002003E000212A681154401C35
:10E23000B0F5806FF8D3DFF8284B26000021706816
:10E2400040687268126A9047706126007FF07F41D3
:10E25000706840687268126A90473061DFF80C1B82
:10E26000200002F09EFC2700DFF8CC6A16F58478C7
:10E27000B86902F00DFC81465FF0FF32414638007C
:10E2800002F024FA002101915FEA5909D9F1050948
:10E29000CDF80090022190FBF1F3D3F140035FF041
:10E2A000FF324146380002F045FADFF8C41A200078
:10E2B00002F077FC270016F1DC08B86902F0E8FBF1
:10E2C00081465FF0FF324146380002F0FFF900213D
:10E2D00001915FEA5909D9F11209CDF800900221A4
:10E2E00090FBF1F3D3F140035FF0FF324146380079
:10E2F00002F020FA270016F1C608B86902F0C8FB40
:10E3000081465FF0FF324146380002F0DFF900211C
:10E3100001915FEA5909D9F11D09CDF80090022158
:10E3200090FBF1F3D3F140035FF0FF324146380038
:10E3300002F000FA2700F236B86902F0A9FB804625
:10E340005FF0FF323100380002F0C0F90021019186
:10E350005FEA5808D8F13508CDF80080022190FB1B
:10E36000F1F3D3F140035FF0FF323100380002F0E7
:10E37000E1F90220FCF792FC00280DD028680290F9
:10E38000DFF8F009019000200090152315222B21C1
:10E39000002001F00FFD0EE00120FCF77FFC296852
:10E3A0000291DFF8D01901910090152315222B213D
:10E3B000002001F0FFFC0220FCF770FC29680291AC
:10E3C000DFF8B41901910090152315222B21162096
:10E3D00001F0F0FC28680290DFF8A009019000200D
:10E3E0000090152315222B21552001F0E3FC28680D
:10E3F0000290DFF88C09019000200090152315226F
:10E400002B216B2001F0D6FCDFF828693078C0079B
:10E410000CD528680290DFF86C090190002000906C
:10E42000082307220221022001F0C4FC3078800773
:10E4300009D5002001900D20009003230122A3A103
:10E44000200002F077F9307840070DD52868029057
:10E45000DFF83409019000200090092307220221EF
:10E46000772001F0A7FC0CE03078000709D50020E8
:10E470000190022000907723012295A1200002F054
:10E4800059F961684868496A8847BDE8F7832DE90A
:10E49000F84F84B0DFF8C04801F080FC2060002015
:10E4A0000AE000212268115405E0B0F5807FF8D21F
:10E4B000012122681154401CB0F5806F05D28028DC
:10E4C000F3D2FF2122681154F5E70120FCF7E6FBA7
:10E4D00000281BD10220FCF7E1FB002816D12020E8
:10E4E000FCF7DCFB002802D0DFF8A05810E0402049
:10E4F000FCF7D4FB002806D0FBF7C8FE002802D1A9
:10E50000DFF88C5804E0DFF88C5801E0DFF8885819
:10E510002020FCF7C3FB002829D10120FCF7BEFB1B
:10E52000002824D10220FCF7B9FB00281FD11020BD
:10E53000FCF7B4FB002807D00820FCF7AFFB00284D
:10E5400002D0DFF8586814E01020FCF7A7FB002881
:10E5500002D0DFF84C680CE00820FCF79FFB002895
:10E5600002D0DFF8406804E0DFF83C6801E0DFF843
:10E5700028680420FCF792FB002802D0DFF82C78F2
:10E5800001E0DFF82C78DFF8D887C2467FF07F49BA
:10E590004946DAF804004068DAF80420126A904725
:10E5A000CAF81400C2460021DAF804004068DAF81C
:10E5B0000420126A9047CAF81000CDF80880DFF8EE
:10E5C00078A7CDF80CA00298806902F061FA834622
:10E5D0005FF0FF320399029802F078F80021019170
:10E5E0005FEA5B0BDBF1030BCDF800B0022190FB7F
:10E5F000F1F3D3F140035FF0FF320399029802F088
:10E6000099F82068029001950020009015231522AA
:10E610001421052001F0CEFB206802900196002015
:10E620000090152315221421242001F0C3FB20683B
:10E6300002900197002000901523152214214520F7
:10E6400001F0B8FB20680290DFF868070190002015
:10E650000090152315221421652001F0ABFB4446E0
:10E660000021606840686268126A904760614446B1
:10E670004946606840686268126A90472061444673
:10E680001AF1C605A06902F003FA06005FF0FF3236
:10E690002900200002F01AF8002101917608D6F135
:10E6A00034060096022190FBF1F3D3F140035FF0B2
:10E6B000FF322900200002F03DF8D8F80410486825
:10E6C000496A884705B0BDE8F08F0000540000009B
:10E6D0002A0000002DE9FE4300F0FEF9DFF8804635
:10E6E00026007FF07F452900706840687268126AD2
:10E6F0009047706126000021706840687268126A55
:10E70000904730612700DFF83066B046B86902F004
:10E71000BFF981465FF0FF324146380001F0D6FF75
:10E72000002101915FEA5909D9F10309CDF8009060
:10E73000022190FBF1F3D3F140035FF0FF32414639
:10E74000380001F0F7FF27000021786840687A68F8
:10E75000126A9047786127002900786840687A68D3
:10E76000126A90473861002001900D200090082324
:10E770005FF0FF3216F11601200001F0DBFF0020F0
:10E7800001901720009008235FF0FF3216F12C0152
:10E79000200001F0CFFF00200190212000900823ED
:10E7A0005FF0FF3216F14201200001F0C3FF0020AC
:10E7B00001902B20009008235FF0FF3216F15801E2
:10E7C000200001F0B7FFDFF86C15086800280CD0B6
:10E7D0000020019009680A204143C91C00910123CF
:10E7E0000122B8A1200001F0A5FF61684868496ACC
:10E7F0008847BDE8F7832DE9FC4100F06DF9DFF8AB
:10E80000604526007FF07F45290070684068726887
:10E81000126A904770612600002170684068726833
:10E82000126A904730612600DFF80C75B06902F07B
:10E830002FF980465FF0FF323900300001F046FFCB
:10E84000002101915FEA5808D8F10308CDF8008053
:10E85000022190FBF1F3D3F140035FF0FF32390066
:10E86000300001F067FF2600002170684068726880
:10E87000126A9047706126002900706840687268CB
:10E88000126A9047306100F089F961684868496A06
:10E890008847BDE8F3810000005000402DE9F84FA3
:10E8A00084B002A8052102F07FF900F015F9DFF825
:10E8B000B04426007FF07F45290070684068726888
:10E8C000126A904770612600002170684068726883
:10E8D000126A904730612600DFF85C74B06902F07C
:10E8E000D7F880465FF0FF323900300001F0EEFECD
:10E8F000002101915FEA5808D8F10308CDF80080A3
:10E90000022190FBF1F3D3F140035FF0FF323900B5
:10E91000300001F00FFF00264CE0A146DFF898041C
:10E92000052101FB06F100EB010AD9F8180002F0FD
:10E93000AFF883465FF0FF325146484601F0C6FE0D
:10E9400001210191B8EB5B08CDF80080022190FB1A
:10E95000F1F03F1A3B005FF0FF325146484601F0AC
:10E96000E9FE26E0062E05D0072E03D0082E01D0A2
:10E97000092ED2D1A1460DF1080AD9F8180002F0EB
:10E9800087F883465FF0FF325146484601F09EFE0D
:10E9900001210191B8EB5B08CDF80080022190FBCA
:10E9A000F1F03F1A3B005FF0FF325146484601F05C
:10E9B000C1FE761C102E7DD216F0030F01D1102758
:10E9C0000CE016F00300012801D1302706E016F014
:10E9D0000300022801D1502700E07027042E02D244
:10E9E0005FF00F080BE0082E02D25FF0190806E076
:10E9F0000C2E02D25FF0230801E05FF02D08CD4815
:10EA00000068F040C00716D5A1462900D9F80400D7
:10EA10004068D9F80420126A9047C9F81400A1464A
:10EA20000021D9F804004068D9F80420126A904700
:10EA3000C9F8100015E0A1460021D9F8040040688B
:10EA4000D9F80420126A9047C9F81400A146290099
:10EA5000D9F804004068D9F80420126A9047C9F830
:10EA60001000FBF713FC01287FF47CAFA146D248CD
:10EA7000052101FB06F100EB010AD9F8180002F0AC
:10EA800007F883465FF0FF325146484601F01EFE0C
:10EA900001210191B8EB5B08CDF80080022190FBC9
:10EAA000F1F03F1A3B005FF0FF325146484601F05B
:10EAB00041FE7EE761684868496A884705B0BDE85D
:10EAC000F08F00003E0000002811002038120020C6
:10EAD0002C1100201011002070B59F4C01F05EF940
:10EAE000206000200BE0974B1B680B4493F88030AC
:10EAF00025685618AB55491C8029F4D3401C0828BA
:10EB000042D2002809D1002200218029F6D2FF2319
:10EB100025685618AB55491CF7E701280BD1802210
:10EB200002FB00F200218029E8D201232568561853
:10EB3000AB55491CF7E7022805D0032803D0042869
:10EB400001D005280BD1802202FB00F20021802990
:10EB5000D4D2002325685618AB55491CF7E7062880
:10EB60000DD1802202FB00F200218029C6D2754B14
:10EB70001B685B5C25685618AB55491CF5E780227D
:10EB800002FB00F20021B7E770BD00002411002055
:10EB9000C1D4010030110020405000402DE9F8435D
:10EBA0008AB001220EE0491C6348162303FB02F3DE
:10EBB0001844405C0028F6D102A800EB820040F81F
:10EBC000041C521C092A01D20021EDE702A9029D72
:10EBD0004868451904984519059845190C6948690C
:10EBE0000419089804190998041906267543D5F1E3
:10EBF00080056D0801274BE0DFF86481C1460021E4
:10EC0000D9F804004068D9F80420126A9047C9F87E
:10EC100014007FF07F41D8F804004068D8F8042041
:10EC2000126A9047C8F810001BE042480068B842DA
:10EC3000E2D1DFF82C81C1467FF07F41D9F8040092
:10EC40004068D9F80420126A9047C9F814000021DE
:10EC5000D8F804004068D8F80420126A9047C8F831
:10EC6000100001200190142000902B005FF0FF3273
:10EC70003148162101FB07F10144394801F05AFDE2
:10EC800002A800EB870050F8040C06FB00557F1C1F
:10EC9000052FCAD37443D4F180046408052543E0EA
:10ECA0002F4FB8460021D8F804004068D8F8042057
:10ECB000126A9047C8F814007FF07F417868406876
:10ECC0007A68126A9047386117E01A480068A842CB
:10ECD000E6D1234FB8467FF07F41D8F80400406862
:10ECE000D8F80420126A9047C8F814000021786808
:10ECF00040687A68126A90473861012001902020AC
:10ED0000009023005FF0FF320B48162101FB05F154
:10ED10000144134801F00EFD02A800EB850050F8F5
:10ED2000040C06FB00446D1C092DCED30BB0BDE8CE
:10ED3000F08300001C110020800900202011002019
:10ED4000ECE4010018110020ECE20100ECE301000A
:10ED5000ECE10100ECE0010014110020E4D9010015
:10ED6000B40F002018F801007CF30100B4E60100A4
:10ED7000ECE5010080EC0100C0EC010040ED010079
:10ED800000ED010020F801008CF3010080ED01008E
:10ED900000F00100C0ED0100C0EE010000EF010035
:10EDA00040EE010080EE010000EE010080EF010066
:10EDB00040EF0100C0EF010030EC010010B5DFF8BA
:10EDC0004445002060610321002000F0AEF80120DE
:10EDD000206010BD80B51F2001F047FBDFF824152F
:10EDE0008A6C42400A650A6D82430A658A6C424019
:10EDF000CA64CA6C0240CA64886401BD10B51020A0
:10EE000001F033FB002801D0002400E0012400F0D1
:10EE10008EFF00280BD1DFF8EC0400218160012C6B
:10EE200002D1002141600DE0012141600AE0DFF8DC
:10EE3000D40400214160012C02D10121816001E054
:10EE400000218160DFF8BC044068012803D1032160
:10EE5000012000F06AF810BD30B4DFF8A814DFF824
:10EE6000A824031F4C6952F82440A34203D2031F75
:10EE70004C6942F82430DFF894244B6952F823306F
:10EE8000042B03D303234C6942F82430DFF8803489
:10EE90004C6953F82440844203D3441E4D6943F81F
:10EEA0002540052805D2486953F82000496942F8F1
:10EEB000210030BC7047002807D1DFF85004DFF88C
:10EEC0004414496950F8210010E0012807D1DFF807
:10EED0004004DFF83014496950F8210006E0DFF8FB
:10EEE0002804DFF82014496950F8210070470028F1
:10EEF00007D1DFF81804DFF80C24526940F822101B
:10EF000012E0012807D1DFF80804DFF8F82352697E
:10EF100040F8221008E0022806D1DFF8EC03DFF801
:10EF2000E423526940F82210704738B50400080005
:10EF3000C0B201280BD1DFF8CC034169072903D205
:10EF40004169491C416109E00021416106E0C9B203
:10EF5000022903D00020DFF8AC134861DFF8A45386
:10EF6000DFF8B00369694454FAF7FAFFA861FAF7C9
:10EF7000F7FFE8610020DFF890136A6941F822008A
:10EF80000020DFF888136A6941F822000020DFF8CA
:10EF900080136A6941F822000020E8622000C0B2B4
:10EFA000122819D02000C0B2132815D02000C0B2FA
:10EFB000142811D0E4B2152C0ED000200AE0302124
:10EFC00005EB000282F82010302105EB000282F8E8
:10EFD0002510401C0528F2D331BDDFF828134869FD
:10EFE000002802D04869401E48610020C86270476E
:10EFF000DFF82003C3494969405C7047C148704746
:10F00000C448C0494969084410F8010C704738B534
:10F0100004000325641EAC4200D22500042000F049
:10F0200067F9002830D00020FFF745FFA84215D32C
:10F030000120FFF740FFA0425BD20120FFF73BFF1A
:10F040000100491C0120FFF752FF0220FFF733FFA8
:10F050000100491C0220FFF74AFF4AE00120FFF7A8
:10F060002AFFA04245D20120FFF725FF0100491CDD
:10F070000120FFF73CFF0020FFF71DFF0100491CA6
:10F080000020FFF734FF34E0022000F031F90028BF
:10F090002FD00020FFF70FFF002815D00120FFF729
:10F0A0000AFF002825D00120FFF705FF0100491EB7
:10F0B0000120FFF71CFF0020FFF7FDFE0100491EA5
:10F0C0000020FFF714FF14E00120FFF7F4FE0028F2
:10F0D0000FD00120FFF7EFFE0100491E0120FFF7CE
:10F0E00006FF0220FFF7E7FE0100491E0220FFF79E
:10F0F000FEFE31BD2DE9F84F06008A4614001F00C0
:10F100000B9D2800C0B200280DD1FAF729FF8249D3
:10F110000860FAF725FF814908604FF4FA708049CA
:10F12000086080490860022000F0E2F800280AD058
:10F130005FF001084FF4FA7079490860FAF710FFA0
:10F140007649086024E0022000F0CDF8002819D0AC
:10F15000FAF706FFDFF8C891DFF8C0B1DBF800105E
:10F16000401AD9F80010884209D35FF00108FAF775
:10F17000F7FECBF800009620C9F8000008E05FF029
:10F18000000805E05FF00008FAF7EAFE634908604E
:10F19000B146CDF800A00A9EB8F1010F1BD100982E
:10F1A000814513D2EDB2022D08D1022000F0A0F863
:10F1B000002803D10A2000FB079901E017EB090999
:10F1C000009848455CD2DDF8009059E0F6B2012E77
:10F1D00056D1A14654E0042000F08AF800280AD055
:10F1E0005FF0010B4FF4FA704E490860FAF7B8FE71
:10F1F0004949086024E0042000F075F8002819D07F
:10F20000FAF7AEFEDFF81C81DFF80CA1DAF8001087
:10F21000401AD8F80010884209D35FF0010BFAF7C2
:10F220009FFECAF800009620C8F8000008E05FF0D2
:10F23000000B05E05FF0000BFAF792FE364908601C
:10F24000BBF1010F1CD14C4515D2EDB2022D0CD1F2
:10F25000042000F04DF8002807D10A2000FB0741E8
:10F26000494502D200FB179901E0B9EB0709A14516
:10F2700006D2A14604E0F6B2012E01D1DDF80090DD
:10F280004846BDE8F28F70B404000026002500E077
:10F29000761CA05D0028FBD1D01A864215D2D21A66
:10F2A000921B02E0605D48556D1CB542FAD3002008
:10F2B00003E020234B556D1C401C9042F9D30020E5
:10F2C00048550CE0605D48556D1CD01A8542F9D355
:10F2D00000204855202001EB050202F8010C002017
:10F2E000887570BC70470749896CC0B20840704788
:10F2F0000449C96CC0B2084070470249096DC0B2E8
:10F3000008407047100F00202810002048100020EF
:10F3100068100020F01000208411002080110020CF
:10F32000881100208C11002010B5FFF747FDDFF891
:10F33000244A042220212000FDF73AF82068002802
:10F3400005D02068012802D0002000F0F3FC10BD99
:10F3500038B5FFF753FDFFF73DFDFFF749FE050008
:10F36000FFF74CFE04005FF0FF30FAF7E0FE0028E4
:10F3700008D02800C0B207280CD003210720FFF7CF
:10F38000D4FD07E02800C0B2072803D103210120E3
:10F39000FFF7CBFD00204FF48051FCF723F9002943
:10F3A00001D1002807D02800C0B2022803DB0321C6
:10F3B0000120FFF7BAFD2800C0B2002804D12000C8
:10F3C00001F0F6FB00F0A7BC2800C0B2012804D170
:10F3D000200001F011FC00F09EBC2800C0B20628FD
:10F3E00004D1200001F02CFF00F095BC2800C0B231
:10F3F000082804D1200002F0C3F900F08CBC2800DA
:10F40000C0B2072804D1200002F0CCF800F083BC81
:10F410002800C0B2022804D1200003F058F800F000
:10F420007ABC2800C0B2922804D1200002F0A0FBD0
:10F4300000F071BC2800C0B2032803D103F082F9A8
:10F4400000F069BC2800C0B2102804D1200002F0EE
:10F45000FAFB00F060BC2800C0B2112804D12000E3
:10F4600002F0B4FC00F057BC2800C0B2122804D14E
:10F47000200002F069FD00F04EBC2800C0B2132845
:10F4800004D1200002F04CFE00F045BC2800C0B2C0
:10F49000142804D1200002F02BFF00F03CBC28000F
:10F4A000C0B2152803D102F09DFF00F034BC280043
:10F4B000C0B2222804D1200003F0ACF900F02BBC2C
:10F4C0002800C0B2232804D1200003F035FA00F050
:10F4D00022BC2800C0B2242804D1200003F0CAFABC
:10F4E00000F019BC2800C0B2252804D1200003F088
:10F4F00079FC00F010BC2800C0B2092803D103F049
:10F5000097FD00F008BC2800C0B20C2803D103F01E
:10F5100063FF00F000BC2800C0B20A2802D103F04B
:10F5200013FDF8E32800C0B20B2802D103F025FE3A
:10F53000F1E32800C0B20D2802D103F0B3FEEAE3E4
:10F540002800C0B2162803D1200002F081FAE2E3BD
:10F550002800C0B2172803D1200003F09DFFDAE392
:10F560002800C0B2182803D1200004F02BF8D2E301
:10F570002800C0B2192803D1200004F0BBF8CAE368
:10F580002800C0B21A2803D1200004F021F9C2E3F8
:10F590002800C0B21B2803D1200004F0A3F9BAE36D
:10F5A0002800C0B21C2802D104F03AFAB3E32800C4
:10F5B000C0B21E2803D1200004F0A3FAABE3280058
:10F5C000C0B21F2803D1200004F0E4FBA3E328000D
:10F5D000C0B2202803D1200004F038FB9BE32800B0
:10F5E000C0B2212803D1200004F072FC93E328006C
:10F5F000C0B21D2802D104F0C9FD8CE32800C0B2BE
:10F60000402803D1200004F04DFE84E32800C0B25E
:10F61000412803D1200004F0D6FE7CE32800C0B2CC
:10F62000262803D1200004F0A1FF74E32800C0B213
:10F63000272803D1200005F0B8F96CE32800C0B2F8
:10F64000422803D1200005F0FDFD64E32800C0B28C
:10F65000432803D1200005F0F5FE5CE32800C0B28A
:10F66000442803D1200005F0ADFF54E32800C0B2C8
:10F67000452803D1200006F009F94CE32800C0B268
:10F68000472803D1200006F024F844E32800C0B244
:10F69000462803D1200006F086F83CE32800C0B2DB
:10F6A000482803D1200006F0B1F934E32800C0B2A5
:10F6B0004A2803D1200006F02FFE2CE32800C0B218
:10F6C000492803D1200006F017FD24E32800C0B22A
:10F6D0004B2803D1200007F005F81CE32800C0B236
:10F6E0004C2803D1200007F06BF814E32800C0B2C7
:10F6F0004D2803D1200007F0C3F90CE32800C0B265
:10F700004E2803D1200007F023F904E32800C0B2FB
:10F710004F2803D1200007F063FAFCE22800C0B2B2
:10F72000502803D1200007F0E9FAF4E22800C0B223
:10F73000512803D1200007F0B3FBECE22800C0B24F
:10F74000522803D1200007F017FCE4E22800C0B2E1
:10F75000532803D1200007F07FFCDCE22800C0B270
:10F76000542803D1200007F0E5FCD4E22800C0B201
:10F77000552803D1200007F05BFDCCE22800C0B281
:10F78000562803D1200007F0DBFDC4E22800C0B2F8
:10F79000572803D1200007F041FEBCE22800C0B288
:10F7A000582803D1200007F0E1FEB4E22800C0B2DF
:10F7B000592803D1200007F0A8FFACE22800C0B20E
:10F7C0005A2803D1200008F00FF8A4E22800C0B2A4
:10F7D0005B2803D1200008F07AF89CE22800C0B230
:10F7E0005C2803D1200008F0E1F894E22800C0B2C0
:10F7F0005D2803D1200008F047F98CE22800C0B250
:10F800005E2803D1200008F0B7F984E22800C0B2D6
:10F810005F2803D1200008F01DFA7CE22800C0B266
:10F82000602803D1200008F080FA74E22800C0B2FA
:10F83000612803D1200008F0E9FA6CE22800C0B288
:10F84000622802D108F086FB65E22800C0B2632876
:10F8500002D108F012FC5EE22800C0B2642802D196
:10F8600008F076FC57E22800C0B2652802D108F003
:10F87000DAFC50E22800C0B22C2803D1200005F0A9
:10F88000EAFB48E22800C0B27F2803D1200008F03C
:10F890004DFD40E22800C0B2802803D1200008F0CE
:10F8A0009CFE38E22800C0B2812803D1200008F075
:10F8B0002DFF30E22800C0B2832803D1200008F0D9
:10F8C000D3FF28E22800C0B2822803D1200009F02B
:10F8D00065F820E22800C0B2842803D1200009F096
:10F8E000EDF818E22800C0B2852803D1200009F005
:10F8F00044F910E22800C0B2862803D1200009F0A4
:10F9000091F908E22800C0B2872803D1200009F04D
:10F9100005FA00E22800C0B2882803D1200009F0CF
:10F9200037FBF8E12800C0B2892803D1200009F094
:10F930009CFDF0E12800C0B28A2803D1200009F024
:10F94000E7FBE8E12800C0B28B2803D1200009F0D2
:10F950008BFCE0E12800C0B28C2803D1200009F024
:10F9600020FDD8E12800C0B28D2803D1200009F085
:10F970005FFED0E12800C0B28E2803D1200009F03C
:10F980003DFFC8E12800C0B28F2803D1200009F054
:10F99000F6FFC0E12800C0B2902804D10121200068
:10F9A0000AF07EF8B7E12800C0B2912804D1022104
:10F9B00020000AF075F8AEE12800C0B22D2803D16E
:10F9C00020000AF021F9A6E12800C0B22E2803D1B8
:10F9D00020000AF000FA9EE12800C0B22F2803D1CF
:10F9E00020000AF011FB96E12800C0B2302803D1B4
:10F9F00020000AF08EFA8EE12800C0B2312803D12F
:10FA000020000AF08DFB86E12800C0B2322803D125
:10FA100020000AF021FC7EE12800C0B2332803D187
:10FA200020000AF019FD76E12800C0B2342803D185
:10FA300020000AF0C2FD6EE12800C0B2352803D1D3
:10FA400020000AF0A3FE66E12800C0B2362803D1E8
:10FA500020000AF02BFF5EE12800C0B2662803D127
:10FA600020000AF0DDFF56E12800C0B2282803D1AB
:10FA7000200005F00DF84EE12800C0B2292803D17E
:10FA8000200005F0E3F846E12800C0B22A2803D19F
:10FA9000200005F0A7F93EE12800C0B22B2803D1D1
:10FAA000200005F031FA36E12800C0B2672803D102
:10FAB00020000BF00FF92EE12800C0B2682803D116
:10FAC00020000BF008FA26E12800C0B2692803D113
:10FAD00020000BF079F91EE12800C0B26A2802D19B
:10FAE0000BF075FA17E12800C0B26B2802D10BF0B9
:10FAF000C9FA10E12800C0B26C2802D10BF038FB23
:10FB000009E12800C0B26D2802D10BF079FB02E1B7
:10FB10002800C0B26E2803D12000FCF7B9FEFAE03D
:10FB20002800C0B27C2803D12000FDF7E9FCF2E0F8
:10FB30002800C0B26F2803D12000FDF74BF9EAE09E
:10FB40002800C0B2702803D12000FDF7A0F9E2E040
:10FB50002800C0B27E2803D12000FDF711FADAE0B8
:10FB60002800C0B2712803D12000FDF789FAD2E045
:10FB70002800C0B2722803D12000FDF7F1FACAE0D4
:10FB80002800C0B2732803D12000FDF762FBC2E059
:10FB90002800C0B2742803D12000FDF7D7FBBAE0DB
:10FBA0002800C0B2752803D12000FDF725FDB2E082
:10FBB0002800C0B2762803D12000FDF78DFDAAE011
:10FBC0002800C0B2772803D12000FDF76FFEA2E025
:10FBD0002800C0B2782803D12000FDF701FF9AE089
:10FBE0002800C0B2792803D12000FDF789FF92E0F8
:10FBF0002800C0B27A2803D12000FEF703F88AE07B
:10FC00002800C0B27D2803D12000FDF7D7FD82E097
:10FC10002800C0B27B2803D12000FEF76FF87AE0FD
:10FC20002800C0B2932803D120000BF029FC72E019
:10FC30002800C0B2942803D120000BF0C4FC6AE075
:10FC40002800C0B2952803D120000BF02DFD62E002
:10FC50002800C0B2962803D120000BF0F5FD5AE031
:10FC60002800C0B2372803D120000BF077FE52E005
:10FC70002800C0B2382803D120000BF084FF4AE0EE
:10FC80002800C0B2392803D120000CF001F842E06E
:10FC90002800C0B23A2803D120000CF079FA3AE0EB
:10FCA0002800C0B23B2803D120000CF0B0F932E0AC
:10FCB0002800C0B23C2803D120000CF0F7FB2AE05A
:10FCC0002800C0B23D2803D120000CF08BFC22E0BC
:10FCD0002800C0B23E2803D120000CF021FD1AE01C
:10FCE0002800C0B23F2803D120000CF0DBFD12E059
:10FCF0002800C0B20E2803D1200001F0ADFC0AE0BC
:10FD0000EDB20F2D03D1200001F005FC03E003212B
:10FD10000120FFF70AF9FEF773F9002803D1032148
:10FD20000120FFF702F90220FAF71DF931BD094859
:10FD30000068704780B5002801D0012806D1054A27
:10FD4000106020211068FCF793FB02E00120FAF715
:10FD5000E9F901BD6411002038B5002003E000215D
:10FD60000F4A1154401C40F205418842F7D300F07D
:10FD7000E2FB0C4C0A4D402380222900200000F0B9
:10FD800075F8280000F004FB074D210028000DF055
:10FD90007BF80649280000F004FF31BD0448704795
:10FDA000C4020020E00F0020B40F0020ECE50100A9
:10FDB000C90200202DE9F0470A9C0D00ED0811F062
:10FDC0000701802606FB050004EB00051C00E40883
:10FDD00013F0070F00D0641CD2F1800300270898AD
:10FDE000099E01E01D447F1CA7423DD25FF0000C3C
:10FDF0009445F7D2002814D195F800E096F80080D9
:10FE000018FA01F858EA0E0E85F800E015F1800E98
:10FE100096F80080D1F1080958FA09F88EF80080A8
:10FE20001DE095F800E096F800807FEA080818FACF
:10FE300001F858EA0E0E85F800E015F1800E9EF8E4
:10FE4000008096F800907FEA0909D1F1080A59FA72
:10FE50000AF959EA080818F007088EF800806D1CA6
:10FE6000761C1CF1010CC3E7BDE8F08710B4282410
:10FE700004604160028143810FF23904C4600FF2D3
:10FE8000610404610FF2192444610FF24D2484616E
:10FE90000FF22934C4610FF2CD4404620FF2F14431
:10FEA000446201200870A1F80120A1F8033010BCC1
:10FEB0007047000030B4B0F80140082592FBF5F51A
:10FEC00004FB05110844401D12F0070201780124CB
:10FED0009440A14313FA02F20A43027030BC704707
:10FEE0002DE9F04105000C000698DDF81CC0089EC5
:10FEF000099FB5F80110C91D5FF0080E91FBFEFEC9
:10FF0000082194FBF1F102FB0E1205EB02014A1DE0
:10FF100014F00704D4F10704BCF1010F00F08C8049
:10FF2000BCF1040F04D0BCF1080F00F0B380B5E0C1
:10FF300013F00103DBB2002B02D0012B2FD081E0A4
:10FF4000002800F07F803378DBB21B09DBB203218D
:10FF50004B43FB5823F07F4315780121A1408D438B
:10FF6000C3F3074C44F6CD4EC3F3072849F20A7198
:10FF700001FB08F80EFB0C8C03F0FF0341F629414E
:10FF800001FB03C3DB0DA3402B43137021004C1E68
:10FF9000002901D10724521C401E0028D0D03378FC
:10FFA00013F00F0303214B43761CFB5823F07F43D0
:10FFB00015780121A1408D43C3F3074C44F6CD4E83
:10FFC000C3F3072849F20A7101FB08F80EFB0C8CF9
:10FFD00003F0FF0341F6294101FB03C3DB0DA340FE
:10FFE0002B43137021004C1E002901D10724521C01
:10FFF000401EA5E711785FF0010C1CFA04FC31EA01
:020000040001F9
:100000000C01D3F1070CAE463EFA0CFE1EF0010EB9
:1000100057F82EC01CFA04FC5CEA010111702100A3
:100020004C1E002901D10724521C5B1C401E082BCA
:1000300001DA0028DED10023002802D03578761CB2
:10004000F5E72BE02AE0337803214B43761CFB587D
:1000500023F07F4315780121A1408D43C3F3074C62
:1000600044F6CD4EC3F3072849F20A7101FB08F8A4
:100070000EFB0C8C03F0FF0341F6294101FB03C387
:10008000DB0DA3402B43137021004C1E002901D12E
:100090000724521C0100481E0029D4D1BDE8F0817C
:1000A00070B4039CB0F80150082693FBF6F605FBEC
:1000B00006152844451D13F0070309E02E7801209A
:1000C0009840864314FA03F006432E706D1C491CB9
:1000D0008A42F3DA70BC704770B4039CB0F80150E8
:1000E000082692FBF6F605FB06110844411D002C7C
:1000F00000D0FF2412F0070F19D012F00706D6F136
:100100000806981A401CB04201DA9E1A761C01209B
:1001100010FA06F6761E12F0070086400878B04303
:10012000264006430E702944D21D32F00702080013
:10013000C00705D5981A072802DB0C70294408323D
:100140000800800715D5981A0F2812DB0C7001EBF8
:100150000500047000EB050110320AE00C7001EBA1
:1001600005000470284404702844047000EB050165
:10017000203212F11F008342F0DA12F10F008342A5
:1001800006DB0C7001EB0500047000EB050110327A
:10019000D01D834202DB0C702944083293420ADBF3
:1001A000FF209A1A521C10FA02F208781040D2432B
:1001B000224002430A7070BC70470000F0B5B0F8EE
:1001C0000140B1F90230082593FBF5F5B1F9003093
:1001D00004FB05352844451D002A00D0FF22B1F953
:1001E000023013F0070F2DD013F00707D7F10807DF
:1001F000B1F90600C01A401CB84203DAB1F9067022
:10020000FF1A7F1C012010FA07F77F1E13F007006A
:100210008740B1F900C02E000CE096F800E03EEAFD
:10022000070E17EA020050EA0E0E86F800E01CF1F5
:10023000010C761CB1F904006045EEDA2544DB1DA3
:1002400033F007032800C00711D5B1F90600C01A22
:1002500007280CDBB1F90060280002E00270761C70
:10026000401CB1F90470B742F8DA2544083328007D
:1002700080071FD5B1F90600C01A0F281ADBB1F9A3
:100280000060280006E0028020442A80674238444B
:10029000761C401CB1F90470B742F4DA25441033DF
:1002A00008E00260761C401CB1F90470B742F8DA2D
:1002B00025440833B1F9060013F11F06B04203DBF1
:1002C000B1F900602800EFE7B1F9060013F10F065D
:1002D000B0421BDBB1F90060280002E00280761C0E
:1002E000401CB1F90470B742F8DA05EB040008339A
:1002F000B1F90060050002E02A80761C6D1CB1F99E
:100300000470B742F8DA00EB04050833B1F90600CF
:10031000DE1DB0420CDBB1F90060280002E0027083
:10032000761C401CB1F90470B742F8DA2544083352
:10033000B1F90600984214DBFF20CC88E31A5B1C5D
:1003400010FA03F3B1F9000007E02C781C40DE43FB
:10035000164034432C70401C6D1CB1F9044084429B
:10036000F3DAF0BD10B4C1F3074244F6CD43C1F354
:10037000072449F20A70444303FB024201F0FF01E3
:1003800041F6294000FB0121C90D080010BC70474F
:1003900080B500F020F901BD10B54A4C01212000C4
:1003A000FBF775FE0A23662201212000FBF7E8FD1A
:1003B00002212000FBF76BFE0A23662202212000A7
:1003C000FBF7DEFD04212000FBF761FE0A23662215
:1003D00004212000FBF7D4FD08212000FBF757FE85
:1003E0000A23662208212000FBF7CAFD8021364837
:1003F000FBF74DFEF9F7B4FD0A38344908600020D8
:100400003349086010BD10B5F9F7AAFD2F4C2168DB
:10041000401A0A2825D3F9F7A3FD206000202D49B2
:100420000968002901D150F001002B490968002911
:1004300001D150F0020029490968002901D150F08A
:10044000040027490968002901D150F00800254916
:100450000968002901D050F0100000F00BF81C4989
:1004600008600120F9F77FFD10BD19490968C0B285
:100470000840704730B402001000002304E01A491D
:1004800051F8231008435B1C032BF8D3164DE96881
:1004900008401300002403E055F824100B40641CAE
:1004A000032CF9D31843E860022106E005EB810331
:1004B00053F8043C45F82130491E0029F6D12A6042
:1004C00030BC704700700040005000405C110020BC
:1004D0005811002004700040087000401070004067
:1004E0002070004000520040A010002010B56A4C5F
:1004F000002201212000FBF7C4FD01220121200080
:10050000FBF7BFFDA02000F09FF8C82000F09CF88A
:10051000812000F099F81F2000F096F82F2000F0BD
:1005200093F8402000F090F8A62000F08DF8AF205E
:1005300000F08AF810BD7CB5584CFBF7B6FB206084
:100540005748FBF714FB5748FBF711FB5648FBF7DE
:100550000EFB564856490860FF2056490860564D24
:1005600028000CF0F5FC5548FBF7C5FD5448FBF797
:10057000C2FD494E06213000FBF7A5FD01213000E8
:10058000FBF78FFD4F4E04213000FBF78AFD082159
:100590003000FBF786FD082001904B4800900023B7
:1005A0000322216828000CF0ABFC28000CF0CAFCE8
:1005B000042204213000FBF764FD082208213000EA
:1005C000FBF75FFD20686421B0FBF1F0FBF7F4FA64
:1005D000FFF78CFF73BD2DE9F041441D002516E0A7
:1005E000354F38000CF0D5FC0028F9D121783800BF
:1005F0000CF0B4FC641C761C802EF1D30920FBF7B0
:10060000DBFA042204214046FBF73BFD6D1C082D5C
:1006100018D255F0B000C0B200F016F8102000F06B
:1006200013F8002000F010F8DFF898800022042171
:100630004046FBF726FD082208214046FBF721FD36
:100640000026D9E7BDE8F08170B504001D4D0022F9
:1006500008212800FBF715FD002204212800FBF7E4
:1006600010FD154E30000CF094FC0028F9D1E4B2D6
:10067000210030000CF072FC30000CF08AFC0028E5
:10068000FAD1042204212800FBF7FBFC08220821F0
:100690002800FBF7F6FC70BD00500240341100202A
:1006A000011C00F0010800F0050800F04B434F4C1E
:1006B00020550240245502400090004002040500ED
:1006C0000208050000500040002D3101FEB505462E
:1006D0000E461446002722E00146A86901AA00F050
:1006E000EEF9B0B9A86901AA2E2100F0E8F980B9A5
:1006F000A86901AA202100F0E2F950B90DF1060025
:1007000000900DF10703A86901AA0DF1050100F0A1
:10071000ABF99DF8040002993F180E44641A3CB1ED
:1007200002AB22463146284600F069F80028D3D1B2
:100730003846FEBD3EB5079C04B10124E4B20194E5
:10074000069C0094C569A84737BD2DE9F04385B0E4
:1007500005460C9E03A80090884614469946A86951
:100760000DF109030DF10A020DF10B0100F07CF906
:10077000B5F90E00B042A1BF9DF809107118B5F986
:100780000A00814202DA05B0BDE8F0830D9F2BE03C
:100790009DF80A0024E0B5F90C108945F3DA01460A
:1007A000A86902AA00F08BF950B9A86902AA2E2103
:1007B00000F085F920B9A86902AA202100F07FF98C
:1007C0000028E5D0019733469DF80B1001F0010198
:1007D00000914A460146284600F026F89DF8080098
:1007E000049981448844641A002CCCD004AB22467E
:1007F0004146284600F003F80028CCD1C3E738B5BD
:100800000446084611001A4601D1002032BD54F8B2
:10081000203F2BB1E47903EBC4035D68A84732BDE8
:1008200001211160007832BD2DE9F64F804683B07A
:10083000B8F90C000E469042A1BF71785118B8F972
:10084000080081420FDB4FF000090227CDF8089025
:10085000CB4601933078874280F2ED80019AB8F957
:100860000E105A449142C0F2E6809DF8380088BBD1
:100870000298002501E000207F1C31788F420DDABC
:10088000F25D00F118039A40B2FA82F10829C8BF5C
:10089000C0F108014D1908180828ECD00024029076
:1008A0003078874243DA0298F15D18308140C943BD
:1008B000B1FA81F00828C4BF0298C0F1080002997B
:1008C000041940180290082802BF002102917F1CE1
:1008D000E6D02CE0F45D24B1250904F00F047F1C60
:1008E00025E0F019BF1C4078C50000061FD505F4AF
:1008F0007E746CE0B8F908008142A1BFB8F90C30F1
:100900008B42B8F90A00824208DB9DF83C0028B10E
:10091000D8F80400D8F8143000F096F86D1ED146CF
:100920007078814504BF0BF1010B4FF00009002DD9
:100930004DD000F083F84ADB0499012D494409F1B8
:10094000010AD7DD70788245D4DA05EB09039842B5
:10095000B8F90A30B4BFA0EB090AAA469A4218DBDC
:100960009DF83C00A8B1049BB8F90800B8F90C1038
:10097000D8F804C04B449842B8BF1846049B4B4477
:1009800053445B1E9942C8BF1946D8F8143000F092
:1009900062F8A5EB0A05D144C2E7B8F90800814224
:1009A000A1BFB8F90C308B42B8F90A00824205DBCE
:1009B000D8F80400D8F8103000F046F8641EA946B4
:1009C0007078814504BF0BF1010B4FF00009002C3A
:1009D0003FF440AF00F032F8FFF63CAF0499012C31
:1009E000494409F10105D8DD70788542D5DA04EB78
:1009F00009039842B4BFA0EB09052546B8F90A00DF
:100A0000824215DB0498B8F90830B8F90C10D8F810
:100A100004C048449842B8BF1846049B4B44EB18A6
:100A20005B1E9942C8BF1946D8F8103000F013F881
:100A3000641BA944C4E705B0BDE8F08F019AB8F97A
:100A40000E005A449042704700F1040CDCF800009C
:100A5000DCF808C06047009313460A460146DCF8FC
:100A60000400DCF814C060477CB50446257806987D
:100A7000AE0605D500906068A4682568A84773BDD8
:100A80000D7061781170A2781A70E178017073BDF1
:100A90003EB504462078202801D0E0783EBD01A86C
:100AA00000900DF10503FFE76068A46825680DF16B
:100AB00006020DF10701A8479DF804003EBDF8B5F8
:100AC00003461878202804D158689B685C68A047C2
:100AD000F2BD45061CD5002000E0401CDD880C243A
:100AE0004443A8421C4406D2A668B142F5D3E76845
:100AF000BE19B142F1D2A84221D02569A0682B4489
:100B0000091A53F82100D8B1184441781170F2BD88
:100B1000000604D5D8689C681D795B7904E0D3F899
:100B2000C4001C1D20257E23A94228BF8B4206D36A
:100B3000491B34F81110084443781370F2BD0020AB
:100B4000F2BD01460878420601D5888870478006C4
:100B500003D5486889688A6810470020704770B5D7
:100B60000446A06910B94FF0FF3070BDFFF7E9FFF0
:100B70000146226A002004F1260300E0401C1D7893
:100B8000A8420BD232F83060A58CAE4202BF02EB15
:100B9000C00675888D42F1D1587070BD0020587024
:100BA000E1E78161DBE7000000220CF001BA000000
:100BB00010B504000020FDF72CFAF9F7D1F9A1696E
:100BC000401A40F6B931884214D3F9F72EFB0028B9
:100BD00010D0002060615FF0FF30F9F7A8FA00281C
:100BE00004D003210720FEF7A0F903E00321012030
:100BF000FEF79BF910BD000038B59CB0040040F230
:100C00005A200021F7F74CFDF9F727FB012804D102
:100C1000DFF8F40A0021F7F743FDF9F706FB062891
:100C200005D116220AA90620F9F79BFB25E0F9F762
:100C3000FCFA04281BD11E20FAF7F3F9162216A994
:100C4000F9F78FFB4FF40070FAF7DCF9002807D0B2
:100C500016ABDFF8B82A16210AA8FBF7D4FD0CE082
:100C600016ABAFA216210AA8FBF7CDFD05E0DFF811
:100C7000A02A16210AA8FBF7C6FDF9F771F9DFF8DB
:100C8000945A2968401A40F2F51188420CD3F9F7BA
:100C900067F92860DFF8800A0168012902D1002184
:100CA000016001E0012101605FF480000021FAF79A
:100CB00099FC002901D1002813D0DFF85C0A0068F4
:100CC000002805D197A2162102A8FBF79CFDD4E0CD
:100CD000DFF8483ADFF8482A162102A8FBF793FD0F
:100CE000CBE000204FF48051FAF77CFC002901D1C1
:100CF000002812D0DFF8200A0068002805D189A258
:100D0000162102A8FBF77FFDB7E0DFF8183A84A2AE
:100D1000162102A8FBF777FDAFE0FAF74DFC00289B
:100D200016D0DFF8F4090068002805D17DA216214D
:100D300002A8FBF768FDA0E0FAF73EFC0090DFF8A0
:100D4000E839DFF8E829162102A8FBF75CFD94E0FA
:100D5000FAF7E0F9002818D0DFF8BC09006800288D
:100D600005D170A2162102A8FBF74DFD85E0FAF728
:100D7000D1F9F9F774FB0090DFF8AC39DFF8B0294E
:100D8000162102A8FBF73FFD77E04FF480400021D9
:100D9000FAF728FC002901D1002811D0DFF87809E2
:100DA0000068002805D15FA2162102A8FBF72BFDE1
:100DB00063E01622DFF87C1902A8FBF7C9FB5CE0B0
:100DC00008200021FAF70EFC002901D1002811D0DB
:100DD000DFF844090068002805D152A2162102A8B4
:100DE000FBF711FD49E01622DFF84C1902A8FBF7CA
:100DF000AFFB42E05FF400300021FAF7F3FB00297B
:100E000001D1002811D0DFF810090068002805D1B1
:100E100044A2162102A8FBF7F6FC2EE01622DFF80A
:100E20001C1902A8FBF794FB27E06C20FAF7F9F8ED
:100E300000281ED06C20FAF7F4F8032808D1DFF858
:100E40000039DFF80029162102A8FBF7DCFC14E0CA
:100E50006020FAF7E6F80500F9F7D7FF0195009052
:100E6000DFF8DC38DFF8E028162102A8FBF7CBFC1E
:100E700003E0162102A8FAF727FAF9F7C0FF812844
:100E800006DBDFF8C828162110A8FBF7BCFC03E03E
:100E9000162110A8F9F75DFF0020FAF711FA0500F6
:100EA0000120FAF70DFA03000095DFF8A4280621C7
:100EB00008A8FBF7A8FC0025F9F7E8F900280BD1F2
:100EC000DFF890080021FAF78DFB002901D10028F6
:100ED00002D055F001050EE0F9F7D8F901280AD142
:100EE000DFF870080021FAF77DFB002901D1002806
:100EF00001D055F001055FF080500021FAF772FB38
:100F0000002901D1002801D055F0020560680128B0
:100F100002D0E068012807D155F0040509E000BFC0
:100F20002573000000000000A068012801D155F0E1
:100F300008050120FDF76DF80AA90C20FDF79EF8C1
:100F400002A90A20FDF79AF810A90920FDF796F8E2
:100F500008A90B20FDF792F82800FDF75EF856204F
:100F6000FAF75FF8800712D4FAF7ACF801280ED12F
:100F70004020F9F793FE002809D02020F9F783FEDE
:100F80004020F9F780FE00200121F7F789FB606817
:100F9000002840F045814FF40050FAF733F800285C
:100FA00002D00120E06001E00020E0600120FEF7B7
:100FB0009AF9002848D00820FEF795F9002843D078
:100FC0000420FEF790F900283ED10220FEF78BF9AD
:100FD000002839D1F8F7C4FFE061F8F7C1FFA16933
:100FE000401A41F289318842C0F02881F8F7B8FFF1
:100FF000A0610120DFF860170860E068012811D1C6
:101000000020E0604FF40050F9F7FCFF002800F0EA
:1010100015814FF40050F9F7FEFF00200821F7F783
:101020003FFB0BE10120E0604FF40050F9F7EAFFCD
:10103000002840F003814FF40050F9F7E7FF00204B
:101040000821F7F72DFBF9E00420FEF74CF9002802
:1010500025D00220FEF747F9002820D00120FEF716
:1010600042F900281BD10820FEF73DF9002816D1CF
:10107000F8F776FFA061F8F773FFE169401A40F6D0
:10108000B9318842C0F0DA80F8F76AFFE0610120E8
:10109000F9F7E8FE00208021F7F702FBCEE0F8F731
:1010A0005FFFA061F8F75CFFE061E068002840F0B6
:1010B000A8800420FEF721F900282FD0F9F7CDF8F9
:1010C000002808D05FF480000021FAF78BFA00298D
:1010D00001D1002804D001210E20FDF726FF90E069
:1010E00000204FF48051FAF77DFA002940F0898002
:1010F000002840F08680A068012806D1032108203E
:10110000FDF713FF002020617BE001210820FDF79F
:101110000CFF01210220FDF708FF72E00820FEF716
:10112000ECF800280ED0DFF830060068002809D15E
:101130000220F9F7B3FD002804D101210620FDF7B4
:10114000F4FE5EE00120FEF7D8F800282FD0DFF88B
:101150000806006800282AD10220F9F79FFD002820
:101160004FD1A068012808D0F9F790F8002804D0E2
:101170000120F9F793FD002810D00120F9F78EFD2A
:10118000002803D00120F9F77EFD02E00120F9F7E5
:1011900070FD00200121F7F783FA32E003210420DB
:1011A000FDF7C3FE01210220FDF7BFFE29E002206A
:1011B000FEF7A3F8002824D0A068012808D0F9F78A
:1011C00065F8002804D00220F9F768FD002810D047
:1011D0000220F9F763FD002803D00220F9F753FD40
:1011E00002E00220F9F745FD00200121F7F758FA47
:1011F00007E003210520FDF798FE01210220FDF7FD
:1012000094FE0820FEF76FF8002817D10120FEF7A2
:101210006AF8002812D10020DFF83C1508600DE0C4
:101220004FF40050F9F7EEFE002807D14FF40050BC
:10123000F9F7ECFE00200821F7F732FA1DB030BDB7
:1012400010B586B042200021F7F72AFA1622DFF8FF
:101250000C156846FBF77CF969460020FCF70EFF89
:1012600016216846F9F775FD0220FCF7D2FE6946A3
:101270000920FCF703FF5620F9F7D3FE800712D4AC
:10128000F9F720FF01280ED14020F9F707FD0028CB
:1012900009D02020F9F7F7FC4020F9F7F4FC0020F2
:1012A0000121F7F7FDF90120FEF727F800284BD0C0
:1012B0000120F9F7F3FC002840F02B81F8F7E6FF56
:1012C000012810D12020F9F7E9FC002803D02020C4
:1012D000F9F7D9FC02E02020F9F7CBFC002001212E
:1012E000F7F7DEF926E04020F9F7D8FC002815D101
:1012F000DFF86C04006801281CD02020F9F7CEFC30
:10130000002803D02020F9F7BEFC02E02020F9F7E6
:10131000B0FC00200121F7F7C3F90BE0DFF840042F
:101320000068012806D04020F9F7ADFC002001211B
:10133000F7F7B6F9F8F714FEDFF828140860002074
:10134000DFF81C140860E4E00120FDF7CCFF002862
:101350004ED05620F9F765FE80073FD5F9F7B2FE6B
:1013600001283BD15720F9F75CFE012836D1DFF880
:10137000F0432068002840F0CC80F8F7F1FDDFF85A
:10138000E4130968401A40F6B9318842C0F0C180C0
:10139000012020604020F9F781FC002813D1402073
:1013A000F9F767FC0820F9F779FC00280ED0102027
:1013B000F9F774FC002809D00820F9F764FC102024
:1013C000F9F761FC02E04020F9F75DFC2020F9F715
:1013D0005AFC00200121F7F763F99AE00020DFF8BA
:1013E00080130860F8F7BCFDDFF87813086090E020
:1013F0000220FDF782FF002864D00120F9F74EFC9F
:10140000002840F086802020F9F748FC002840F0B2
:101410008080F8F73BFF01280FD10820F9F73EFC48
:10142000002803D10820F9F724FC02E00820F9F78E
:101430002AFC1020F9F727FC3FE00820F9F72EFCE2
:1014400000280BD11020F9F729FC002806D108202C
:10145000F9F70FFC1020F9F716FC2EE00820F9F739
:101460001DFC00280BD01020F9F718FC002806D02E
:101470001020F9F708FC0820F9F705FC1DE008200A
:10148000F9F70CFC002806D01020F9F7F2FB082031
:10149000F9F7F9FB11E04020F9F700FC002806D12C
:1014A0001020F9F7E6FB0820F9F7E3FB05E0102030
:1014B000F9F7E9FB0820F9F7E6FB00200121F7F72F
:1014C000EFF826E00420FDF718FF002810D00420D4
:1014D000F9F7E4FB002803D00420F9F7D4FB02E07D
:1014E0000420F9F7C6FB00200121F7F7D9F810E036
:1014F0000820FDF702FF002807D003210120FDF797
:1015000014FD00209649086003E0F8F729FD95498D
:10151000086006B010BD10B586B078200021F7F73E
:10152000BFF8162269460620F8F71BFF694600201F
:10153000FCF7A4FD0420FCF76CFD0120FCF7C1FDC5
:10154000162289496846FBF703F869460120FCF733
:1015500095FD6CA421000220FCF790FD21000320E2
:10156000FCF78CFD21000420FCF788FD21000520FC
:10157000FCF784FD21000620FCF780FD21000720F8
:10158000FCF77CFD21000820FCF778FD0020FCF72B
:1015900044FD0820FDF7B1FE002801D0FDF71DFD38
:1015A00006B010BD18B587B002200021F7F778F813
:1015B00016226E4901A8FAF7CBFF01A90020FCF71B
:1015C0005DFDF8F7B8FD0090574B694A162101A858
:1015D000FBF719F90420FCF71CFD0020FCF771FD56
:1015E00001A90120FCF74AFD0020FCF716FD45A4E7
:1015F00021000220FCF742FD21000320FCF73EFD04
:1016000021000420FCF73AFD21000520FCF736FDFF
:1016100021000620FCF732FD21000720FCF72EFDFB
:1016200021000820FCF72AFD0420FDF75CFE0028BD
:1016300010D00220FDF757FE00280BD00120FDF747
:1016400052FE002806D10820FDF74DFE002801D1EA
:10165000F8F78FFC08B010BD10B58CB0F8F716FE87
:10166000002805D1434A16216846FBF7CCF804E070
:10167000414A16216846FBF7C6F869460020FCF788
:10168000FDFC0420FCF7C5FC0120FCF71AFD162226
:10169000224906A8FAF75CFFF8F7DFFD012804D11C
:1016A000364A16216846FBF7AEF869460120FCF77A
:1016B000E5FC06A90520FCF7E1FC12A421000220AC
:1016C000FCF7DCFC21000320FCF7D8FC21000420FF
:1016D000FCF7D4FC21000620FCF7D0FC21000720F9
:1016E000FCF7CCFC21000820FCF7C8FC0020FCF72C
:1016F00094FC0820FDF701FE002801D0FDF76DFCE9
:101700000CB010BD0000000080001000C8F90100FE
:10171000D0F90100701100206C11002040F7030087
:10172000A8F5010028F2010020E50300B4F501004E
:10173000C0F5010020E30300A0E1030060F0030016
:10174000D0F40100CCF50100D8F50100D8F9010072
:10175000E4F50100299E3F6C7411002020EC030089
:10176000781100207C11002080F0030000D00300DD
:10177000E0F90100E8F90100F0F90100F8F90100D1
:10178000F0B5BDB0040058200021F6F789FF1622FD
:10179000DFF880136846FAF7DBFE69460020FCF7A5
:1017A0006DFC0320FCF735FC0420FCF78AFCDFF815
:1017B0006833DFF86823162106A8FBF724F8DFF862
:1017C0006033DFF8602316210DF12E00FBF71BF8C4
:1017D000DFF85433DFF85423162111A8FBF713F870
:1017E000DFF84C33DFF84C2316210DF15A00FBF7DC
:1017F0000AF85720F9F715FC01282CD1DFF8383307
:10180000DFF8382316211CA8FAF7FDFFDFF8303384
:10181000DFF8302316210DF18600FAF7F4FFCA4BEA
:10182000CA4A162127A8FAF7EEFFC94BC94A162162
:101830000DF1B200FAF7E7FFC74BC84A162132A8EC
:10184000FAF7E1FFC64BC74A16210DF1DE00FAF7A1
:10185000DAFF0A2526E0BA4BB84A16211CA8FAF787
:10186000D2FFB94BB74A16210DF18600FAF7CBFF2C
:10187000B74BB64A162127A8FAF7C5FFB64BB54AAB
:1018800016210DF1B200FAF7BEFFB54BB34A16218F
:1018900032A8FAF7B8FF9EA216210DF1DE00FAF782
:1018A000B2FF09252800FDF7D7FA0020FDF703FB5A
:1018B000401CFCF7B2FB0220FDF7FDFA06001627DC
:1018C00006A807FB06F101440120FCF7D7FB06A898
:1018D00007FB06F1084410F116010220FCF7CEFBCD
:1018E00006A807FB06F1084410F12C010320FCF7C1
:1018F000C5FB06A87E43304410F142010420FCF7EA
:10190000BDFB0820FDF7F9FC002800F092800120C3
:10191000FDF7D1FA002809D101214020FDF705FB90
:101920000BF02AFC2063206BE0638FE0012813D1C9
:10193000A068012802D02069002808D101212620B2
:10194000FDF7F3FA01210220FDF7EFFA7EE0012115
:101950002620FDF7EAFA79E0022818D1F8F796FC7C
:10196000012804D101210A20FDF7DFFA6EE04FF4CF
:101970000070F9F747FB002804D001210A20FDF789
:10198000D4FA63E001210920FDF7CFFA5EE00328D5
:1019900004D101210D20FDF7C8FA57E004280BD12E
:1019A0000A2D04D001211620FDF7BFFA4EE00121D7
:1019B0008720FDF7BAFA49E005280BD10A2D04D09B
:1019C00001212220FDF7B1FA40E001211620FDF7A8
:1019D000ACFA3BE006280BD10A2D04D001213720B8
:1019E000FDF7A3FA32E001212220FDF79EFA2DE057
:1019F00007280BD10A2D04D001219220FDF795FA7A
:101A000024E001213720FDF790FA1FE008280BD1D0
:101A10000A2D04D001219320FDF787FA16E0012159
:101A20009220FDF782FA11E001219320FDF77DFA63
:101A30000CE00120FDF761FC002804D00321012007
:101A4000FDF773FA02E02800FDF7E1FA3DB0F0BDC2
:101A500018B591B088200021F6F722FE0220FDF78C
:101A6000FBF9162236496846FAF772FD69460020EE
:101A7000FCF704FB0320FCF7CCFA0420FCF721FB65
:101A8000394B264A162106A8FAF7BDFE374B254AE0
:101A900016210DF12E00FAF7B6FE0020FDF70BFA25
:101AA000401CFCF7BAFA06A90120FCF7E7FA0DF191
:101AB0002E010220FCF7E2FA15A421000320FCF716
:101AC000DDFA21000420FCF7D9FA0820FDF715FC07
:101AD000002810D00120FDF7EEF9002804D10121E3
:101AE0001B20FDF722FA11E001280FD10121172058
:101AF000FDF71BFA0AE00120FDF7FFFB002802D0EA
:101B0000FDF76BFA02E00220FDF781FA12B010BD7A
:101B100000000000C0D9030020D2030078F90100C2
:101B200040D2030080F9010060D2030088F901006F
:101B300080D2030090F9010020F1030098F9010020
:101B4000E0F20300A0F90100C0D20300A8F90100EF
:101B5000E0D20300B0F9010000D30300B8F901009E
:101B600020D30300C0F90100A0D20300C4F4010097
:101B700030B591B0040002200021F6F791FD02205B
:101B8000FDF76AF91622DFF8581C6846FAF7E0FC00
:101B900069460020FCF772FA0320FCF73AFA0420A9
:101BA000FCF78FFADFF83C3CDFF83C2C162106A846
:101BB000FAF729FEDFF8343CDFF8342C16210DF15A
:101BC0002E00FAF720FE06A90120FCF757FA0DF1C6
:101BD0002E010220FCF752FA7BA529000320FCF716
:101BE0004DFA29000420FCF749FA0020FDF763F9BB
:101BF000401CFCF712FA0820FDF77FFB002815D0E7
:101C00000120FDF758F900280BD101211020FDF724
:101C10008CF92069002814D101210220FDF785F9F3
:101C20000FE001211120FDF780F90AE00120FDF706
:101C300064FB002802D0FDF7D0F902E00220FDF796
:101C4000E6F911B030BD30B587B0050002200021A3
:101C5000F6F726FD1622DFF89C1B01A8FAF778FCA0
:101C600001A90020FCF70AFA0420FCF7D2F90420AD
:101C7000FCF727FAB3A421000120FCF7FFF92100AB
:101C80000220FCF7FBF921000320FCF7F7F9210003
:101C90000420FCF7F3F94CA421000520FCF7EEF931
:101CA00021000620FCF7EAF921000720FCF7E6F9FD
:101CB00021000820FCF7E2F90020FCF7AEF9E86A01
:101CC000284490F820008DF8000000208DF80100D5
:101CD000E86A012804D169460120FCF7CFF916E033
:101CE000E86A022804D169460220FCF7C7F90EE031
:101CF000E86A032804D169460320FCF7BFF906E02F
:101D0000E86A042803D169460420FCF7B7F9EC6AB5
:101D10000220FDF7EDFA00281BD0002C03D1E86A61
:101D2000401CE8624DE005EB040090F820003928E3
:101D300009DA05EB040090F82000401C05EB0401D3
:101D400081F820003DE0302005EB040181F82000FF
:101D500037E00420FDF7CCFA00281BD0002C03D17B
:101D6000E86A401CE8622CE005EB040090F82000D3
:101D7000312809DB05EB040090F82000401E05EB3C
:101D8000040181F820001CE0392005EB040181F8F2
:101D9000200016E00820FDF7B0FA00280AD0042C35
:101DA00004D102211220FDF7C0F80AE0E86A401CC5
:101DB000E86206E00120FDF7A0FA002801D0FDF757
:101DC0000CF907B030BD00000000000030B587B04E
:101DD000050002200021F6F763FC1622DFF81C1A2A
:101DE00001A8FAF7B5FB01A90020FCF747F9042088
:101DF000FCF70FF90420FCF764F952A4210001203C
:101E0000FCF73CF921000220FCF738F921000320FF
:101E1000FCF734F921000420FCF730F9BEA42100BE
:101E20000520FCF72BF921000620FCF727F92100FB
:101E30000720FCF723F921000820FCF71FF90020F8
:101E4000FCF7EBF8EC6A05EB040090F820008DF845
:101E5000000000208DF80100012C04D1694601200A
:101E6000FCF70CF913E0022C04D169460220FCF7C0
:101E700005F90CE0032C04D169460320FCF7FEF8B9
:101E800005E0042C03D169460420FCF7F7F8022092
:101E9000FDF72EFA00281BD0002C03D1E86A401C65
:101EA000E8624DE005EB040090F82000392809DADB
:101EB00005EB040090F82000401C05EB040181F8BC
:101EC00020003DE0302005EB040181F8200037E0E0
:101ED0000420FDF70DFA00281BD0002C03D1E86A7E
:101EE000401CE8622CE005EB040090F8200031284B
:101EF00009DB05EB040090F82000401E05EB04010F
:101F000081F820001CE0392005EB040181F8200055
:101F100016E00820FDF7F1F900280AD0042C04D1BE
:101F200002211320FDF701F80AE0E86A401CE8628C
:101F300006E00120FDF7E1F9002801D0FDF74DF89A
:101F400007B030BD2A00000030B587B00500022080
:101F50000021F6F7A5FB1622DFF8A41801A8FAF76E
:101F6000F7FA01A90020FCF789F80420FCF751F8E2
:101F70000420FCF7A6F869A421000120FCF77EF8F4
:101F800021000220FCF77AF821000320FCF776F804
:101F900021000420FCF772F85FA421000520FCF763
:101FA0006DF821000620FCF769F821000720FCF7F6
:101FB00065F821000820FCF761F80020FCF72DF8F7
:101FC000EC6A05EB040090F825008DF80000002075
:101FD0008DF80100012C04D169460120FCF74EF870
:101FE00013E0022C04D169460220FCF747F80CE00C
:101FF000032C04D169460320FCF740F805E0042CCB
:1020000003D169460420FCF739F80220FDF770F986
:1020100000281BD0002C03D1E86A401CE86279E05C
:1020200005EB040090F82500392809DA05EB0400D7
:1020300090F82500401C05EB040181F8250069E0BB
:10204000302005EB040181F8250063E00420FDF752
:102050004FF900281BD0002C03D1E86A401CE8622D
:1020600058E005EB040090F82500312809DB05EB6A
:10207000040090F82500401E05EB040181F82500BE
:1020800048E0392005EB040181F8250042E00820F2
:10209000FDF733F9002836D0042C30D195F826000E
:1020A00095F82110884225D195F8270095F822103F
:1020B00088421FD195F8280095F82310884219D13D
:1020C00095F8290095F82410884213D10221142094
:1020D000FCF72BFF95F8293095F8282095F8271064
:1020E00095F82600F8F74AFD00204FF48071F6F7C6
:1020F000D7FA0FE002211220FCF717FF0AE0E86A86
:10210000401CE86206E00120FDF7F7F8002801D046
:10211000FCF763FF07B030BD000000002A0000009C
:1021200030B587B0050002200021F6F7B9FA162273
:10213000DFF8D01601A8FAF70BFA01A90020FBF787
:102140009DFF0420FBF765FF0420FBF7BAFFA3A463
:1021500021000120FBF792FF21000220FBF78EFFF8
:1021600021000320FBF78AFF21000420FBF786FFF4
:102170009BA421000520FBF781FF21000620FBF72F
:102180007DFF21000720FBF779FF21000820FBF7E6
:1021900075FF0020FBF741FFEC6A05EB040090F8A7
:1021A00025008DF8000000208DF80100012C04D1DD
:1021B00069460120FBF762FF13E0022C04D1694657
:1021C0000220FBF75BFF0CE0032C04D169460320DF
:1021D000FBF754FF05E0042C03D169460420FBF70C
:1021E0004DFF0220FDF784F800281BD0002C03D1FE
:1021F000E86A401CE86279E005EB040090F82500ED
:10220000392809DA05EB040090F82500401C05EB9D
:10221000040181F8250069E0302005EB040181F814
:10222000250063E00420FDF763F800281BD0002C94
:1022300003D1E86A401CE86258E005EB040090F81E
:102240002500312809DB05EB040090F82500401E2D
:1022500005EB040181F8250048E0392005EB040175
:1022600081F8250042E00820FDF747F8002836D025
:10227000042C30D195F8260095F82110884225D1FC
:1022800095F8270095F8221088421FD195F828006C
:1022900095F82310884219D195F8290095F8241053
:1022A000884213D102211520FCF73FFE95F8293012
:1022B00095F8282095F8271095F82600F8F781FC66
:1022C00000204FF40071F6F7EBF90FE00221132024
:1022D000FCF72BFE0AE0E86A401CE86206E00120F9
:1022E000FDF70BF8002801D0FCF777FE07B030BDF2
:1022F00010B586B002200021F6F7D2F90420FBF7D2
:1023000088FE1622DFF8EC146846FAF721F96946D0
:102310000020FBF7B3FE0020F8F76DFC040000205E
:10232000F8F762FCE4B2844224D10120F8F763FCA0
:1023300004000120F8F758FCE4B284421AD10220CC
:10234000F8F759FC04000220F8F74EFCE4B284428E
:1023500010D10320F8F74FFC04000320F8F744FCE9
:10236000E4B2844206D11622DFF89C146846FAF7DC
:10237000EFF805E01622DFF894146846FAF7E8F85B
:1023800069460120FBF77AFE15A421000220FBF725
:1023900075FE21000320FBF771FE21000420FBF7EE
:1023A0006DFE21000520FBF769FE21000620FBF7EA
:1023B00065FE21000720FBF761FE21000820FBF7E6
:1023C0005DFE0120FBF77DFE0820FCF796FF00284C
:1023D00001D0FCF702FE06B010BD00002A0000008C
:1023E0000000000010B586B002200021F6F758F971
:1023F0000420FBF70EFE1622DFF800146846FAF7F9
:10240000A7F869460020FBF739FE0020F8F7F3FB38
:1024100004000020F8F7E8FBE4B2844224D1012054
:10242000F8F7E9FB04000120F8F7DEFBE4B2844290
:102430001AD10220F8F7DFFB04000220F8F7D4FBE2
:10244000E4B2844210D10320F8F7D5FB0400032046
:10245000F8F7CAFBE4B2844206D11622DFF8A813CB
:102460006846FAF775F805E01622DFF8A01368460B
:10247000FAF76EF869460120FBF700FEB0A42100D0
:102480000220FBF7FBFD21000320FBF7F7FD2100F5
:102490000420FBF7F3FD21000520FBF7EFFD2100F1
:1024A0000620FBF7EBFD21000720FBF7E7FD2100ED
:1024B0000820FBF7E3FD0120FBF703FE0820FCF7F3
:1024C0001CFF002801D0FCF788FD06B010BD78B5D0
:1024D00087B00600FCF794FD050002200021F6F706
:1024E000DFF80420FBF795FD042D03D0052D01D066
:1024F000082D05D11622C64901A8FAF729F804E0EB
:102500001622B84901A8FAF723F801A90020FBF721
:10251000B5FD0420FBF7D5FDB0A421000120FBF799
:10252000ADFD21000220FBF7A9FD21000320FBF7F0
:10253000A5FD21000420FBF7A1FD81A421000520B9
:10254000FBF79CFD21000620FBF798FD21000720EA
:10255000FBF794FD21000820FBF790FD0020FBF71E
:102560005CFDF46A06EB040090F820008DF804008E
:1025700000208DF80500012C04D101A90120FBF7F2
:102580007DFD13E0022C04D101A90220FBF776FDAA
:102590000CE0032C04D101A90320FBF76FFD05E03B
:1025A000042C03D101A90420FBF768FD0220FCF7ED
:1025B0009FFE00281ED0002C07D1F06A401CF0625C
:1025C000F16A0020FCF793FC14E006EB040090F89D
:1025D0002000392809DA06EB040090F82000401C9E
:1025E00006EB040181F8200004E0302006EB040132
:1025F00081F820000420FCF77BFE00281ED0002C70
:1026000007D1F06A401CF062F16A0020FCF76FFC11
:1026100014E006EB040090F82000312809DB06EBFB
:10262000040090F82000401E06EB040181F8200011
:1026300004E0392006EB040181F820000820FCF7B3
:102640005CFE002871D0042C67D196F8240000901D
:1026500096F8233096F8222096F821100120F8F7FA
:1026600031FA040096F82400009096F8233096F88A
:10267000222096F821100020F8F724FA082D14D112
:10268000002C04D1012802D10121316101E0002197
:102690003161012C01D0012802D1FCF79EFC4DE0F4
:1026A00002210320FCF741FC48E0042D14D1012C49
:1026B00001D001280BD10120F8F7DBFA002001211D
:1026C000F5F7EEFF03210120FCF72FFC36E0022195
:1026D0000320FCF72AFC31E0052D14D1012C01D098
:1026E00001280BD10220F8F7C4FA00200121F5F7E8
:1026F000D7FF03210120FCF718FC1FE00221032073
:10270000FCF713FC1AE0012802D1FCF766FC15E087
:1027100002210320FCF709FC10E0F06A401CF06283
:10272000F16A0020FCF7E3FB08E00120FCF7E5FD7F
:10273000002803D0FCF751FCFCF74FFC08B070BD3B
:102740000000000010B586B002200021F5F7A8FFB8
:10275000162223496846F9F7FBFE69460020FBF77D
:102760008DFC0420FBF755FC0120FBF7AAFC162288
:1027700026496846F9F7ECFE69460120FBF77EFC26
:102780001DA421000220FBF779FC21000320FBF7A8
:1027900075FC21000420FBF771FC21000520FBF7EC
:1027A0006DFC21000620FBF769FC21000720FBF7E8
:1027B00065FC21000820FBF761FC0120FCF79DFD72
:1027C000002804D10820FCF798FD002803D0FCF76E
:1027D00004FCFCF702FC06B010BD00002A0000005B
:1027E00000D3030040EE030088FB010060EE03000D
:1027F00090FB010080EE030000000000C0EE03002B
:10280000A0EE0300E0EE030000EF030040EC030045
:1028100060EC030030B591B0040040200021F5F7D2
:102820003FFFDFF8CC3690A216210BA8F9F7EBFF9B
:102830000BA90020FBF722FC0320FBF7EAFB042096
:10284000FBF73FFC0020FCF736FB401CFBF7E5FBE9
:10285000DFF8A036DFF8A02616216846F9F7D3FF87
:10286000DFF89836DFF8982616210DF11600F9F7F3
:10287000CAFF7EA52A0016210BA8F9F7C4FF6946F6
:102880000120FBF7FBFB0DF116010220FBF7F6FB25
:102890000BA90320FBF7F2FB29000420FBF7EEFB5A
:1028A0000120FCF72AFD002802D0FCF796FB41E04E
:1028B0000820FCF722FD002839D00120FCF7FBFAA4
:1028C000002810D101212420FCF72FFB0220F8F76B
:1028D000F7FC20630420F8F7F3FC60630520F8F7A9
:1028E000EFFCA0631EE001280CD101212320FCF79E
:1028F0001CFB0120F8F7E4FC20630020F8F7E0FC63
:1029000060630FE002280DD101212520FCF70DFBAB
:102910000120F8F777FB002802D00120206301E0B6
:10292000002020630020DFF8DC15086002E00220B0
:10293000FCF76DFB11B030BD38B588B0040016222D
:10294000DFF8B81502A8F9F703FE02A90020FBF78B
:1029500095FB0420FBF75DFB0420FBF7B2FBDFF8DF
:10296000A855236B2A00032102A8F9F74CFF02A9FE
:102970000120FBF783FB3EA10220FBF77FFB636B8B
:102980002A00032102A8F9F73EFF02A90320FBF762
:1029900075FB36A529000420FBF770FB29000520F4
:1029A000FBF76CFB29000620FBF768FB29000720DA
:1029B000FBF764FB29000720FBF760FBDFF84455B9
:1029C0002868FBF72AFB0120FCF797FC002802D0BF
:1029D000FCF703FB45E00820FCF78FFC002815D02E
:1029E000286803280ED1216B0120F8F765FC616B84
:1029F0000020F8F761FC00202021F5F751FEFCF7DC
:102A0000ECFA2EE02868401C28602AE0286800289C
:102A100003D12868401C286023E0286801280BD1D6
:102A20000120019001200090012300221721206B3A
:102A3000FCF760FB206314E02868022803D12868B3
:102A4000401C28600DE0286803280AD1012001906D
:102A500001200090012300223B21606BFCF74AFB20
:102A6000606309B030BD0000257300000000000065
:102A70003A00000078B593B004001622DFF8741411
:102A800002A8F9F765FD02A90020FBF7F7FA042078
:102A9000FBF7BFFA0420FBF714FBDFF86854286843
:102AA00000281BD1A06B0190606B0090236BDFF8B6
:102AB0005C24092102A8F9F7A6FE02A90120FBF770
:102AC000DDFAC6A631000220FBF7D8FA3100032058
:102AD000FBF7D4FA31000420FBF7D0FA286801286C
:102AE00021D1236BDFF82024032102A8F9F78BFE04
:102AF00002A90120FBF7C2FAA06B0090636BDFF81C
:102B00001024072102A8F9F77EFE02A90220FBF794
:102B1000B5FAB2A631000320FBF7B0FA3100042069
:102B2000FBF7ACFA48E02868022825D1236BDFF8D0
:102B3000E423042102A8F9F766FE02A90120FBF7AD
:102B40009DFA636BDFF8C023032102A8F9F75BFE4F
:102B500002A90220FBF792FAA36BDFF8BC23042141
:102B600002A8F9F750FE02A90320FBF787FA9BA100
:102B70000420FBF783FA1FE0606B0090236BDFF803
:102B80009C23062102A8F9F73EFE02A90120FBF7CB
:102B900075FA93A10220FBF771FAA36BDFF86823A3
:102BA000032102A8F9F72FFE02A90320FBF766FA1A
:102BB0008AA10420FBF762FA01200A9032200990D2
:102BC000206B0B90606B401E0C90A06B64300D90DE
:102BD00008A8F7F7E5FE08A9F7F78DFE0E9801287B
:102BE00006D10422DFF8381302A8F9F7B1FC32E06D
:102BF0000E98022806D10422DFF8281302A8F9F75C
:102C0000A7FC28E00E98032805D10422C64902A893
:102C1000F9F79EFC1FE00E98042805D10422C34951
:102C200002A8F9F795FC16E00E98052805D10422B4
:102C3000BF4902A8F9F78CFC0DE00E98062805D1D3
:102C40000422BC4902A8F9F783FC04E00422BA4933
:102C500002A8F9F77DFC00208DF80B00206B0028FE
:102C60000AD0606B002807D0A06B002804D002A90E
:102C70000520FBF703FA03E058A10520FBF7FEF956
:102C800056A631000620FBF7F9F931000720FBF7C3
:102C9000F5F931000820FBF7F1F92868FBF7BDF9D9
:102CA0000120FCF72AFB002802D0FCF796F993E0FC
:102CB0000820FCF722FB00285BD02868032830D1CD
:102CC000206B1D2808D1606B022805D194F83800CC
:102CD00010F0030F40F080800220F8F7F1FA216B2A
:102CE00081420BD10420F8F7EBFA616B814205D1E8
:102CF0000520F8F7E5FAA16B81420FD0216B022085
:102D0000F8F7DAFA616B0420F8F7D6FAA16B052020
:102D1000F8F7D2FA00202021F5F7C2FCFCF75DF9A4
:102D20005AE02868022820D1606B022806D1206B67
:102D30001E2851D22868401C28604DE0606B042892
:102D400008D0606B062805D0606B092802D0606B44
:102D50000B2806D1206B1F283ED22868401C286013
:102D60003AE02868401C286036E02868401C28604B
:102D700032E02868002803D12868401C28602BE036
:102D8000286801280BD10120019001200090012327
:102D900001221F21206BFCF7ADF920631CE028689D
:102DA00002280BD101200190012000900123012273
:102DB0000C21606BFCF79EF960630DE02868032826
:102DC0000AD10120019001200090012300226321FB
:102DD000A06BFCF78FF9A06314B070BD0000000079
:102DE0002F00000038B588B0040040200021F5F71E
:102DF00057FC524B3CA2162102A8F9F704FD02A988
:102E00000020FBF73BF90420FBF703F90420FBF754
:102E100058F9206B002805D11622494902A8F9F774
:102E200097FB04E01622474902A8F9F791FB02A993
:102E30000120FBF723F92DA529000220FBF71EF93D
:102E400029000320FBF71AF929000420FBF716F9E3
:102E500029000520FBF712F929000620FBF70EF9DF
:102E600029000720FBF70AF929000820FBF706F9DB
:102E70000820FCF742FA002820D0206B002804D05C
:102E80000120F8F7BFF8002807D0206B002812D1E6
:102E90000120F8F7B7F800280DD0206B002803D1E7
:102EA0000120F8F7B8F802E00120F8F7AFF80020A9
:102EB0000821F5F7F5FBFCF790F812E00120FCF78C
:102EC0001CFA002802D0FCF788F80AE000200190E4
:102ED00000200090012300220121206BFCF70AF959
:102EE000206309B030BD0000257300000000000021
:102EF000C0D2030080ED030030F90100A0ED030013
:102F000038F901006811002040F90100FCF30100CC
:102F100084F5010048F9010050F9010090F5010025
:102F200000EB030020EB030040EB030060EB030029
:102F300080EB0300A0EB0300C0EB030060ED030097
:102F400080E60300E0D9030030B591B04FF4006093
:102F50000021F5F7A5FBDFF81C4516222100684685
:102F6000F9F7F6FA2300DFF81025162106A8F9F77D
:102F70004AFCF7F78BF9012808D12300DFF8FC247D
:102F800016210DF12E00F9F73EFC07E02300DFF8D3
:102F9000F02416210DF12E00F9F735FC0220FBF785
:102FA0005BFF0320FBF735F80420FBF78AF869463E
:102FB0000020FBF763F80020FBF77DFF401CFBF7C8
:102FC0002CF80220FBF777FF040006A90120FBF78D
:102FD00055F80DF12E010220FBF750F8B0A529009D
:102FE0000320FBF74BF829000420FBF747F80120EA
:102FF000FCF783F9002802D0FBF7EFFF16E008206A
:10300000FCF77BF900280ED00120FBF754FF0128C4
:1030100004D101210B20FBF788FF07E001210920E3
:10302000FBF783FF02E02000FBF7F1FF11B030BD9A
:1030300070B5B2B01622DFF83C146846F9F788FA8A
:1030400069460020FBF71AF80320FAF7E2FF042094
:10305000FBF737F800200AE0002206AB162404FB39
:1030600000F423445A54491C1629F5D3401C08285F
:1030700001D20021F8E7012400265FF0FF30F8F7C5
:1030800093FA05000EE025420BD0F7F7FFF8020097
:10309000210006A8162303FB06F31844F8F7AEFA3E
:1030A000761C6400082E01D2002CECD13000FBF716
:1030B000D3FE002D03D10020FAF7AFFF05E000207A
:1030C000FBF7F9FE401CFAF7A8FF0220FBF7F3FE1E
:1030D0000500162406A804FB05F101440120FAF7B7
:1030E000CDFF06A804FB05F1084410F116010220EB
:1030F000FAF7C4FF06A804FB05F1084410F12C01FF
:103100000320FAF7BBFF06A86543284410F14201EB
:103110000420FAF7B3FF0120FCF7EFF8002802D0F3
:10312000FBF75BFF27E00820FCF7E7F800281FD03B
:103130000120FBF7C0FE0500F7F7A8F802001021F8
:103140006846F8F75BFA1222694606A865432844E8
:10315000F9F760FB002808D1F8F74DFA002804D0F1
:1031600002210C20FBF7E1FE05E0FBF736FF02E051
:103170003000FBF74CFF32B070BD70B5B2B04FF409
:1031800000600021F5F78CFAF7F780F8012806D1E6
:10319000B84BBC4A16216846F9F735FB05E0B54B3C
:1031A000B94A16216846F9F72EFB69460020FAF75E
:1031B00065FF0320FAF72DFF0420FAF782FF0020B5
:1031C0000AE0002206AB162404FB00F423445A5400
:1031D000491C1629F5D3401C082801D20021F8E724
:1031E000012400265FF0FF30F8F7E2F905000BE05C
:1031F000254208D0210006A8162202FB06F2104440
:10320000F8F724FA761C6400082E01D2002CEFD1C6
:103210003000FBF721FE002D03D10020FAF7FDFE60
:1032200005E00020FBF747FE401CFAF7F6FE0220FF
:10323000FBF741FE0400162506A805FB04F1014436
:103240000120FAF71BFF06A805FB04F1084410F162
:1032500016010220FAF712FF06A805FB04F1084444
:1032600010F12C010320FAF709FF06A86C43204453
:1032700010F142010420FAF701FF0820FCF73DF8A5
:10328000002804D10120FCF738F8002802D0FBF711
:10329000A4FE02E03000FBF7BAFE32B070BD0000C1
:1032A000000000002DE97043C8B048200021F5F768
:1032B000F7F9162275496846F9F74AF900200AE03D
:1032C000002206AB162404FB00F423445A54491C84
:1032D0001629F5D3401C0C2801D20021F8E701245F
:1032E000002500265FF0FF306949F8F77BF980463A
:1032F000894615E018EA040019EA0501002901D100
:10330000002809D022002B0006A8162101FB06F197
:103310000844F8F7ADF9761C6D0045EAD4756400F1
:103320000C2E03D2002DE5D1002CE3D13000FBF7A9
:1033300093FD0320FAF76DFE0420FAF7C2FE6946FA
:103340000020FAF79BFEB9F1000F06D1B8F1000F8B
:1033500003D10020FAF761FE05E00020FBF7ABFD8A
:10336000401CFAF75AFE0220FBF7A5FD04001625C3
:1033700006A805FB04F101440120FAF77FFE06A828
:1033800005FB04F1084410F116010220FAF776FE5D
:1033900006A805FB04F1084410F12C010320FAF7FC
:1033A0006DFE06A86C43204410F142010420FAF798
:1033B00065FE0820FBF7A1FF002804D10120FBF7E0
:1033C0009CFF002802D0FBF708FE02E03000FBF76C
:1033D0001EFE48B0BDE8708310B58CB0F8F70BF94D
:1033E00004002C4B20A2162106A8F9F70CFA2300A2
:1033F0001EA216216846F9F706FA0420FAF709FE1C
:103400000120FAF75EFE06A90020FAF737FE6946AA
:103410000120FAF733FE16A421000220FAF72EFE4F
:1034200021000320FAF72AFE21000420FAF726FEE5
:1034300021000520FAF722FE21000620FAF71EFEE1
:1034400021000720FAF71AFE21000820FAF716FEDD
:103450000020FAF7E2FD0820FBF74FFF002801D01B
:10346000FBF7BBFD0CB010BD257300002564000008
:103470000000000060D2030058F901009CF5010033
:1034800060F9010068F9010070F9010080D20300C1
:10349000FFFF0F00E0DD030038B598B0040088207E
:1034A0000021F5F7FDF80320FBF7D6FC1622DFF824
:1034B000FC1312A8F9F74CF812A90020FAF7DEFD68
:1034C0000320FAF7A6FD0420FAF7FBFDDFF8E0334E
:1034D000DFF8E023162101A8F9F795F96C20F7F73A
:1034E000A0FD03280CD1B9A52A0016210DF11A0060
:1034F000F9F789F92A0016210CA8F9F784F913E0E5
:10350000DFF8B433DFF8B42316210DF11A00F9F710
:103510007AF9DFF8AC030090DFF8A833DFF8A823CE
:1035200016210CA8F9F76FF90020FBF7C4FC401C2A
:10353000FAF773FD01A90120FAF7A0FD0DF11A01B8
:103540000220FAF79BFD0CA90320FAF797FD9FA133
:103550000420FAF793FD0820FBF7CFFE002824D0C3
:103560000120FBF7A8FC002808D101211820FBF757
:10357000DCFC6C20F7F755FD206313E0012808D12F
:1035800001211920FBF7D1FC6020F7F74AFD2063E9
:1035900008E0022806D1F7F738FC206301211A2041
:1035A000FBF7C3FC206BE0630AE00120FBF7A5FEFC
:1035B000002802D0FBF711FD02E00320FBF727FDF6
:1035C00019B030BD38B588B0040088200021F5F767
:1035D00067F8B74BBD4A162102A8F9F714F902A9FA
:1035E0000020FAF74BFD206B032806D1B54BB84AF3
:1035F000162102A8F9F707F91CE0206B022808D170
:10360000B4480090AF4BB44A162102A8F9F7FBF872
:1036100010E0206B012808D1B0480090A94BAE4AB9
:10362000162102A8F9F7EFF804E01622AC4902A827
:10363000F8F78EFF0420FAF7ECFC0420FAF741FDBE
:103640000020FAF7EAFC02A90120FAF717FD5FA5AE
:1036500029000220FAF712FD29000320FAF70EFDD7
:1036600029000420FAF70AFD29000520FAF706FDD3
:1036700029000620FAF702FD29000720FAF7FEFCD0
:1036800029000820FAF7FAFC0820FBF736FE00288C
:103690000FD0206BE16B884208D0216B6C20F7F7CC
:1036A000E6FC00204FF40051F4F7FAFFFBF795FC1D
:1036B0001EE00120FBF721FE002802D0FBF78DFC65
:1036C00016E05720F7F7ADFC022801D3032105E0EF
:1036D0000221206B814201D2022020630020019050
:1036E0000120009001230022206BFBF703FD2063E3
:1036F00009B030BD38B588B0040088200021F4F747
:10370000CFFF6D4B66A2162102A8F9F77CF802A93B
:103710000020FAF7B3FC0420FAF77BFC0420FAF748
:10372000D0FC236B5FA2062102A8F9F76CF802A96E
:103730000120FAF7A3FC25A529000220FAF79EFC38
:1037400029000320FAF79AFC29000420FAF796FCD6
:1037500029000520FAF792FC29000620FAF78EFCD2
:1037600029000720FAF78AFC29000820FAF786FCCE
:103770000020FAF752FC0120FBF7BFFD002802D021
:10378000FBF72BFC20E00820FBF7B7FD00280FD04B
:10379000206BE16B884208D0216B6020F7F767FC53
:1037A00000204FF40051F4F77BFFFBF716FC0BE011
:1037B0000220019001200090012301224FF47A7130
:1037C000206BFBF797FC206309B030BD00000000C0
:1037D00038B588B0040088200021F4F761FF38482C
:1037E0000090384B3C4A162102A8F9F70CF802A9C0
:1037F0000020FAF743FC0420FAF70BFC0420FAF748
:1038000060FC0020FAF709FC236B26A2162102A80F
:10381000F8F7F9FF02A90120FAF730FC22A52900E8
:103820000220FAF72BFC29000320FAF727FC2900D5
:103830000420FAF723FC29000520FAF71FFC2900D1
:103840000620FAF71BFC29000720FAF717FC2900CD
:103850000820FAF713FC0820FBF74FFD002809D0D9
:10386000206BE16B884202D0206BF7F780FBFBF7FF
:10387000B4FB13E00120FBF740FD002802D0FBF76A
:10388000ACFB0BE0022001900120009001230022FC
:103890004FF47A71206BFBF72DFC206309B030BD2B
:1038A000257300002564000000000000C4F401003E
:1038B00040D8030098FB010060F70300A0FB010063
:1038C00048F80100D0F40100A8FB0100F8F601005F
:1038D00004F70100A0EA0300B0FB010040F801007A
:1038E00080E6030018B597B0040049200021F4F7E2
:1038F000D7FE0320FBF7B0FA1622DFF8441968461A
:10390000F8F726FE69460020FAF7B8FB0320FAF71D
:1039100080FB0420FAF7D5FBDFF82839DFF82829E7
:10392000162106A8F8F76FFFDFF82039DFF8202905
:1039300016210DF12E00F8F766FFDFF81839DFF8D1
:103940001829162111A8F8F75EFF0020FBF7B3FA3B
:10395000401CFAF762FB06A90120FAF78FFB0DF174
:103960002E010220FAF78AFB11A90320FAF786FB41
:10397000B5A10420FAF782FB0820FBF7BEFC002863
:1039800041D00120FBF797FA002804D101211C2027
:10399000FBF7CBFA42E001281FD101211E20FBF7E3
:1039A000C4FAA068012802D02069002803D10121AF
:1039B0000220FBF7BAFA4FF40040F7F723FB002888
:1039C00006D1F6F763FC002802D10020206301E055
:1039D00001202063206BE06320E002281ED1A06854
:1039E000012802D02069002808D101211D20FBF701
:1039F0009CFA01210220FBF798FA0FE001211D201B
:103A0000FBF793FA0AE00120FBF777FC002802D0CD
:103A1000FBF7E3FA02E00320FBF7F9FA18B010BD58
:103A200030B58DB049200021F4F73AFE1622DFF8B8
:103A3000141801A8F8F78CFD01A90020FAF71EFB65
:103A40000420FAF7E6FA0120FAF73BFB0A231522D5
:103A500007A9DFF80808FBF716FCF7F7C8FADFF844
:103A60000048A04201D3DFF8FC07F7F7C0FADFF8FF
:103A7000F857009007AB2A00162101A8F8F7C3FEFB
:103A800001A90120FAF7FAFA0A23152207A9DFF89B
:103A9000DC07FBF7F8FBF7F7A7FAA04201D3DFF842
:103AA000C407009007AB2A00162101A8F8F7ABFE67
:103AB00001A90520FAF7E2FA63A421000220FAF72F
:103AC000DDFA21000320FAF7D9FA21000420FAF7E1
:103AD000D5FA21000620FAF7D1FA21000720FAF7DB
:103AE000CDFA21000820FAF7C9FA0020FAF795FA72
:103AF0000820FBF702FC002801D0FBF76EFA0DB09E
:103B000030BD38B588B0040078200021F4F7C8FD36
:103B10001622DFF85C1702A8F8F71AFD02A90020A8
:103B2000FAF7ACFA0420FAF774FAF6F7AFFB0028BC
:103B300003D10420FAF7C5FA04E00320FAF7C1FA2A
:103B400001202063206B002807D1DFF8283790A2DE
:103B5000162102A8F8F757FE06E0DFF81C378CA202
:103B6000162102A8F8F74FFE02A90120FAF786FAFB
:103B700035A529000220FAF781FA29000320FAF777
:103B80007DFA29000420FAF779FA29000520FAF7CE
:103B900075FA29000620FAF771FA29000720FAF7CA
:103BA0006DFA29000820FAF769FA0020FAF735FAC9
:103BB0000120FBF7A2FB002802D0FBF70EFA40E041
:103BC0000820FBF79AFB002830D0206BE16B88427D
:103BD0000FD0206B002804D04FF40040F7F716FAFE
:103BE00003E04FF40040F7F716FA00200821F4F73D
:103BF00057FD206B002808D002211F20FBF795F904
:103C00004020F7F70EFA20630DE002212020FBF799
:103C10008CF90820F7F7F6F9002802D0012020637C
:103C200001E000202063206BE0630AE000200190A7
:103C300000200090012300220121206BFBF75AFA9B
:103C4000206309B030BD00000000000038B588B026
:103C5000040078200021F4F723FD1622DFF81C165B
:103C600002A8F8F775FC02A90020FAF707FA042069
:103C7000FAF7CFF90420FAF724FA206B002807D1CD
:103C8000DFF8F03542A2162102A8F8F7BCFD06E0E5
:103C9000DFF8E4353EA2162102A8F8F7B4FD02A928
:103CA0000120FAF7EBF988A529000220FAF7E6F9D6
:103CB00029000320FAF7E2F929000420FAF7DEF9D7
:103CC00029000520FAF7DAF929000620FAF7D6F9D3
:103CD00029000720FAF7D2F929000820FAF7CEF9CF
:103CE0000020FAF79AF90120FBF707FB002802D021
:103CF000FBF773F949E00820FBF7FFFA002839D0F9
:103D0000206BE16B88420DD0206B002803D0082087
:103D1000F7F77CF902E00820F7F77DF90020082189
:103D2000F4F7BEFC206B002821D002212120FBF7F4
:103D3000FCF85020F7F775F920635120F7F771F977
:103D400060635220F7F76DF9A063206B002805D05F
:103D5000606B002802D0A06B002805D101202063F1
:103D6000012060631420A0630020E0630DE0FBF7F6
:103D700034F90AE000200190002000900123002285
:103D80000121206BFBF7B6F9206309B030BD0000BC
:103D90002573000038B588B0040078200021F4F7BE
:103DA0007FFC1622DFF8C81402A8F8F7D1FB02A99D
:103DB0000020FAF763F90420FAF72BF9F6F766FA10
:103DC000002803D10420FAF77CF902E00320FAF777
:103DD00078F9236B3DA2162102A8F8F714FD02A979
:103DE0000120FAF74BF938A529000220FAF746F925
:103DF00029000320FAF742F929000420FAF73EF9D6
:103E000029000520FAF73AF929000620FAF736F9D1
:103E100029000720FAF732F929000820FAF72EF9CD
:103E20000020FAF7FAF80120FBF767FA002802D021
:103E3000FBF7D3F845E00820FBF75FFA00281CD019
:103E4000206BE16B884207D0216B4020F7F70FF918
:103E500000200821F4F724FC02212020FBF765F85C
:103E60000820F7F7CFF8002802D00120206301E0F6
:103E700000202063206BE06323E0F6F707FA0128B7
:103E800002D1DFF8FC1301E0DFF8F813206B42F2F7
:103E90001072B0FBF2F302FB1300002808D0206B75
:103EA00042F21073B0FBF3F02063206B50432063A9
:103EB00001200190002000901300206BFBF71AF9FD
:103EC000206309B030BD0000000000002564000040
:103ED00038B588B0040040200021F4F7E1FB162239
:103EE000DFF8981302A8F8F733FB02A90020FAF7CD
:103EF000C5F80420FAF78DF80420FAF7E2F8E06B31
:103F0000FAF78BF8E06B00281CD1A06B0190606B76
:103F10000090236BDFF87023092102A8F8F773FCE7
:103F200002A90120FAF7AAF897A529000220FAF7BA
:103F3000A5F829000320FAF7A1F829000420FAF7D0
:103F40009DF866E0E06B01281FD1236BCF4A032167
:103F500002A8F8F758FC02A90120FAF78FF8A06B25
:103F60000090636BCA4A072102A8F8F74CFC02A92B
:103F70000220FAF783F884A529000320FAF77EF8D7
:103F800029000420FAF77AF843E0E06B022822D1F6
:103F9000236BC04A042102A8F8F735FC02A90120CE
:103FA000FAF76CF8636BB94A032102A8F8F72BFC07
:103FB00002A90220FAF762F8A36BB74A042102A80B
:103FC000F8F721FC02A90320FAF758F86EA10420A3
:103FD000FAF754F81DE0606B0090236BAF4A06219E
:103FE00002A8F8F710FC02A90120FAF747F891A1FE
:103FF0000220FAF743F8A36BA44A032102A8F8F7BA
:1040000002FC02A90320FAF739F85FA10420FAF7AD
:1040100035F85DA529000520FAF730F829000620BB
:10402000FAF72CF829000720FAF728F829000820C9
:10403000FAF724F80120FBF760F9002802D0FAF71C
:10404000CCFF9FE00820FBF758F9002861D0E06B17
:10405000032830D1206B1D2808D1606B022805D1C0
:1040600094F8380010F0030F40F08C805020F6F7E1
:10407000D8FF216B81420BD15120F6F7D2FF616B43
:10408000814205D15220F6F7CCFFA16B81420FD0BF
:1040900000200821F4F704FB216B5020F6F7E7FF1E
:1040A000616B5120F6F7E3FFA16B5220F6F7DFFFBB
:1040B000FAF793FF66E0E06B022820D1606B0228DC
:1040C00006D1206B1E285DD2E06B401CE06359E0F6
:1040D000606B042808D0606B062805D0606B092847
:1040E00002D0606B0B2806D1206B1F284AD2E06BF0
:1040F000401CE06346E0E06B401CE06342E0E06BA4
:10410000012803D1E06B401CE0633BE0FAF765FF58
:1041100038E0E06B01280BD10120019001200090D4
:10412000012301221F21206BFAF7E4FF206329E01D
:10413000E06B02280BD101200190012000900123A7
:1041400001220C21606BFAF7D5FF60631AE0E06B87
:1041500003280BD1012001900120009001230022AF
:104160006321A06BFAF7C6FFA0630BE00220FBF708
:10417000BFF8002804D10420FBF7BAF8002801D0CA
:104180000120E06309B030BD0000000010B586B02A
:10419000162230496846F8F7DBF969460020F9F73E
:1041A0006DFF0420F9F735FF0320F9F78AFF3C4B38
:1041B00021A216216846F8F726FB69460120F9F787
:1041C0005DFF0020F9F729FF1CA421000220F9F768
:1041D00055FF21000320F9F751FF21000420F9F7D2
:1041E0004DFF21000520F9F749FF21000620F9F7CE
:1041F00045FF21000720F9F741FF21000720F9F7CB
:104200003DFF0120FBF779F8002802D0FAF7E5FE20
:104210000EE00820FBF771F8002809D05FF000706D
:10422000F6F720FE00208021F4F73AFAFAF7D5FEDF
:1042300006B010BD2F000000257300000000000034
:10424000A0D2030000ED0300F8F8010020ED030008
:1042500000F9010040ED030008F90100C0EC030083
:1042600000CA9A3BFFC99A3B10F90100E0EC030039
:10427000A0DD030080E60300E0D9030080EC03002A
:1042800040420F0080841E00ECF3010018F9010089
:104290006CF5010020F9010028F9010078F5010012
:1042A000E0DA030078B5ADB004000720FAF7D4FDDA
:1042B00016229C496846F8F74BF99B4B9B4A1621FE
:1042C00006A8F8F7A0FA9A4B9A4A16210DF12E008B
:1042D000F8F799FA984B994A162111A8F8F793FA2A
:1042E000974B984A16210DF15A00F8F78CFA964B25
:1042F000964A16211CA8F8F786FA954B954A16217E
:104300000DF18600F8F77FFA934B944A162127A8FF
:10431000F8F779FA0320F9F77CFE0420F9F7D1FECB
:1043200069460020F9F7AAFE0220FAF7C4FD05004D
:10433000162606A806FB05F101440120F9F79EFEAA
:1043400006A806FB05F1084410F116010220F9F752
:1043500095FE06A806FB05F1084410F12C01032088
:10436000F9F78CFE06A87543284410F14201042099
:10437000F9F784FE0020FAF79EFD401CF9F74DFE88
:104380000820FAF7BAFF00280BD0206BE16B8842B7
:1043900004D001214120FAF7C8FD12E0FAF71DFE12
:1043A0000FE00120FAF7A9FF002802D0FAF715FE66
:1043B00007E00720FAF72BFE0120FAF77CFD401CEE
:1043C00020632EB070BD38B58CB00400162255495C
:1043D00006A8F8F7BDF8206B012806D1524B4FA272
:1043E00016216846F8F70FFA55E0206B022806D12F
:1043F0004F4B4AA216216846F8F705FA4BE0206BAE
:10440000032806D14C4B45A216216846F8F7FBF964
:1044100041E0206B042806D1494B40A21621684692
:10442000F8F7F1F937E0206B052806D1464B3BA29F
:1044300016216846F8F7E7F92DE0206B062806D12B
:10444000434B36A216216846F8F7DDF923E0206BCE
:10445000072806D1404B31A216216846F8F7D3F958
:1044600019E0206B082806D13D4B2CA21621684686
:10447000F8F7C9F90FE0206B092806D1394B27A2BC
:1044800016216846F8F7BFF905E0374B23A216213D
:104490006846F8F7B8F90420F9F7BBFD0320F9F7EF
:1044A00010FE06A90020F9F7E9FD69460120F9F799
:1044B000E5FD1BA529000220F9F7E0FD29000320F6
:1044C000F9F7DCFD29000420F9F7D8FD29000520C3
:1044D000F9F7D4FD29000620F9F7D0FD29000720BF
:1044E000F9F7CCFD29000820F9F7C8FD0020F9F7FD
:1044F00094FD0120FAF701FF002802D0FAF76DFDC4
:1045000009E00820FAF7F9FE002804D0206B08F033
:10451000DBFDFAF762FD0DB030BD000025733F00F2
:104520000000000020D2030020D0030070FA010038
:1045300040D0030078FA010060D0030080FA010047
:1045400080D0030088FA0100A0D0030090FA010097
:10455000C0D0030098FA0100E0D00300A0FA0100E7
:1045600000D1030020D1030040D10300F0B5C3B057
:10457000050070200021F4F793F8F5F787FE002876
:1045800004D15FF400000021F4F78AF8F5F77EFE0D
:10459000012801D1092400E00B242000FAF75CFC7B
:1045A0001622DFF8A81B6846F7F7D2FFF5F76EFE74
:1045B00001285BD1DFF8983BDFF8982B162106A87D
:1045C000F8F721F9DFF8903BDFF8902B16210DF179
:1045D0002E00F8F718F9DFF88C3BDFF88C2B16214A
:1045E00011A8F8F710F9DFF8843BDFF8882B1621C3
:1045F0000DF15A00F8F707F9DFF87C3BDFF87C2B68
:1046000016211CA8F8F7FFF8DFF8743BDFF8742BCD
:1046100016210DF18600F8F7F6F8DFF86C3BDFF8AD
:104620006C2B162127A8F8F7EEF8DFF8643BDFF8CB
:10463000642B16210DF1B200F8F7E5F8DFF8583BCE
:10464000DFF8582B162132A8F8F7DDF806A632005D
:1046500016210DF1DE00F8F7D6F8320016213DA83C
:10466000F8F7D1F85FE000BF00000000DFF8303B52
:10467000DFF8E02A162106A8F8F7C5F8DFF8243B92
:10468000DFF8D82A16210DF12E00F8F7BCF8DFF874
:10469000C03ADFF8D42A162111A8F8F7B4F8DFF8E9
:1046A000B83ADFF8D02A16210DF15A00F8F7ABF826
:1046B000DFF8B03ADFF8C42A16211CA8F8F7A3F8EF
:1046C000DFF8A83ADFF8BC2A16210DF18600F8F7CA
:1046D0009AF8DFF8A43ADFF8B42A162127A8F8F7E9
:1046E00092F8DFF89C3ADFF8AC2A16210DF1B200FF
:1046F000F8F789F8DFF8903ADFF8A02A162132A8F7
:10470000F8F781F8DFF8883ADFF89C2A16210DF1D6
:10471000DE00F8F778F8DFF8803ADFF8902A162103
:104720003DA8F8F770F80320F9F773FC0420F9F7B7
:10473000C8FC69460020F9F7A1FC0020FAF7BBFB92
:10474000401CF9F76AFC0220FAF7B5FB06001627B1
:1047500006A807FB06F101440120F9F78FFC06A823
:1047600007FB06F1084410F116010220F9F786FC58
:1047700006A807FB06F1084410F12C010320F9F705
:104780007DFC06A87E43304410F142010420F9F775
:1047900075FC0120FAF7B1FD002802D0FAF71DFCE4
:1047A00001E10820FAF7A9FD002800F0F9800120B6
:1047B000FAF781FB0400F5F769FD01284BD1002CC5
:1047C00004D101214220FAF7B0FBE6E0012C04D12C
:1047D00001214F20FAF7A9FBDFE0022C04D10121CF
:1047E0006220FAF7A2FBD8E0032C0ED101212C2085
:1047F000FAF79BFB1020F6F705FC002802D00120F9
:104800002863CAE000202863C7E0042C04D10121FA
:104810002D20FAF78AFBC0E0052C04D101213220BB
:10482000FAF783FBB9E0062C04D101216620FAF7E0
:104830007CFBB2E0072C04D101217F20FAF775FB45
:10484000ABE0082C04D101216E20FAF76EFBA4E046
:10485000FAF7C3FBA1E0002C07D101212720FAF7CA
:1048600064FBF5F7EEFC286397E0012C29D10121C8
:104870002820FAF75AFBF5F711FD012802D1042090
:1048800028638AE0F5F718FD012802D10320286388
:1048900083E0F5F71FFD012802D1012028637CE0A9
:1048A000F5F726FD012802D10220286375E0F5F70F
:1048B0002DFD012802D1052028636EE00020286329
:1048C0006BE0022C08D1F5F72FFD002804D101215F
:1048D0004220FAF72AFB60E0032C08D1F5F724FD0B
:1048E000002804D101214F20FAF71FFB55E0042CCA
:1048F00008D1F5F719FD002804D101216220FAF74B
:1049000014FB4AE0052C12D1F5F70EFD00280ED15C
:1049100001212C20FAF709FB1020F6F773FB002881
:1049200002D00120286338E00020286335E0062CFF
:1049300008D1F5F7F9FC002804D101212D20FAF760
:10494000F4FA2AE0072C08D1F5F7EEFC002804D190
:1049500001213220FAF7E9FA1FE0082C08D1F5F717
:10496000E3FC002804D101216620FAF7DEFA14E006
:10497000092C08D1F5F7D8FC002804D101217F20AB
:10498000FAF7D3FA09E00A2C07D1F5F7CDFC002895
:1049900003D101216E20FAF7C8FA286BE86302E020
:1049A0002000FAF734FB43B0F0BD38B58EB00400F8
:1049B00028200021F3F774FEF5F768FC002804D1E5
:1049C0005FF400000021F3F76BFE1622DFF8E0171A
:1049D00008A8F7F7BDFD236B99A2162102A8F7F7E7
:1049E00012FF0420F9F715FB0420F9F76AFB0020F9
:1049F000F9F713FB08A90020F9F740FB02A90120F1
:104A0000F9F73CFB8FA529000220F9F737FB2900B5
:104A10000320F9F733FB29000420F9F72FFB2900C5
:104A20000520F9F72BFB29000620F9F727FB2900C1
:104A30000720F9F723FB29000820F9F71FFB0820BE
:104A4000FAF75BFC00280ED0E06B216B884207D0A0
:104A5000206BF5F7CFFB00204FF40061F3F720FE49
:104A6000FAF7BBFA12E00120FAF747FC002802D05F
:104A7000FAF7B3FA0AE00020019001200090012328
:104A800000220421206BFAF735FB20630FB030BD04
:104A900038B594B0040050200021F3F701FE16222F
:104AA000DFF800170EA8F7F753FD206B01280AD195
:104AB000162208A90920F5F754FC63A2162102A8C2
:104AC000F7F7A1FE41E0206B02280AD1162208A9BF
:104AD0000420F5F746FCBEA2162102A8F7F793FEC4
:104AE00033E0206B03280AD1162208A90820F5F725
:104AF00038FCB8A2162102A8F7F785FE25E0206B46
:104B000004280AD1162208A90720F5F72AFCB2A228
:104B1000162102A8F7F777FE17E0206B05280AD1C7
:104B2000162208A90A20F5F71CFCACA2162102A83F
:104B3000F7F769FE09E0AAA2162108A8F7F763FEB5
:104B400040A2162102A8F7F75EFE0420F9F761FAE9
:104B50000420F9F7B6FA0EA90020F9F78FFA08A990
:104B60000120F9F78BFA02A90520F9F787FA35A594
:104B700029000220F9F782FA29000320F9F77EFACA
:104B800029000420F9F77AFA29000620F9F776FAC5
:104B900029000720F9F772FA29000820F9F76EFAC0
:104BA0000020F9F73AFA0820FAF7A7FB002822D0EC
:104BB000206B002841D0206BE16B884204D001219A
:104BC0002920FAF7B2F938E0206B042810D101212E
:104BD0002A20FAF7AAF90220F6F714FA002802D1DF
:104BE0000020206301E001202063206BE06324E0CB
:104BF000FAF7F3F921E00120FAF77FFB002802D051
:104C0000FAF7EBF919E0206B00280BD00020019097
:104C100001200090012301220521206BFAF76AFA96
:104C200020630AE00020019001200090012300226F
:104C30000521206BFAF75EFA206315B030BD000045
:104C400025640000000000002831290038B592B02A
:104C5000040078200021F3F723FD1622DFF8441525
:104C60006846F7F775FC69460020F9F707FADFF8A0
:104C70004435A3A2162106A8F7F7C5FD206B04282A
:104C800005D1162269460720F5F76BFB1FE0206B64
:104C9000022805D1162269460420F5F762FB16E0CA
:104CA000206B032805D1162269460820F5F759FB29
:104CB0000DE0206B052805D1162269460A20F5F77C
:104CC00050FB04E0162269460920F5F74AFB6B46C3
:104CD000DFF8E42416210CA8F7F795FD0420F9F776
:104CE00098F90320F9F7EDF90020F9F796F906A9EC
:104CF0000120F9F7C3F983A529000220F9F7BEF9CD
:104D000029000320F9F7BAF929000420F9F7B6F9C8
:104D100029000520F9F7B2F929000620F9F7AEF9C4
:104D200029000720F9F7AAF929000820F9F7A6F9C0
:104D30000820FAF7E2FA002840D0206B042804D1BA
:104D400007211E20F6F793F91BE0206B022804D1FF
:104D500004211E20F6F78BF913E0206B032804D101
:104D600008211E20F6F783F90BE0206B052804D1FB
:104D70000A211E20F6F77BF903E009211E20F6F731
:104D800076F900200221F3F78BFC206B042810D168
:104D900002212A20FAF7C9F80220F6F733F9002891
:104DA00002D10020206301E001202063206BE0633A
:104DB0000CE0FAF712F9FAF710F907E00120FAF718
:104DC0009CFA002802D0200000F010FA13B030BD89
:104DD00028322900283329002834290028352900C1
:104DE0004E4F000038B58EB0040078200021F3F754
:104DF00057FC1622DFF8C41308A8F7F7A9FB206BAD
:104E0000002806D11622DFF8B81302A8F7F7A0FB96
:104E100005E01622DFF8AC1302A8F7F799FB04208F
:104E2000F9F7F7F80420F9F74CF90020F9F7F5F84D
:104E300008A90020F9F722F902A90120F9F71EF9C3
:104E400030A529000220F9F719F929000320F9F704
:104E500015F929000420F9F711F929000520F9F7BF
:104E60000DF929000620F9F709F929000720F9F7BB
:104E700005F929000820F9F701F90820FAF73DFAA9
:104E8000002826D0E06B216B88420DD0206B0028D3
:104E900003D00220F6F7BAF802E00220F6F7BBF8DA
:104EA00000200821F3F7FCFB1E20F6F7BAF80728CC
:104EB0000AD15E20F6F7B5F82063206BE06302218B
:104EC0002B20FAF732F818E0FAF787F8FAF785F8A6
:104ED00013E00120FAF711FA002803D0200000F0B7
:104EE00085F90AE0002001900120009001230022B2
:104EF0000121206BFAF7FEF820630FB030BD0000EF
:104F0000257300000000000038B58EB00400482072
:104F10000021F3F7C5FB0420F9F77BF81622AA4914
:104F200002A8F7F715FB02A90020F9F7A7F802205D
:104F3000F6F768F8216B002912D1002805D1A34AA1
:104F4000162102A8F7F75FFC04E0A14A162102A887
:104F5000F7F759FC7BA2162108A8F7F754FC27E0C5
:104F6000216B012912D1002805D19A4A162102A8E5
:104F7000F7F749FC04E0984A162102A8F7F743FC2A
:104F800071A2162108A8F7F73EFC11E0002805D110
:104F9000924A162102A8F7F736FC04E0904A16213F
:104FA00002A8F7F730FC6EA2162108A8F7F72BFC31
:104FB0000020F9F732F802A90120F9F75FF86CA593
:104FC00029000220F9F75AF829000320F9F756F8CA
:104FD00029000420F9F752F808A90520F9F74EF83E
:104FE00029000620F9F74AF829000720F9F746F8C2
:104FF00029000820F9F742F80420F9F762F80820A0
:10500000FAF77BF9002810D0E06B216B884207D0BB
:10501000216B5E20F6F72BF800200821F3F740FB08
:10502000F9F7DBFFF9F7D9FF13E00120FAF765F98B
:10503000002803D0200000F0D9F80AE000200190F9
:1050400001200090012300220221206BFAF752F880
:1050500020630FB030BD38B58EB004007020002141
:10506000F3F71EFB1622414908A8F7F771FA206BE7
:10507000002805D116225B4902A8F7F769FA04E077
:105080001622594902A8F7F763FA0420F8F7C1FF7E
:105090000420F9F716F80020F8F7BFFF08A9002050
:1050A000F8F7ECFF02A90120F8F7E8FF30A5290086
:1050B0000220F8F7E3FF29000320F8F7DFFF2900BB
:1050C0000420F8F7DBFF29000520F8F7D7FF2900B7
:1050D0000620F8F7D3FF29000720F8F7CFFF2900B3
:1050E0000820F8F7CBFF0820FAF707F9002814D0BA
:1050F000206BE16B88420DD0206B002803D110207B
:10510000F5F789FF02E01020F5F780FF0020082165
:10511000F3F7C6FAF9F761FF12E00120FAF7EDF8AC
:10512000002802D0F9F759FF0AE000200190012081
:105130000090012300220121206BF9F7DBFF20639F
:105140000FB030BD283129002832290040D2030099
:1051500040D30300B8FB010060D30300C0FB010093
:105160002833290080F10300C8FB010080D303002D
:1051700000000000D0FB0100A0D30300D8FB010019
:10518000C0D30300E0FB0100E0D30300E8FB010013
:1051900020F10300F0FB010020D40300F8FB010024
:1051A00028F2010060F4030000FC010008FC01008B
:1051B000ACF30100E0DA03006CF4010000DA030054
:1051C000C0DA0300A0DA030000F6030010F70100C4
:1051D0001CF701002CF301007CF4010028F701000A
:1051E00034F7010080E60300E0D9030010B50400A5
:1051F000F5F754F8012802D1042020631DE0F5F7EB
:105200005BF8012802D10320206316E0F5F762F86D
:10521000012802D1012020630FE0F5F769F8012889
:1052200002D10220206308E0F5F770F8012802D1CE
:105230000520206301E000202063206BE063F9F784
:10524000CCFE10BD78B5A7B0040070200021F3F7A4
:1052500027FA0620F9F700FEF5F718F8012801D122
:10526000062500E005251622C5496846F7F770F9BE
:10527000F5F70CF8012828D1C24E3300C24A162196
:1052800006A8F7F7C0FAC14BC14A16210DF12E004E
:10529000F7F7B9FA3300BF4A162111A8F7F7B3FAA6
:1052A0003300BD4A16210DF15A00F7F7ACFA33006E
:1052B000BA4A16211CA8F7F7A6FAB94BB94A162123
:1052C0000DF18600F7F79FFA26E0AE4E3300AE4AA6
:1052D000162106A8F7F797FAAC4BAD4A16210DF147
:1052E0002E00F7F790FA3300AF4A162111A8F7F70E
:1052F0008AFA3300AD4A16210DF15A00F7F783FA06
:10530000A74BAB4A16211CA8F7F77DFA9BA21621E2
:105310000DF18600F7F777FA0320F8F77AFE0420FC
:10532000F8F7CFFE0020F9F7C6FD401CF8F775FE30
:1053300069460020F8F7A2FE0220F9F7BCFD162608
:1053400006A9704301440120F8F798FE0220F9F7FE
:10535000B2FD06A97043084410F116010220F8F7C7
:105360008DFE0220F9F7A7FD06A97043084410F14D
:105370002C010320F8F782FE0220F9F79CFD06A914
:1053800006FB00F601EB060010F142010420F8F7DD
:1053900075FE0120F9F7B1FF002802D0F9F71DFED4
:1053A0004EE00820F9F7A9FF002846D00120F9F7C0
:1053B00082FD002804D101214420F9F7B6FD3FE029
:1053C000012804D101214B20F9F7AFFD38E0022874
:1053D00004D101214520F9F7A8FD31E003280DD1C2
:1053E000F4F754FF012804D101214620F9F79DFD6F
:1053F00026E001214720F9F798FD21E0042811D18A
:10540000F4F744FF012804D101214720F9F78DFD6D
:1054100016E001214320F9F788FD3B20F5F701FE56
:1054200020630DE005280BD101214320F9F77DFD14
:105430003B20F5F7F6FD206302E02800F9F7E7FDD1
:1054400028B070BD38B58CB0040070200021F3F78F
:1054500027F9534B574A162106A8F7F7D4F9206BC2
:10546000012805D1162254496846F7F771F80FE074
:10547000206B022805D1162250496846F7F768F8D4
:1054800006E016224E496846F7F762F800202063CE
:105490000420F8F7BEFD0420F8F713FE06A900204B
:1054A000F8F7ECFD69460120F8F7E8FD33A529007F
:1054B0000220F8F7E3FD29000320F8F7DFFD2900BB
:1054C0000420F8F7DBFD29000520F8F7D7FD2900B7
:1054D0000620F8F7D3FD29000720F8F7CFFD2900B3
:1054E0000820F8F7CBFD0020F8F797FD0120F9F729
:1054F00004FF002802D0F9F770FD3CE00820F9F71E
:10550000FCFE002810D03B20F5F78BFD216B81427B
:1055100007D0216B3B20F5F7AAFD00200421F3F70B
:10552000BFF8F9F75AFD26E00220F9F7E1FE00285E
:105530000ED0206B012802D1022020631BE0206BDB
:10554000022802D10020206315E00120206312E030
:105550000420F9F7CDFE00280DD0206B022802D1DF
:105560000120206307E0206B012802D10020206386
:1055700001E0022020630DB030BD000000000000FB
:1055800040D3030080D403002CF60100A0D4030014
:1055900038F6010044F6010050F601005CF6010007
:1055A00020D5030068F6010074F6010080F60100C2
:1055B0008CF6010010FA010080D90300A0D9030085
:1055C00080E6030010B59CB0040070200021F3F7C2
:1055D00067F80420F9F740FCDFF8103BDFF8102BE8
:1055E00016216846F7F70FF91622A4A106A8F6F7C8
:1055F000AFFF1622A2A10DF12E00F6F7A9FF162289
:10560000A0A111A8F6F7A4FF16229FA10DF15A0040
:10561000F6F79EFF0320F8F7FCFC0420F8F751FD95
:105620000020F9F748FC401CF8F7F7FC6946002019
:10563000F8F724FD06A90120F8F720FD0DF12E0151
:105640000220F8F71BFD11A90320F8F717FD0DF153
:105650005A010420F8F712FD0120F9F74EFE002848
:1056600002D0F9F7BAFC32E00820F9F746FE00282C
:105670002AD00120F9F71FFC002806D1012001F0F3
:1056800027F820630120606417E0012806D102207A
:1056900001F01EF82063022060640EE0022806D1AB
:1056A00003206064032001F013F8206305E0042068
:1056B0006064042001F00CF8206301214820F9F710
:1056C00034FC206BE06302E00420F9F7A0FC1CB07E
:1056D00010BD30B591B0040070200021F2F7E0FF5A
:1056E0000220F9F7B9FBDFF8043ADFF8082A16219F
:1056F0006846F7F788F869460020F8F7BFFC0320F2
:10570000F8F787FC0420F8F7DCFC1622B6A106A8FF
:10571000F6F71EFF1622B5A10DF12E00F6F718FFC1
:105720000020F9F7C8FB401CF8F777FC06A9012018
:10573000F8F7A4FC0DF12E010220F8F79FFCACA5B0
:1057400029000320F8F79AFC29000420F8F796FCBA
:105750000820F9F7D2FD002818D00120F9F7ABFB9B
:10576000002806D109206064092000F0B1FF206301
:1057700005E00A2060640A2000F0AAFF20630121EE
:105780004820F9F7D2FB206BE0630AE00120F9F72B
:10579000B4FD002802D0F9F720FC02E00220F9F75E
:1057A00036FC11B030BD30B591B00400702000213E
:1057B000F2F776FF0220F9F74FFBDFF83039DFF818
:1057C0004C2B16216846F7F71EF869460020F8F7BB
:1057D00055FC0320F8F71DFC0420F8F772FC0020AC
:1057E000F9F769FB401CF8F718FC82A2162106A8FD
:1057F000F7F709F880A216210DF12E00F7F703F84C
:1058000006A90120F8F73AFC0DF12E010220F8F765
:1058100035FC77A529000320F8F730FC2900042087
:10582000F8F72CFC0820F9F768FD002818D00120B3
:10583000F9F741FB002806D10B2060640B2000F033
:1058400047FF206305E00C2060640C2000F040FF5F
:10585000206301214820F9F768FB206BE0630AE030
:105860000120F9F74AFD002802D0F9F7B6FB02E063
:105870000220F9F7CCFB11B030BD00004931000027
:1058800049320000493300004934000070B59CB033
:105890000400F4F7FBFC012801D1042500E00225F7
:1058A00070200021F2F7FCFE0420F9F7D5FADFF8AA
:1058B0003C38DFF8602A162116A8F6F7A4FF4FA29D
:1058C00016216846F6F79FFF4DA216210DF116002E
:1058D000F6F799FFF4F7DAFC01280BD149A216215B
:1058E0000BA8F6F790FF48A216210DF14200F6F73B
:1058F0008AFF0BE03EA6320016210BA8F6F783FFC5
:10590000320016210DF14200F6F77DFF0320F8F773
:1059100080FB0420F8F7D5FB0020F9F7CCFA401CF7
:10592000F8F77BFB16A90020F8F7A8FB69460120D1
:10593000F8F7A4FB0DF116010220F8F79FFB0BA965
:105940000320F8F79BFB0DF142010420F8F796FBCA
:105950000120F9F7D2FC002802D0F9F73EFB41E024
:105960000820F9F7CAFC002839D00120F9F7A3FA7A
:10597000002806D1052000F0ABFE206305206064FE
:1059800026E0012811D1F4F781FC012806D1062078
:1059900000F09EFE20630620606419E0082000F0FD
:1059A00097FE20630820606412E002280AD1F4F711
:1059B0006DFC012806D1072000F08AFE2063072035
:1059C000606405E0082000F083FE20630820606426
:1059D00001214820F9F7A9FA206BE06302E02800D2
:1059E000F9F715FB1CB070BD4531000045320000D1
:1059F0000000000020490000204500005331000055
:105A000053320000533300005334000070B58EB0A1
:105A100004000420F8F7FDFA70200021F2F740FEA0
:105A200002A9606C00F024FDDFF83C0A009002AB94
:105A3000DFF8382A162108A8F6F7E5FE08A90020A5
:105A4000F8F71CFB226B162102A8F5F751FE02A9FC
:105A50000120F8F713FB0CA631000220F8F70EFB2B
:105A600031000320F8F70AFB31000420F8F706FBA9
:105A7000206B002802D0206B222807D33200162189
:105A800002A8F6F7C0FE0CE000000000206BF5F75E
:105A900046FE05002B00DFF8BC2A162102A8F6F707
:105AA000B2FE02A90520F8F7E9FA31000620F8F75E
:105AB000E5FA31000720F8F7E1FA31000820F8F79D
:105AC000DDFA0020F8F7A9FA0420F8F7FAFA08201E
:105AD000F9F713FC002800F01781206BE16B884276
:105AE0001BD0206BF5F724FE0500206B0C280ED090
:105AF000206B0D280BD0206B102808D0206B0F28AE
:105B000005D0206B0E2802D035F0C00501E055F01D
:105B1000C0052900606C00F092FDF4F7B7FB012886
:105B200040F0C88000206063206B1B2808D0206BE9
:105B30001C2805D0206B112802D0206B12283CD1E4
:105B4000606C012806D12900022000F078FD0120B8
:105B50006063AFE0606C032806D12900042000F0E8
:105B60006EFD01206063A5E0606C052806D1290068
:105B7000062000F064FD012060639BE0606C072854
:105B800006D12900082000F05AFD0120606391E051
:105B9000606C092806D129000A2000F050FD012080
:105BA000606387E0606C0B2840F0848029000C2043
:105BB00000F045FD012060637CE0606C012811D19C
:105BC000022000F0F1FC30F0C000102805D01128B0
:105BD00003D00B2801D00A286CD100212A20F5F728
:105BE00046FA67E0606C032811D1042000F0DCFC69
:105BF00030F0C000102805D0112803D00B2801D0A8
:105C00000A2857D100212E20F5F731FA52E0606CB6
:105C1000092811D10A2000F0C7FC30F0C00010287C
:105C200005D0112803D00B2801D00A2842D1002129
:105C30003220F5F71CFA3DE0606C052811D10620F2
:105C400000F0B2FC30F0C000102805D0112803D0BD
:105C50000B2801D00A282DD100212220F5F707FAC0
:105C600028E0606C072811D1082000F09DFC30F07E
:105C7000C000102805D0112803D00B2801D00A2815
:105C800018D100212620F5F7F2F913E0606C0B28FB
:105C900010D10C2000F088FC30F0C000102805D096
:105CA000112803D00B2801D00A2803D10021362067
:105CB000F5F7DDF900200421F2F7F2FC206B002853
:105CC0001FD0206B02281CD0206B032819D0206B1A
:105CD000052816D0206B062813D0606C00F064FCF9
:105CE00010F08000002802D00120206301E0002095
:105CF000206302214920F9F718F9206BE0630EB008
:105D000070BDF9F76AF9FAE70120F9F7F6FA002809
:105D100002D0F9F762F9F2E7F4F7B8FA01285BD19B
:105D2000606C02280ED0606C04280BD0606C0628D2
:105D300008D0606C082805D0606C0A2802D0606C1E
:105D40000C2849D1606C022804D1012000F0C0FC6D
:105D5000050026E0606C042804D1032000F0B8FCA4
:105D600005001EE0606C0A2804D1092000F0B0FC98
:105D7000050016E0606C062804D1052000F0A8FCA0
:105D800005000EE0606C082804D1072000F0A0FC9C
:105D9000050006E0606C0C2803D10B2000F098FC95
:105DA00005001B2D05D01C2D03D0112D01D0122D67
:105DB00004D125630120F8F784F9A0E7206B1B28A4
:105DC00008D0206B1C2805D0206B112802D0206B36
:105DD000122801D1002020630020019001200090B2
:105DE000012300222121206BF9F784F92063F4F7C5
:105DF0004DFA012840F01E81606C0B2836D1206BD3
:105E00001A281BD0206B132818D0206B142815D00B
:105E1000206B152812D0206B16280FD0206B172866
:105E20000CD0206B0E2809D0206B1F2806D0206BC9
:105E30001E2803D0206B1A287FF461AF0020019048
:105E400001200090012300222121206BF9F752F953
:105E500020630220F9F74CFA0028D0D10420F9F78A
:105E600042FA0028CBD100202063C8E7606C0C28E0
:105E700042D1206B1A2827D0206B132824D0206B06
:105E8000142821D0206B15281ED0206B16281BD07B
:105E9000206B112818D0206B122815D0206B1728E2
:105EA00012D0206B0E280FD0206B1F280CD0206B37
:105EB0001B2809D0206B1C2806D0206B1E2803D07D
:105EC000206B1A287FF41BAF002001900120009066
:105ED000012300222121206BF9F70CF92063022015
:105EE000F9F706FA0028C4D10420F9F7FCF90028D4
:105EF000BFD100202063BCE7606C02280BD0606C2F
:105F0000042808D0606C062805D0606C082802D0F0
:105F1000606C0A284ED1206B132833D0206B1428D4
:105F200030D0206B15282DD0206B16282AD0206B5E
:105F3000112827D0206B122824D0206B172821D0BD
:105F4000206B0E281ED0206B1F281BD0206B1B2817
:105F500018D0206B1C2815D0206B1E2812D0206B67
:105F60001A280FD0206B03280CD0206B022809D0F0
:105F7000206B062806D0206B052803D0206B1A283A
:105F80007FF4BDAE0020019001200090012300228B
:105F90002121206BF9F7AEF820630220F9F7A8F968
:105FA0000028B8D10420F9F79EF90028B3D10020C9
:105FB0002063B0E7206B132824D0206B142821D055
:105FC000206B15281ED0206B16281BD0206B17289D
:105FD00018D0206B0E2815D0206B1F2812D0206BF4
:105FE0001E280FD0206B1A280CD0206B032809D054
:105FF000206B022806D0206B062803D0206B0528D2
:106000007FF47DAE0020019001200090012300224A
:106010002121206BF9F76EF820630220F9F768F967
:106020000028C7D10420F9F75EF90028C2D100206A
:106030002063BFE7F4F732F9012803D0F4F766F9DB
:10604000012834D1206B022812D0206B03280FD0F6
:10605000206B05280CD0206B062809D0206B09285E
:1060600006D0206B0B2803D0206B1D287FF447AE91
:106070000020019001200090012300222121206BAB
:10608000F9F738F820630220F9F732F90028D9D15E
:106090000420F9F728F90028D4D100202063D1E7A3
:1060A0000420F9F720F9002801D100202063206B9B
:1060B000022809D0206B032806D0206B052803D0C6
:1060C000206B06287FF41BAE002001900120009079
:1060D000012300222121206BF9F70CF82063022014
:1060E000F9F706F90028E2D1DAE7000080D40300CE
:1060F00098F60100A4F6010038B58EB004007020B7
:106100000021F2F7CDFA02A9606C00F0B1F902AB00
:10611000DFF87C24162108A8F6F775FB206B002811
:1061200006D11622DFF86C1402A8F6F711FA05E082
:106130001622DFF8641402A8F6F70AFA0420F7F72B
:1061400068FF0420F7F7BDFF08A90020F7F796FFC6
:1061500002A90120F7F792FF6DA529000220F7F7A9
:106160008DFF29000320F7F789FF29000420F7F7A6
:1061700085FF29000520F7F781FF29000620F7F7A2
:106180007DFF29000720F7F779FF29000820F7F79E
:1061900075FF0020F7F741FF0820F9F7AEF8002857
:1061A00070D0606C00F000FA0500206BE16B884253
:1061B00007D0206B002802D135F0800501E055F0B2
:1061C00080052900606C00F03AFAF4F75FF80128C6
:1061D00031D1606B00282ED0606C012804D12900D9
:1061E000022000F02CFA26E0606C032804D129007C
:1061F000042000F024FA1EE0606C052804D1290078
:10620000062000F01CFA16E0606C072804D1290073
:10621000082000F014FA0EE0606C092804D129006F
:106220000A2000F00CFA06E0606C0B2803D129006C
:106230000C2000F004FA00200421F2F731FA606C1F
:1062400000F046FA0C2807D00F2805D0102803D0FC
:106250000D2801D00E2812D1606C00F0A5F910F0C5
:106260004000002802D00120206301E000202063CC
:10627000206BE06302214A20F8F757FE43E0F8F76D
:10628000ACFE40E00120F9F738F8002802D0F8F71A
:10629000A4FE38E0F3F7FAFF012820D1606C00F08B
:1062A00017FA616C02290ED0616C04290BD0616C65
:1062B000062908D0616C082905D0616C0A2902D032
:1062C000616C0C290BD11B2805D01C2803D0112888
:1062D00001D0122803D10120F7F7F3FE13E00020CC
:1062E000019001200090012300220121206BF8F78A
:1062F00001FF2063606C00F057F930F0C0001728F0
:1063000001D1002020630FB030BD000018FA010059
:1063100000000000B0F6010038B58EB00400702017
:106320000021F2F7BDF902A9606C00F0A1F802AB00
:106330009A4A162108A8F6F766FA206B002805D1BC
:106340001622974902A8F6F703F904E016229549A8
:1063500002A8F6F7FDF80420F7F75BFE0420F7F734
:10636000B0FE08A90020F7F789FE02A90120F7F77F
:1063700085FE79A529000220F7F780FE2900032079
:10638000F7F77CFE29000420F7F778FE29000520A6
:10639000F7F774FE29000620F7F770FE29000720A2
:1063A000F7F76CFE29000820F7F768FE0020F7F7E2
:1063B00034FE0820F8F7A1FF002819D0606C00F027
:1063C000F3F80100206BE26B904207D0206B0028AD
:1063D00002D131F0400101E051F04001606C00F069
:1063E0002EF900200421F2F75BF9F8F7F6FD38E00A
:1063F0000120F8F782FF002802D0F8F7EEFD30E028
:10640000F3F744FF012821D1606C02280ED0606CA4
:1064100004280BD0606C062808D0606C082805D0D2
:10642000606C0A2802D0606C0C280FD1206B1B28EE
:1064300008D0206B1C2805D0206B112802D0206BBF
:10644000122803D10120F7F73CFE0AE0002001905A
:1064500001200090012300220121206BF8F74AFE61
:1064600020630FB030BD000040D8030020FA0100C7
:1064700010B50C00012805D138A204212000F6F740
:10648000C2F966E0022805D135A204212000F6F702
:10649000BAF95EE0032805D132A204212000F6F704
:1064A000B2F956E0042805D12FA204212000F6F706
:1064B000AAF94EE0092805D12CA204212000F6F704
:1064C000A2F946E00A2805D129A204212000F6F706
:1064D0009AF93EE0052805D126A204212000F6F70E
:1064E00092F936E0062805D123A204212000F6F710
:1064F0008AF92EE0072805D120A204212000F6F712
:1065000082F926E008280FD1F3F7C0FE012805D153
:106510001BA204212000F6F776F91AE016A2042146
:106520002000F6F770F914E00B2805D115A204211C
:106530002000F6F768F90CE00C2805D112A204211E
:106540002000F6F760F904E010A204212000F6F71D
:106550005AF910BD28FA010000000000493100007E
:106560004932000049330000493400004531000041
:106570004532000053310000533200005333000015
:10658000533400004900000045000000457200003F
:10659000BCF6010040D9030060D9030030FA0100C5
:1065A00080E60300E0D9030080B5012803D128204C
:1065B000F4F737FD42E0022803D12A20F4F731FD39
:1065C0003CE0032803D12C20F4F72BFD36E004280F
:1065D00003D12E20F4F725FD30E0052803D120203B
:1065E000F4F71FFD2AE0062803D12220F4F719FD55
:1065F00024E0072803D12420F4F713FD1EE0082827
:1066000003D12620F4F70DFD18E0092803D130202E
:10661000F4F707FD12E00A2803D13220F4F701FD58
:106620000CE00B2803D13420F4F7FBFC06E00C2827
:1066300003D13620F4F7F5FC00E0002002BD80B560
:10664000012803D12820F4F712FD40E0022803D1ED
:106650002A20F4F70CFD3AE0032803D12C20F4F7AC
:1066600006FD34E0042803D12E20F4F700FD2EE0CF
:10667000052803D12020F4F7FAFC28E0062803D1EE
:106680002220F4F7F4FC22E0072803D12420F4F7B9
:10669000EEFC1CE0082803D12620F4F7E8FC16E005
:1066A0000B2803D13420F4F7E2FC10E00C2803D1CE
:1066B0003620F4F7DCFC0AE0092803D13020F4F797
:1066C000D6FC04E00A2802D13220F4F7D0FC01BD48
:1066D00080B5FFF769FF30F0C000F5F7AFF8C0B242
:1066E00002BD000030B591B0040070200021F1F728
:1066F000D7FF0220F8F7B0FBDFF8B434DFF8B4249A
:1067000016216846F6F77FF88FA2162106A8F6F73D
:106710007AF88EA216210DF12E00F6F774F80320F8
:10672000F7F777FC0420F7F7CCFC0020F8F7C3FB61
:10673000401CF7F772FC69460020F7F79FFC06A99A
:106740000120F7F79BFC0DF12E010220F7F796FCD4
:10675000CAA529000320F7F791FC29000420F7F7C8
:106760008DFC0120F8F7C9FD002802D0F8F735FCB0
:1067700024E00820F8F7C1FD00281CD00120F8F71C
:106780009AFB002808D10D2060644820F4F749FCEA
:1067900030F0C000206307E00E2060644920F4F769
:1067A00040FC30F0C000206301214C20F8F7BDFB15
:1067B000206BE06302E00220F8F729FC11B030BD45
:1067C00038B58EB0040070200021F1F769FF042075
:1067D000F7F71FFC606C0D2808D1DFF8DC33DFF819
:1067E000DC23162108A8F6F70EF807E0DFF8C83317
:1067F000DFF8CC23162108A8F6F705F808A9002031
:10680000F7F73CFC226BD2B2162102A8F5F79DF8EF
:1068100002A90120F7F732FC98A529000220F7F71A
:106820002DFC29000320F7F729FC29000420F7F7A5
:1068300025FC226BDFF88C1302A8F5F7D9FF02A91B
:106840000520F7F71BFC29000620F7F717FC2900A5
:106850000720F7F713FC29000820F7F70FFC0020AA
:10686000F7F7DBFB0420F7F72CFC0820F8F745FDD1
:10687000002853D0206BE16B88421FD0606C0D283C
:1068800006D14820F4F7CDFB010011F0800105E0AE
:106890004920F4F7C6FB010011F08001206B014391
:1068A000606C0D2803D14820F4F7E1FB02E0492099
:1068B000F4F7DDFB00200821F1F7F2FE206B092838
:1068C00010D102214E20F8F730FB606C0D2804D166
:1068D0004A20F4F7A6FB206333E04B20F4F7A1FB3A
:1068E00020632EE002214D20F8F71FFB606C0D287D
:1068F00005D14820F4F795FB10F0800004E0492012
:10690000F4F78FFB10F08000002802D001202063F4
:1069100001E000202063206BE06312E00120F8F723
:10692000ECFC002802D0F8F758FB0AE000200190A8
:1069300001200090012300221421206BF8F7DAFBDC
:1069400020630FB030BD00004F3100004F32000017
:1069500038B58EB0040070200021F1F7A1FE606C04
:106960000D2806D1984B954A162108A8F5F74BFF3C
:1069700005E0954B924A162108A8F5F744FF236BD2
:10698000924A162102A8F5F73EFF0420F7F741FBD3
:106990000420F7F796FB0020F7F73FFB08A900203B
:1069A000F7F76CFB02A90120F7F768FB33A5290074
:1069B0000220F7F763FB29000320F7F75FFB2900AC
:1069C0000420F7F75BFB29000520F7F757FB2900A8
:1069D0000620F7F753FB29000720F7F74FFB2900A4
:1069E0000820F7F74BFB0820F8F787FC00282FD08A
:1069F000206BE16B88420FD0606C0D2804D1216BB5
:106A00004A20F4F734FB03E0216B4B20F4F72FFB13
:106A100000200821F1F744FE02214D20F8F785FA05
:106A2000606C0D2805D14820F4F7FBFA10F08000C7
:106A300004E04920F4F7F5FA10F08000002802D0B5
:106A40000120206301E000202063206BE06312E05E
:106A50000120F8F752FC002802D0F8F7BEFA0AE04D
:106A6000012001900020009001230122F021206BE1
:106A7000F8F740FB20630FB030BD000000000000BD
:106A800038B58EB0040070200021F1F709FE606C6B
:106A90000D2805D14E4A162108A8F5F7B4FE04E0EA
:106AA0004C4A162108A8F5F7AEFE206B002805D148
:106AB0001622494902A8F5F74BFD04E01622474982
:106AC00002A8F5F745FD0420F7F7A3FA0420F7F72D
:106AD000F8FA0020F7F7A1FA08A90020F7F7CEFA94
:106AE00002A90120F7F7CAFA30A529000220F7F71A
:106AF000C5FA29000320F7F7C1FA29000420F7F7A7
:106B0000BDFA29000520F7F7B9FA29000620F7F7A2
:106B1000B5FA29000720F7F7B1FA29000820F7F79E
:106B2000ADFA0120F8F7E9FB002802D0F8F755FA92
:106B300039E00820F8F7E1FB002829D0206BE16B51
:106B4000884222D0606C0D2806D14820F4F769FAFB
:106B5000010031F0800105E04920F4F762FA0100FC
:106B600031F08001206B002801D051F08001606C71
:106B70000D2803D14820F4F77AFA02E04920F4F70F
:106B800076FA00200821F1F78BFDF8F726FA0AE0E3
:106B90000020019001200090012300220121206BA0
:106BA000F8F7A8FA20630FB030BD00000000000025
:106BB000A0D40300D4F6010040D8030068FB010014
:106BC00070FB010078FB010020D9030080FB01006D
:106BD000E0F60100ECF6010040D9030060D90300A3
:106BE00010B59CB0040070200021F1F759FD04207D
:106BF000F8F732F9DFF80C39A8A216216846F5F744
:106C000002FEDFF80439DFF80429162106A8F5F79B
:106C1000FAFDDFF8FC38DFF8FC2816210DF12E0014
:106C2000F5F7F1FDDFF8F038DFF8F028162111A8AC
:106C3000F5F7E9FDDFF8E838DFF8E82816210DF16F
:106C40005A00F5F7E0FD0320F7F7E3F90420F7F722
:106C500038FA0020F8F72FF9401CF7F7DEF96946FB
:106C60000020F7F70BFA06A90120F7F707FA0DF154
:106C70002E010220F7F702FA11A90320F7F7FEF917
:106C80000DF15A010420F7F7F9F90820F8F735FB60
:106C9000002826D00120F8F70EF9002804D10121A0
:106CA0005020F8F742F919E0012804D101215820B9
:106CB000F8F73BF912E0022808D101216020F8F72B
:106CC00034F95420F4F7ADF9206307E00121612085
:106CD000F8F72BF95C20F4F7A4F92063206BE0634C
:106CE0000AE00120F8F709FB002802D0F8F775F94F
:106CF00002E00420F8F78BF91CB010BD78B5A7B0FE
:106D0000040070200021F1F7CBFC0620F8F7A4F86E
:106D1000DFF8F43761A216216846F5F774FDDFF855
:106D20000838DFF8E827162106A8F5F76CFDDFF82C
:106D3000FC37DFF8E02716210DF12E00F5F763FD93
:106D4000DFF8EC37DFF8D427162111A8F5F75BFD43
:106D5000DFF8E037DFF8CC2716210DF15A00F5F700
:106D600052FDDFF8D437DFF8D42716211CA8F5F739
:106D70004AFDDFF8CC37DFF8CC2716210DF186006D
:106D8000F5F741FD0320F7F744F90420F7F799F9E7
:106D90000020F8F790F8401CF7F73FF9694600200B
:106DA000F7F76CF90220F8F786F80500162606A812
:106DB00006FB05F101440120F7F760F906A806FB80
:106DC00005F1084410F116010220F7F757F906A85B
:106DD00006FB05F1084410F12C010320F7F74EF9EA
:106DE00006A87543284410F142010420F7F746F93C
:106DF0000820F8F782FA002842D00120F8F75BF863
:106E0000002808D101215120F8F78FF81620F4F757
:106E100008F920633FE0012808D101215220F8F74A
:106E200084F81020F4F7FDF8206334E0022808D13C
:106E300001215420F8F779F80E20F4F7F2F82063D6
:106E400029E0032808D101215520F8F76EF81C200D
:106E5000F4F7E7F820631EE0042808D1012156204A
:106E6000F8F763F80420F4F7DCF8206313E001215D
:106E70005720F8F75AF80620F4F7D3F820630AE011
:106E80000120F8F73AFA002802D0F8F7A6F802E055
:106E90000620F8F7BCF828B070BD0000257300008C
:106EA00038B58EB0040070200021F1F7F9FB1622EE
:106EB000DFF8941608A8F5F74BFB236B9CA216216C
:106EC00002A8F5F7A0FC0420F7F7A3F80420F7F7D1
:106ED000F8F80020F7F7A1F808A90020F7F7CEF896
:106EE00002A90120F7F7CAF8D0A529000220F7F778
:106EF000C5F829000320F7F7C1F829000420F7F7A7
:106F0000BDF829000520F7F7B9F829000620F7F7A2
:106F1000B5F829000720F7F7B1F829000820F7F79E
:106F2000ADF80820F8F7E9F9002810D01620F4F79A
:106F300078F8216B814207D0216B1620F4F797F87F
:106F400000200221F1F7ACFBF8F747F812E001202E
:106F5000F8F7D3F9002802D0F8F73FF80AE000204C
:106F6000019001200090012301220A21206BF8F7F3
:106F7000C1F820630FB030BD38B58EB0040070206A
:106F80000021F1F78DFB1622DFF8C01508A8F5F7F0
:106F9000DFFA236BDFF8B825162102A8F5F733FCDA
:106FA0000420F7F736F808A90020F7F767F802A9D8
:106FB0000120F7F763F89DA529000220F7F75EF896
:106FC00029000320F7F75AF829000420F7F756F8AC
:106FD00029000520F7F752F829000620F7F74EF8A8
:106FE00029000720F7F74AF829000820F7F746F8A4
:106FF0000020F7F712F80820F8F77FF9002816D0DC
:107000001020F4F70EF8216B814207D0216B10207D
:10701000F4F72DF800200221F1F742FB0221532062
:10702000F7F783FF0020F3F7FCFF206312E0012055
:10703000F8F763F9002802D0F7F7CFFF0AE0012044
:1070400001900020009001230022C821206BF8F756
:1070500051F820630FB030BD38B58EB004007020F9
:107060000021F1F71DFB1622DFF8E81408A8F5F758
:107070006FFA236BB1A2162102A8F5F7C4FB042016
:10708000F6F7C7FF0420F7F71CF808A90020F6F769
:10709000F5FF02A90120F6F7F1FF64A529000220FF
:1070A000F6F7ECFF29000320F6F7E8FF290004209B
:1070B000F6F7E4FF29000520F6F7E0FF2900062097
:1070C000F6F7DCFF29000720F6F7D8FF2900082093
:1070D000F6F7D4FF0020F6F7A0FF0820F8F70DF927
:1070E000002810D00020F3F79CFF216B814207D0CD
:1070F000216B0020F3F7BBFF00200221F1F7D0FA4B
:10710000F7F76BFF12E00120F8F7F7F8002802D03C
:10711000F7F763FF0AE000200190002000900123B0
:1071200001220321206BF7F7E5FF20630FB030BD8C
:107130002532640038B58EB0040070200021F1F7CC
:10714000AFFA1622DFF8101408A8F5F701FA236B3E
:10715000B1A2162102A8F5F756FB0420F6F759FF55
:10716000F3F794F8012803D10120F6F7AAFF02E013
:107170000420F6F7A6FF08A90020F6F77FFF02A972
:107180000120F6F77BFF29A529000220F6F776FFFC
:1071900029000320F6F772FF29000420F6F76EFF9E
:1071A00029000520F6F76AFF29000620F6F766FF9A
:1071B00029000720F6F762FF29000820F6F75EFF96
:1071C0000020F6F72AFF0820F8F797F8002810D0DB
:1071D0000E20F3F726FF216B814207D0216B0E2092
:1071E000F3F745FF00200221F1F75AFAF7F7F5FE11
:1071F0001AE00120F8F781F8002806D0F3F746F8E6
:10720000012811D0F7F7E9FE0EE0F3F73FF8012867
:107210000AD00020019000200090012301220A21C1
:10722000206BF7F767FF20630FB030BD0000000050
:1072300030B58FB0040070200021F1F731FA16222A
:10724000C64909A8F5F784F9236BC54A032102A8AA
:10725000F5F7D9FA9DF808008DF80C0003A82E2147
:1072600041709DF8091081700021C1700420F6F76B
:10727000D0FEF3F70BF8012803D10120F6F721FF28
:1072800002E00420F6F71DFF09A90020F6F7F6FE3C
:1072900003A90120F6F7F2FE96A10220F6F7EEFE12
:1072A00095A529000320F6F7E9FE29000420F6F74A
:1072B000E5FE29000520F6F7E1FE29000620F6F795
:1072C000DDFE29000720F6F7D9FE29000820F6F791
:1072D000D5FE0020F6F7A1FE0820F8F70EF80028EA
:1072E0000FD01C20F3F79DFE216B814207D0216B4C
:1072F0001C20F3F7BCFE00200221F1F7D1F9F7F7CB
:107300006CFE0120F7F7F9FF002806D0F2F7BEFF68
:10731000012811D0F7F761FE0EE0F2F7B7FF012860
:107320000AD00120019000200090012301221E219B
:10733000206BF7F7DFFE20630FB030BD256400003F
:1073400038B58EB0040070200021F1F7A9F916229B
:10735000844908A8F5F7FCF8236B68A2162102A857
:10736000F5F751FA0420F6F754FE0420F6F7A9FECB
:107370000020F6F752FE08A90020F6F77FFE02A9CA
:107380000120F6F77BFE5CA529000220F6F776FEC9
:1073900029000320F6F772FE29000420F6F76EFE9E
:1073A00029000520F6F76AFE29000620F6F766FE9A
:1073B00029000720F6F762FE29000820F6F75EFE96
:1073C0000820F7F79AFF002810D00420F3F729FED1
:1073D000216B814207D0216B0420F3F748FE002087
:1073E0000221F1F75DF9F7F7F8FD12E00120F7F758
:1073F00084FF002802D0F7F7F0FD0AE0002001909A
:1074000000200090012301220A21206BF7F772FE71
:1074100020630FB030BD00002532640038B58EB057
:10742000040070200021F1F73BF916224E4908A80C
:10743000F5F78EF8236B32A2162102A8F5F7E3F9CF
:107440000420F6F7E6FD0420F6F73BFE0020F6F7F1
:10745000E4FD08A90020F6F711FE02A90120F6F7C5
:107460000DFE25A529000220F6F708FE29000320BD
:10747000F6F704FE29000420F6F700FE2900052097
:10748000F6F7FCFD29000620F6F7F8FD2900072095
:10749000F6F7F4FD29000820F6F7F0FD0820F7F7CD
:1074A0002CFF002810D00620F3F7BBFD216B814292
:1074B00007D0216B0620F3F7DAFD00200221F1F757
:1074C000EFF8F7F78AFD12E00120F7F716FF002822
:1074D00002D0F7F782FD0AE0002001900020009022
:1074E000012301220A21206BF7F704FE20630FB06D
:1074F00030BD000020730000000000002564000083
:107500002532640060D3030080D50300E8FA01004F
:10751000A0D50300F0FA0100C0F50300F8FA01005D
:1075200020F7030000FB0100C0D50300E0D50300F5
:1075300000D6030020D6030040D6030008FB01005C
:1075400060D6030010FB010080D60300A0D6030024
:1075500018FB0100C0D60300E0D6030000D70300EB
:1075600020FB010020D7030040D7030078B5A7B067
:10757000040070200021F1F793F80620F7F76CFC67
:10758000DFF8703997A216216846F5F73CF9DFF865
:107590006839DFF86829162106A8F5F734F9DFF80D
:1075A0006039DFF8602916210DF12E00F5F72BF96F
:1075B000DFF85439DFF85429162111A8F5F723F91B
:1075C000DFF84C39DFF84C2916210DF15A00F5F798
:1075D0001AF9DFF84439DFF8442916211CA8F5F719
:1075E00012F9DFF83C39DFF83C2916210DF186004D
:1075F000F5F709F90320F6F70CFD0420F6F761FD15
:107600000020F7F758FC401CF6F707FD69460020FC
:10761000F6F734FD0220F7F74EFC0500162606A803
:1076200006FB05F101440120F6F728FD06A806FB3C
:1076300005F1084410F116010220F6F71FFD06A817
:1076400006FB05F1084410F12C010320F6F716FDA6
:1076500006A87543284410F142010420F6F70EFDF8
:107660000820F7F74AFE002842D00120F7F723FC54
:10767000002808D101215920F7F757FC1820F3F70B
:10768000D0FC20633FE0012808D101215A20F7F700
:107690004CFC1220F3F7C5FC206334E0022808D12B
:1076A00001215C20F7F741FC0C20F3F7BAFC2063C2
:1076B00029E0032808D101215D20F7F736FC1A20C4
:1076C000F3F7AFFC20631EE0042808D101215E20FF
:1076D000F7F72BFC0820F3F7A4FC206313E001214B
:1076E0005F20F7F722FC0A20F3F79BFC20630AE0F7
:1076F0000120F7F702FE002802D0F7F76EFC02E047
:107700000620F7F784FC28B070BD38B58EB00400B1
:1077100070200021F0F7C4FF1622DFF80C1808A82B
:10772000F4F716FF236BA0A2162102A8F5F76BF859
:107730000420F6F76EFC0420F6F7C3FC0020F6F7F1
:107740006CFC08A90020F6F799FC02A90120F6F7C5
:1077500095FCCCA529000220F6F790FC2900032017
:10776000F6F78CFC29000420F6F788FC2900052098
:10777000F6F784FC29000620F6F780FC2900072094
:10778000F6F77CFC29000820F6F778FC0820F7F7CC
:10779000B4FD002810D01820F3F743FC216B814280
:1077A00007D0216B1820F3F762FC00200221F0F7CC
:1077B00077FFF7F712FC12E00120F7F79EFD002893
:1077C00002D0F7F70AFC0AE00020019000200090A8
:1077D000012301220A21206BF7F78CFC20630FB0F4
:1077E00030BD00002573000038B58EB00400702055
:1077F0000021F0F755FF1622DFF8301708A8F4F73C
:10780000A7FE236BDFF82827162102A8F4F7FBFF59
:107810000420F6F7FEFB0420F6F753FC08A900202D
:10782000F6F72CFC02A90120F6F728FC95A5290003
:107830000220F6F723FC29000320F6F71FFC29009D
:107840000420F6F71BFC29000520F6F717FC290099
:107850000620F6F713FC29000720F6F70FFC290095
:107860000820F6F70BFC0020F6F7D7FB0820F7F707
:1078700044FD002816D01220F3F7D3FB216B814280
:1078800007D0216B1220F3F7F2FB00200221F0F762
:1078900007FF02215B20F7F748FB0220F3F7C1FB4B
:1078A000206312E00120F7F728FD002802D0F7F747
:1078B00094FB0AE0012001900020009001230022A7
:1078C000C821206BF7F716FC20630FB030BD38B528
:1078D0008EB0040070200021F0F7E2FE1622DFF8DF
:1078E000541608A8F4F734FE236B2FA2162102A821
:1078F000F4F789FF0420F6F78CFB0420F6F7E1FB90
:1079000008A90020F6F7BAFB02A90120F6F7B6FB9A
:107910005CA529000220F6F7B1FB29000320F6F749
:10792000ADFB29000420F6F7A9FB29000520F6F796
:10793000A5FB29000620F6F7A1FB29000720F6F792
:107940009DFB29000820F6F799FB0020F6F765FB60
:107950000820F7F7D2FC002810D00220F3F761FBD3
:10796000216B814207D0216B0220F3F780FB0020BE
:107970000221F0F795FEF7F730FB12E00120F7F750
:10798000BCFC002802D0F7F728FB0AE00020019099
:1079900000200090012301220321206BF7F7AAFBAE
:1079A00020630FB030BD00002564000038B58EB0F4
:1079B000040070200021F0F773FE1622DFF878151E
:1079C00008A8F4F7C5FD236BA1A2162102A8F4F7BD
:1079D0001AFF0420F6F71DFB0420F6F772FB08A936
:1079E0000020F6F74BFB02A90120F6F747FB25A57F
:1079F00029000220F6F742FB29000320F6F73EFBA0
:107A000029000420F6F73AFB29000520F6F736FB9B
:107A100029000620F6F732FB29000720F6F72EFB97
:107A200029000820F6F72AFB0020F6F7F6FA0820CE
:107A3000F7F763FC002810D00C20F3F7F2FA216B63
:107A4000814207D0216B0C20F3F711FB00200221AB
:107A5000F0F726FEF7F7C1FA12E00120F7F74DFC28
:107A6000002802D0F7F7B9FA0AE0002001900020C0
:107A70000090012301220A21206BF7F73BFB2063D2
:107A80000FB030BD0000000030B58FB00400702092
:107A90000021F0F705FE1622DFF8A01409A8F4F77C
:107AA00057FD236BDFF89824032102A8F4F7ABFEFF
:107AB0009DF808008DF80C0003A82E2141709DF858
:107AC000091081700021C1700420F6F7A2FA042089
:107AD000F6F7F7FA09A90020F6F7D0FA03A9012072
:107AE000F6F7CCFAC6A10220F6F7C8FAC5A5290018
:107AF0000320F6F7C3FA29000420F6F7BFFA29009D
:107B00000520F6F7BBFA29000620F6F7B7FA290098
:107B10000720F6F7B3FA29000820F6F7AFFA00209D
:107B2000F6F77BFA0820F7F7E8FB00280FD01A20B9
:107B3000F3F777FA216B814207D0216B1A20F3F714
:107B400096FA00200221F0F7ABFDF7F746FA012084
:107B5000F7F7D3FB002802D0F7F73FFA0AE001203D
:107B6000019000200090012301221E21206BF7F7D5
:107B7000C1FA20630FB030BD38B58EB0040070205C
:107B80000021F0F78DFD1622DFF8B81308A8F4F7EE
:107B9000DFFC236B9CA2162102A8F4F734FE04201C
:107BA000F6F737FA0420F6F78CFA0020F6F735FAE4
:107BB00008A90020F6F762FA02A90120F6F75EFA9A
:107BC00090A529000220F6F759FA29000320F6F7BC
:107BD00055FA29000420F6F751FA29000520F6F796
:107BE0004DFA29000620F6F749FA29000720F6F792
:107BF00045FA29000820F6F741FA0820F7F77DFB3F
:107C0000002810D00820F3F70CFA216B814207D02E
:107C1000216B0820F3F72BFA00200221F0F740FD3A
:107C2000F7F7DBF912E00120F7F767FB002802D035
:107C3000F7F7D3F90AE0002001900020009001231B
:107C400001220A21206BF7F755FA20630FB030BDEF
:107C50002532640038B58EB0040070200021F0F7A2
:107C60001FFD1622B84908A8F4F772FC236B66A220
:107C7000162102A8F4F7C7FD0420F6F7CAF904207C
:107C8000F6F71FFA0020F6F7C8F908A90020F6F762
:107C9000F5F902A90120F6F7F1F95AA52900022009
:107CA000F6F7ECF929000320F6F7E8F9290004209B
:107CB000F6F7E4F929000520F6F7E0F92900062097
:107CC000F6F7DCF929000720F6F7D8F92900082093
:107CD000F6F7D4F90820F7F710FB002810D00A2097
:107CE000F3F79FF9216B814207D0216B0A20F3F74C
:107CF000BEF900200221F0F7D3FCF7F76EF912E08D
:107D00000120F7F7FAFA002802D0F7F766F90AE03F
:107D10000020019000200090012301220A21206B05
:107D2000F7F7E8F920630FB030BD38B58EB0040026
:107D300070200021F0F7B4FC1622844908A8F4F75B
:107D400007FC236B30A2162102A8F4F75CFD042087
:107D5000F6F75FF90420F6F7B4F90020F6F75DF9BD
:107D600008A90020F6F78AF902A90120F6F786F99A
:107D700024A529000220F6F781F929000320F6F74F
:107D80007DF929000420F6F779F929000520F6F796
:107D900075F929000620F6F771F929000720F6F792
:107DA0006DF929000820F6F769F90820F7F7A5FA18
:107DB000002810D05420F3F734F9216B814207D00A
:107DC000216B5420F3F753F900200821F0F768FCE9
:107DD000F7F703F912E00120F7F78FFA002802D035
:107DE000F7F7FBF80AE00020019000200090012343
:107DF00001220521206BF7F77DF920630FB030BD1C
:107E000020730000000000002564000038B58EB02B
:107E1000040070200021F0F743FC4D4B32A21621E4
:107E200008A8F4F7F0FC236B30A2162102A8F4F79F
:107E3000EAFC0420F6F7EDF808A90020F6F71EF991
:107E400002A90120F6F71AF929A529000220F6F760
:107E500015F929000320F6F711F929000420F6F797
:107E60000DF929000520F6F709F929000620F6F793
:107E700005F929000720F6F701F929000820F6F78F
:107E8000FDF80020F6F7C9F80820F7F736FA0028C1
:107E90000ED0206BE16B884207D0216B5C20F3F79A
:107EA000E6F800200821F0F7FBFBF7F796F819E059
:107EB0000120F7F722FA002802D0F7F78EF811E038
:107EC000F2F7E4F9012802D1002020630AE0002043
:107ED000019001200090012300220A21206BF7F776
:107EE00009F920630FB030BD25730000253264000E
:107EF00000000000A0D50300C0D5030028FB01004E
:107F0000E0D5030030FB010000D6030038FB010080
:107F100020D6030040FB010040D6030048FB0100CF
:107F200060D6030050FB010060D7030080D7030038
:107F300058FB0100A0D70300C0D70300E0D703001F
:107F400060FB010000D8030020D80300C0F5030047
:107F500020F7030030B597B070200021F0F7A0FBA8
:107F60000320F6F779FF1622DFF89C136846F4F732
:107F7000EFFADFF89833DFF89823162106A8F4F714
:107F800042FCDFF89033DFF8902316210DF12E002C
:107F9000F4F739FCE14BE24A162111A8F4F733FC5F
:107FA0000320F6F736F80420F6F78BF80020F6F7F2
:107FB00082FF401CF6F731F80220F6F77CFF040040
:107FC00069460020F6F75AF8162506A805FB04F1C5
:107FD00001440120F6F752F806A805FB04F1084415
:107FE00010F116010220F6F749F806A805FB04F186
:107FF000084410F12C010320F6F740F806A86C4362
:10800000204410F142010420F6F738F80120F7F778
:1080100074F9002802D0F6F7E0FF2CE00820F7F70B
:108020006CF9002824D00120F6F745FF002809D17B
:1080300001216320F6F779FF3820F2F7F2FFB94902
:10804000086018E0012809D101216420F6F76DFFCE
:108050003920F2F7E6FFB34908600CE00121652002
:10806000F6F763FF3A20F2F7DCFFAE49086002E062
:108070000320F6F7CCFF17B030BD38B588B07020BC
:108080000021F0F70DFB1622A04902A8F4F760FAD0
:1080900002A90020F5F7F2FF0420F5F7BAFFA14C82
:1080A0002368A14A162102A8F4F7ADFB02A901201A
:1080B000F5F7E4FF0420F6F704F891A52900022063
:1080C000F5F7DCFF29000320F5F7D8FF290004208D
:1080D000F5F7D4FF29000520F5F7D0FF2900062089
:1080E000F5F7CCFF29000720F5F7C8FF2900082085
:1080F000F5F7C4FF0020F5F790FF0820F7F7FDF82B
:10810000002810D03820F2F78CFF2168814207D078
:1081100021683820F2F7ABFF00200421F0F7C0FA05
:10812000F6F75BFF12E00120F7F7E7F8002802D02E
:10813000F6F753FF0AE00120019000200090012390
:1081400000221E212068F6F7D5FF206009B030BD5F
:1081500038B58EB070200021F0F7A2FA0420F5F7B0
:1081600058FF0420F5F7ADFF16226A4908A8F4F776
:10817000EFF908A90020F5F781FF6A4C23686A4AE5
:10818000162102A8F4F73FFB02A90120F5F776FFBC
:108190005BA529000220F5F771FF29000320F5F700
:1081A0006DFF29000420F5F769FF29000520F5F788
:1081B00065FF29000620F5F761FF29000720F5F784
:1081C0005DFF29000820F5F759FF0020F5F725FF8E
:1081D0000820F7F792F8002810D03920F2F721FF95
:1081E0002168814207D021683920F2F740FF002042
:1081F0000421F0F755FAF6F7F0FE12E00120F7F748
:108200007CF8002802D0F6F7E8FE0AE00120019091
:108210000020009001230022F0212068F6F76AFF79
:1082200020600FB030BD38B58EB070200021F0F75F
:1082300037FA3A4B33A2162108A8F4F7E4FA394C7E
:108240002368394A162102A8F4F7DDFA0420F5F76D
:10825000E0FE0420F5F735FF0020F5F7DEFE08A963
:108260000020F5F70BFF02A90120F5F707FF24A571
:1082700029000220F5F702FF29000320F5F7FEFE92
:1082800029000420F5F7FAFE29000520F5F7F6FE8F
:1082900029000620F5F7F2FE29000720F5F7EEFE8B
:1082A00029000820F5F7EAFE0120F7F726F8002854
:1082B00002D0F6F792FE20E00820F7F71EF800281B
:1082C00010D03A20F2F7ADFE2168814207D0216834
:1082D0003A20F2F7CCFE00200421F0F7E1F9F6F79E
:1082E0007CFE0AE001200190002000900123002282
:1082F000F0212068F6F7FEFE20600FB030BD0000D0
:10830000000000002573000080F1030040D403004A
:1083100010FC010060D4030018FC010060D50300CC
:1083200020FC01009011002028FC01002DE9F841FB
:10833000A7B0050048200021F0F7B2F91622DFF8B7
:10834000741921A8F4F704F921A90020F5F796FE85
:108350005720F2F766FE0400002C06D1DFF85829FA
:1083600016216846F4F74FFA06E02300DFF84C299F
:1083700016216846F4F747FA002C0CD05620F2F785
:1083800050FE800707D5DFF8382916210DF11600B9
:10839000F4F739FA06E0DFF82C2916210DF1160062
:1083A000F4F731FA002C0BD05620F2F73AFE4007D2
:1083B00006D5DFF8142916210BA8F4F724FA05E0F6
:1083C000DFF8082916210BA8F4F71DFA002C0CD0B1
:1083D0005620F2F726FE000707D5DFF8F42816210D
:1083E0000DF14200F4F70FFA06E0DFF8E828162155
:1083F0000DF14200F4F707FA012C12D10626DFF83E
:10840000D838DFF8D828162116A8F4F7FCF9DFF8D9
:10841000D038DFF8D02816210DF16E00F4F7F3F90B
:108420000CE0B9A63200162116A8F4F7ECF93200D8
:1084300016210DF16E00F4F7E6F904263000F6F788
:108440000BFD0320F5F7E5FD0420F5F73AFE0020CB
:10845000F6F731FD401CF5F7E0FD0220F6F72BFDA5
:1084600007005FF01608684608FB07F10144012089
:10847000F5F704FE684608FB07F1084410F1160101
:108480000220F5F7FBFD684608FB07F1084410F1F0
:108490002C010320F5F7F2FD684608FB07F7384486
:1084A00010F142010420F5F7E9FD0120F6F725FF60
:1084B000002802D0F6F791FD8CE00820F6F71DFFAA
:1084C000002800F084800120F6F7F5FC002808D190
:1084D00001218020F6F729FD5720F2F7A2FD28633D
:1084E00072E0012828D1F1F7D1FE012804D1012141
:1084F0000F20F6F71AFD67E0012C01D0032C16D1EE
:1085000001218120F6F711FD5620F2F78AFD800740
:1085100002D40020286357E05820F2F782FD022899
:1085200002D1022028634FE0012028634CE00121A2
:108530008620F6F7FAFC47E0022820D1F1F7A6FEE4
:10854000012804D101210F20F6F7EFFC3CE0002CBC
:1085500010D0092C0ED201218320F6F7E6FC56201C
:10856000F2F75FFD400702D4002028632CE00120D1
:10857000286329E001218620F6F7D7FC24E00328B0
:1085800017D1002C10D0082C0ED201218220F6F732
:10859000CCFC5620F2F745FD000702D400202863EA
:1085A00012E0012028630FE001218620F6F7BDFCD0
:1085B0000AE0042804D101218420F6F7B6FC03E088
:1085C00001218720F6F7B1FC286BE86302E0300058
:1085D000F6F71DFD28B0BDE8F08138B58EB0040077
:1085E000C8200021F0F75CF8DFF8C836DFF8F8267D
:1085F000162108A8F4F707F9206B002807D1DFF847
:10860000EC3698A2162102A8F4F7FDF806E0236BD9
:10861000DFF8DC26162102A8F4F7F5F80420F5F7B8
:10862000F8FC0420F5F74DFD08A90020F5F726FD1C
:1086300002A90120F5F722FD33A529000220F5F754
:108640001DFD29000320F5F719FD29000420F5F789
:1086500015FD29000520F5F711FD29000620F5F785
:108660000DFD29000720F5F709FD29000820F5F781
:1086700005FD0020F5F7D1FC0820F6F73EFE0028A6
:108680002DD0206BE16B884226D0216B5720F2F76A
:10869000EEFC6C20F2F7C5FC03280BD1206B0228FE
:1086A00008D200216C20F2F7E2FC00204FF40051C8
:1086B000EFF7F6FF00215620F2F7D9FC206B0228D5
:1086C00006D30020F2F764FE00204021EFF7E8FF18
:1086D00000200821EFF7E4FFF6F77FFC12E001200D
:1086E000F6F70BFE002802D0F6F777FC0AE0002030
:1086F000019001200090012300220F21206BF6F74A
:10870000F9FC20630FB030BD0000000038B58EB01A
:10871000040048200021EFF7C3FF0420F5F779FC9F
:108720001622DFF8D01508A8F3F712FF08A90020D9
:10873000F5F7A4FC206B002806D11622DFF8AC1553
:1087400002A8F3F705FF0FE0206B012806D11622DF
:10875000DFF8A41502A8F3F7FBFE05E01622DFF808
:108760009C1502A8F3F7F4FE02A90120F5F786FC98
:1087700089A529000220F5F781FC29000320F5F7DF
:108780007DFC29000420F5F779FC206B002804D13A
:1087900029000520F5F772FC11E05720F2F741FCA3
:1087A000012801D1032300E00123DFF8542516211D
:1087B00002A8F4F728F802A90520F5F75FFC2900C4
:1087C0000620F5F75BFC29000720F5F757FC290088
:1087D0000820F5F753FC0020F5F71FFC0420F5F7FF
:1087E00070FC0820F6F789FD002826D0206BE16B8D
:1087F00088421FD05620F2F714FC010031F002012C
:10880000206B002801D1012409E0206B012803D14D
:1088100051F00201012402E051F00201022456202D
:10882000F2F725FC21005820F2F721FC0020082156
:10883000EFF736FFF6F7D1FB12E00120F6F75DFD0A
:10884000002802D0F6F7C9FB0AE0002001900120C1
:108850000090012300220221206BF6F74BFC2063DD
:108860000FB030BD2573000070B58EB004004820F5
:108870000021EFF715FF0420F5F7CBFB1622DFF8F8
:10888000841408A8F3F764FE08A90020F5F7F6FBA6
:108890005720F2F7C6FB0500E80701D46D1E00E083
:1088A0006D1C206B012806D11622DFF85C1402A88B
:1088B000F3F74EFE05E01622DFF8301402A8F3F7B6
:1088C00047FE02A90120F5F7D9FB33A631000220AB
:1088D000F5F7D4FB31000320F5F7D0FB310004207D
:1088E000F5F7CCFB206B002804D131000520F5F70B
:1088F000C5FB0AE02B00DFF80824162102A8F3F7D5
:1089000082FF02A90520F5F7B9FB31000620F5F733
:10891000B5FB31000720F5F7B1FB31000820F5F772
:10892000ADFB0020F5F779FB0420F5F7CAFB082022
:10893000F6F7E3FC002819D05620F2F772FB01008D
:10894000206BE26B90420ED0206B012802D151F0D7
:10895000040101E031F004015620F2F788FB002009
:108960000821EFF79DFEF6F738FB12E00120F6F73D
:10897000C4FC002802D0F6F730FB0AE0002001908A
:1089800001200090012300220121206BF6F7B2FBA9
:1089900020630EB070BD00000000000070B58EB006
:1089A000040048200021EFF77BFE0420F5F731FB9F
:1089B000D64B9BA2162108A8F3F725FF08A9002093
:1089C000F5F75CFB5720F2F72CFB05000835206B10
:1089D000012805D11622CC4902A8F3F7B9FD04E01D
:1089E0001622C24902A8F3F7B3FD02A90120F5F748
:1089F00045FBAEA631000220F5F740FB3100032015
:108A0000F5F73CFB31000420F5F738FB206B00281C
:108A100004D131000520F5F731FB09E02B00B84AFD
:108A2000162102A8F3F7EFFE02A90520F5F726FBB1
:108A300031000620F5F722FB31000720F5F71EFB79
:108A400031000820F5F71AFB0020F5F7E6FA0420BC
:108A5000F5F737FB0820F6F750FC002819D0562010
:108A6000F2F7DFFA0100206BE26B90420ED0206B30
:108A7000012802D151F0080101E031F0080156202F
:108A8000F2F7F5FA00200821EFF70AFEF6F7A5FA4B
:108A900012E00120F6F731FC002802D0F6F79DFA2B
:108AA0000AE0002001900120009001230022012112
:108AB000206BF6F71FFB20630EB070BD38B58CB08D
:108AC000040048200021EFF7EBFD55A5824B2A005A
:108AD000162106A8F3F797FE8D4B2A00162168464B
:108AE000F3F791FE0420F5F794FA0320F5F7E9FA7D
:108AF0000020F5F792FA06A90020F5F7BFFA6946BB
:108B00000120F5F7BBFA69A529000220F5F7B6FAAE
:108B100029000320F5F7B2FA29000420F5F7AEFA90
:108B200029000520F5F7AAFA29000620F5F7A6FA8C
:108B300029000720F5F7A2FA29000820F5F79EFA88
:108B40000820F6F7DAFB00280ED04020F2F78AF969
:108B500000208021EFF7A4FD02218520F6F7E5F93A
:108B6000F1F7FEF9206306E00120F6F7C6FB0028C6
:108B700001D0F6F732FA0DB030BD38B58CB0040034
:108B80001622554906A8F3F7E3FC624A1621684607
:108B9000F3F739FE0420F5F73CFA0020F5F791FAD7
:108BA00006A90020F5F76AFA69460120F5F766FA8A
:108BB0003EA529000220F5F761FA29000320F5F708
:108BC0005DFA29000420F5F759FA29000520F5F788
:108BD00055FA29000620F5F751FA29000720F5F784
:108BE0004DFA29000820F5F749FA0020F5F715FAA3
:108BF000F1F7B6F9216B401A40F2D17188420CD3DB
:108C00005FF080700021F2F7EDFC002905D100280B
:108C100003D102218720F6F788F90DB030BD00009E
:108C20002573000010B58CB021A2162106A8F3F719
:108C3000EAFD394A16216846F3F7E5FD0420F5F709
:108C4000E8F90120F5F73DFA06A90020F5F716FA34
:108C500069460120F5F712FA14A421000220F5F765
:108C60000DFA21000320F5F709FA21000420F5F799
:108C700005FA21000520F5F701FA21000620F5F795
:108C8000FDF921000720F5F7F9F921000820F5F793
:108C9000F5F90020F5F7C1F90820F6F72EFB0028BA
:108CA00001D0F6F79AF90CB010BD000000000000EA
:108CB0002049440020F1030050F101003CF2010082
:108CC00050F2010068F1010064F2010080F101003E
:108CD00078F2010098F1010080E0030070F80100D3
:108CE00020F6030078F8010080F8010080E6030018
:108CF00088F8010080F4030040F6030060F60300EA
:108D000000F50100A0F40300E0D90300ACF4010079
:108D1000E0DA03000CF5010090F801002DE9F043C2
:108D2000E9B00400DFF8540A0021EFF7B9FC002590
:108D30000DE095A216210EA8162303FB05F3184497
:108D4000F3F761FD00205BA941F825006D1C0E2D95
:108D5000EFD3012601205B90F2F7E7F98046F2F7A6
:108D6000CEF90500F2F7D6F907005FF0FF30F2F711
:108D70001BFC002801D057F001075FF002090BE04F
:108D80004846F1F7B4FD18EA000F03D05BA840F89D
:108D90002690761C19F10109B9F1100FF0D35FF09C
:108DA00000082AE002A8019008A8009059F828308D
:108DB000DFF8CC2916210EA85FF0160C0CFB08FC7E
:108DC0006044F3F720FD16E070A2162102A8F3F725
:108DD0001AFD59F828001028E4D302A8009008AB27
:108DE000DFF8A02916210EA85FF0160C0CFB08FC7A
:108DF0006044F3F708FD18F10108B04546D20DF5BF
:108E0000B67959F82800F2F707FA162208A9F1F7FF
:108E1000A8FA59F82800F1F76AFD054203D159F87C
:108E200028100129D0D1074218D059F82800F2F7AC
:108E30000CFA00280CD059F82800F2F706FAFF289F
:108E400006D0DFF84429162102A8F3F7DCFCC0E7BE
:108E50004EA2162102A8F3F7D6FCBAE759F828006B
:108E6000F2F7F3F900280BD059F82800F2F7EDF9E2
:108E7000FF2805D0A5A2162102A8F3F7C4FCA8E795
:108E800041A2162102A8F3F7BEFCA2E73000F5F7D5
:108E9000E3FF0320F5F7BDF80420F5F712F91622D9
:108EA000DFF8E81802A8F3F753FB02A90020F5F752
:108EB000E5F80020F5F7FFFF401CF5F7AEF80220BB
:108EC000F5F7F9FF07005FF016080EA808FB07F199
:108ED00001440120F5F7D2F80EA808FB07F1084479
:108EE00010F116010220F5F7C9F80EA808FB07F1EA
:108EF000084410F12C010320F5F7C0F80EA808FB78
:108F000007F7384410F142010420F5F7B7F80120C3
:108F1000F6F7F3F9002802D0F6F75FF830E0082002
:108F2000F6F7EBF9002828D00120F5F7C4FF5BA97C
:108F300051F820002064206CF2F76EF90600206CD6
:108F4000F1F7D5FC054206D0162202A93000F1F750
:108F500008FA012802D0206C012811D1206CF2F708
:108F60005BF9102804D101218E20F5F7DEFF07E020
:108F700001218820F5F7D9FF02E03000F6F747F825
:108F800069B0BDE8F083000000000000282129003E
:108F900078B5A9B00400206CEFF78DFB5FF480007A
:108FA0000021EFF77DFB206CF2F736F9162201A9BC
:108FB000F1F7D7F9002802D1F6F70FF8A3E001A8DE
:108FC0000090236CDFF8C827162107A8F3F71BFCD5
:108FD00007A90020F5F752F8DFF8B82716210DA8E9
:108FE000F3F711FCDFF8B037DFF8B02716210DF1E9
:108FF0004A00F3F708FCDFF8A837DFF8A8271621A6
:1090000018A8F3F700FCDFF8A037DFF8A027162137
:109010000DF17600F3F7F7FBDFF89437DFF89427CC
:10902000162123A8F3F7EFFB0520F5F715FF032022
:10903000F4F7EFFF0420F5F744F80220F5F73BFFC3
:10904000050016260DA806FB05F101440120F5F7E1
:1090500015F80DA806FB05F1084410F116010220D1
:10906000F5F70CF80DA806FB05F1084410F12C01EA
:109070000320F5F703F80DA87543284410F14201C9
:109080000420F4F7FBFF0020F5F715FF401CF4F770
:10909000C4FF0120F6F731F9002802D0F5F79DFF53
:1090A00031E00820F6F729F9002829D00120F5F74A
:1090B00002FF002804D101218920F5F736FF1CE0CA
:1090C000012804D101218B20F5F72FFF15E002289C
:1090D00004D101218A20F5F728FF0EE0032804D1EE
:1090E00001218C20F5F721FF07E0206CF2F7ADF8A5
:1090F000206301218D20F5F718FF206BE06302E06B
:109100000520F5F784FF2AB070BD0000282A290049
:109110002DE9F043CFB00700386CEFF7CCFA5FF4DD
:1091200080000021EFF7BCFA386CF2F775F81622D0
:1091300001A9F1F716F901A800903B6CDFF8502661
:10914000162107A8F3F75FFB07A90020F4F796FFA5
:1091500000200AE000220DAB162404FB00F4234497
:109160005A54491C1629F5D3401C0C2801D2002161
:10917000F8E7012400250026386CF1F7EFFF804660
:10918000894615E018EA040019EA0501002901D111
:10919000002809D022002B000DA8162101FB06F1A2
:1091A0000844F2F765FA761C6D0045EAD475640050
:1091B0000C2E03D2002DE5D1002CE3D13000F5F7C1
:1091C0004BFE0320F4F725FF0420F4F77AFF07A9EC
:1091D0000020F4F753FFB9F1000F06D1B8F1000FEA
:1091E00003D10020F4F719FF05E00020F5F763FE36
:1091F000401CF4F712FF0220F5F75DFE040016256F
:109200000DA805FB04F101440120F4F737FF0DA878
:1092100005FB04F1084410F116010220F4F72EFFBB
:109220000DA805FB04F1084410F12C010320F4F70C
:1092300025FF0DA86C43204410F142010420F4F7EF
:109240001DFF0820F6F759F8002804D10120F6F791
:1092500054F8002802D0F5F7C0FE02E03000F5F720
:10926000D6FE4FB0BDE8F083F0B5B9B00400206C75
:10927000EFF721FA5FF480000021EFF711FA206C7C
:10928000F1F7CAFF162201A9F1F76BF801A80090C7
:10929000236CDFF8FC24162107A8F3F7B4FA07A91A
:1092A0000020F4F7EBFE0320F4F7B3FE0420F4F7FC
:1092B00008FF00200AE000220DAB162505FB00F593
:1092C0002B445A54491C1629F5D3401C082801D2B6
:1092D0000021F8E7206CF1F733FF0500206CF1F76F
:1092E0009BFF062801D1012700E00027012400266A
:1092F0000CE0254209D03A0021000DA8162303FBFB
:1093000006F31844F2F77AF9761C6400082E01D2AD
:10931000002CEED13000F5F79FFD002D03D1002089
:10932000F4F77BFE05E00020F5F7C5FD401CF4F7DF
:1093300074FE0220F5F7BFFD040016250DA805FBFD
:1093400004F101440120F4F799FE0DA805FB04F196
:10935000084410F116010220F4F790FE0DA805FB59
:1093600004F1084410F12C010320F4F787FE0DA846
:109370006C43204410F142010420F4F77FFE0820E2
:10938000F5F7BBFF002804D10120F5F7B6FF002850
:1093900002D0F5F722FE02E03000F5F738FE39B0D2
:1093A000F0BD18B58DB00400206CEFF784F95FF4C0
:1093B00080000021EFF774F9206CF1F72DFF1622E1
:1093C00007A9F0F7CEFF07A80090236CDFF8C023B1
:1093D000162101A8F3F717FA01A90020F4F74EFEB1
:1093E0000420F4F716FE0120F4F76BFE0A23152281
:1093F00007A9DFF8C403F5F746FF206CF1F7C8FEB4
:10940000009007ABDFF8B423162101A8F3F7FBF9AE
:1094100001A90120F4F732FE84A421000220F4F710
:109420002DFE21000320F4F729FE21000420F4F78B
:1094300025FE21000520F4F721FE21000620F4F787
:109440001DFE21000720F4F719FE21000820F4F783
:1094500015FE0020F4F7E1FD0820F5F74EFF002887
:1094600001D0F5F7BAFD0EB010BD30B5A5B00400BF
:1094700002A8D3490A680260206CEFF71CF95FF478
:1094800080000021EFF70CF9206CF1F7C5FE1622E1
:1094900009A9F0F766FF09A80090236CBC4A1621C1
:1094A00003A8F3F7B0F903A90020F4F7E7FD0320C0
:1094B000F4F7AFFD0120F4F704FE0121206CF1F771
:1094C00089FE05000021206CF1F784FE01950090D3
:1094D00002ABBC4A16210FA8F3F795F90FA901209A
:1094E000F4F7CCFD206CF1F797FE10280DD14FA4B6
:1094F00021000220F4F7C2FD21000320F4F7BEFD95
:1095000021000420F4F7BAFD77E0206CF1F726FE85
:1095100010F0000011F48071002901D1002818D04A
:10952000206C012801D103200AE0206C032801D11E
:10953000012005E0206C052801D1072000E005206E
:109540000090A14BA14A16210DF15200F3F75BF9EF
:1095500006E09D4B9E4A16210DF15200F3F753F998
:1095600094F84000C00702D4256C6D1E01E0256C04
:109570006D1C206CF1F7F2FD10F0000011F080017D
:10958000002901D1002807D00095924B924A16215C
:109590001AA8F3F738F905E08E4B904A16211AA85D
:1095A000F3F731F9256C0835206CF1F7D7FD10F091
:1095B000000011F04001002901D1002808D00095D9
:1095C000874B884A16210DF17E00F3F71CF906E05F
:1095D000834B854A16210DF17E00F3F714F90DF146
:1095E00052010220F4F74AFD1AA90320F4F746FDC0
:1095F0000DF17E010420F4F741FD0CA421000620AA
:10960000F4F73CFD21000720F4F738FD2100082085
:10961000F4F734FD0020F4F700FD0820F5F76DFEA7
:10962000002801D0F5F7D9FC25B030BD00000000BE
:1096300038B58EB00400206CEFF73DF85FF4800081
:109640000021EFF72DF8206CF1F7E6FD162202A9B4
:10965000F0F787FE02A80090236C4D4A162108A857
:10966000F3F7D1F808A90020F4F708FD236C5F4A4E
:10967000162102A8F3F7C7F802A90020F4F7FEFCB0
:10968000206B002805D11622594902A8F2F760FF85
:109690000DE0206B012805D11622564902A8F2F7E9
:1096A00057FF04E01622544902A8F2F751FF0420A4
:1096B000F4F7AFFC0420F4F704FD0020F4F7ADFC50
:1096C00002A90120F4F7DAFC2BA529000220F4F707
:1096D000D5FC29000320F4F7D1FC29000420F4F77D
:1096E000CDFC29000520F4F7C9FC29000620F4F779
:1096F000C5FC29000720F4F7C1FC29000820F4F775
:10970000BDFC0820F5F7F9FD00281BD0E06B216BAC
:10971000884214D0206C012808D1216B5920F1F720
:10972000A6FC00200821EEF7BBFF08E0216B206CAF
:10973000F1F7A1FD00204FF48061EEF7B1FFF5F7DE
:109740004CFC17E00120F5F7D8FD002802D0F5F712
:1097500044FC0FE0206C012801D1012100E002212E
:10976000002001900120009001230022206BF5F7DA
:10977000C1FC20630FB030BD00000000400030008D
:10978000BCF3010024F50100B8F8010020F6030045
:1097900030F50100C0F8010060D20300C8F80100F4
:1097A00080D20300D0F8010000ED0300D8F80100DA
:1097B00020ED0300E0F80100E0EC0300E8F8010010
:1097C000D8FD01008CF2010080F40300CCF301000D
:1097D0003CF50100A0F4030048F50100F0F8010099
:1097E000ACF40100DCF3010054F5010060F5010068
:1097F00080E6030060E40300E0F5030078B59DB067
:109800000400206CEEF757FF5FF480000021EEF7B4
:1098100047FF206C012807D1DFF8C4339FA216212F
:1098200001A8F2F7F0FF09E0DFF8B4030090236C21
:10983000DFF8B023162101A8F2F7E5FF01A9002007
:10984000F4F71CFCDFF8A023162107A8F2F7DBFFD2
:10985000DFF89833DFF8982316210DF13200F2F784
:10986000D2FFDFF890532B00DFF88C23162112A8CB
:10987000F2F7C9FF2B00DFF8842316210DF15E00FB
:10988000F2F7C1FF0420F5F7E7FA0320F4F7C1FB74
:109890000420F4F716FC0220F5F70DFB0500162650
:1098A00007A806FB05F101440120F4F7E7FB07A830
:1098B00006FB05F1084410F116010220F4F7DEFB67
:1098C00007A806FB05F1084410F12C010320F4F76A
:1098D000D5FB07A87543284410F142010420F4F792
:1098E000CDFB0020F5F7E7FA401CF4F796FB206C5F
:1098F000F1F762FC05000120F5F7FFFC002802D01B
:10990000F5F76BFB39E00820F5F7F7FC002831D0BC
:109910000120F5F7D0FAFF2D29D0002804D101212C
:109920008920F5F702FB22E001280DD101218F20CB
:10993000F5F7FBFAA80702D40120206301E000201C
:109940002063206BE06312E0022808D101219020FF
:10995000F5F7EBFAC5F38200401C206307E0012114
:109960009120F5F7E2FAC5F34210401C2063206B0A
:10997000E06302E00420F5F74AFB1EB070BD38B585
:1099800088B00400206CEEF796FE5FF480000021A2
:10999000EEF786FE206C012806D1914B3FA21621DE
:1099A00002A8F2F730FF07E08D480090236C8D4A43
:1099B000162102A8F2F727FF02A90020F4F75EFBA8
:1099C000206B002805D116228D4902A8F2F7C0FDB0
:1099D00004E016228B4902A8F2F7BAFD0420F4F73E
:1099E00018FB0420F4F76DFB0020F4F716FB02A926
:1099F0000120F4F743FB77A529000220F4F73EFB92
:109A000029000320F4F73AFB29000420F4F736FB81
:109A100029000520F4F732FB29000620F4F72EFB7D
:109A200029000720F4F72AFB29000820F4F726FB79
:109A3000206CF1F7C1FB05000820F5F75EFC00285B
:109A400016D0206BE16B88420FD035F00205206BF9
:109A5000002801D155F002052900206CF1F7B5FB73
:109A600000204FF48061EEF71BFEF5F7B6FA12E026
:109A70000120F5F742FC002802D0F5F7AEFA0AE023
:109A80000020019001200090012300220121206B81
:109A9000F5F730FB206309B030BD000025730000EE
:109AA00070B588B004000D00206CEEF704FE5FF482
:109AB00080000021EEF7F4FD206C012806D1484B10
:109AC00045A2162102A8F2F79EFE07E04448009046
:109AD000236C444A162102A8F2F795FE02A9002041
:109AE000F4F7CCFA236B3DA2162102A8F2F78BFE05
:109AF0000420F4F78EFA0420F4F7E3FA02A9012017
:109B0000F4F7BCFA33A631000220F4F7B7FA3100BB
:109B10000320F4F7B3FA31000420F4F7AFFA310070
:109B20000520F4F7ABFA31000620F4F7A7FA31006C
:109B30000720F4F7A3FA31000820F4F79FFA002079
:109B4000F4F76BFA0820F5F7D8FB00282DD0206B2E
:109B5000E16B884226D0206CF1F72EFB022D0CD150
:109B6000216B491E2163216B490111F0E001216342
:109B700030F0E000216B08430BE0216B491E2163AC
:109B8000216B890011F01C01216330F01C00216B56
:109B900008430100206CF1F718FB00204FF48061AE
:109BA000EEF77EFDF5F719FA12E00120F5F7A5FBB7
:109BB000002802D0F5F711FA0AE0002001900020F9
:109BC0000090012301220421206BF5F793FA206312
:109BD00008B070BD0000000025730000256400007F
:109BE000ACF4010018F5010098F8010040D803001A
:109BF000A0F80100C0D50300A8F80100B0F80100EA
:109C000080E60300E0D9030078B59DB00400702021
